:020000040001F9
:10900000888E00208DA2020093C0010077C101006C
:10901000BFC3010003C4010007C401000000000039
:109020000000000000000000000000000FF7010039
:1090300007F80100000000000B050200E325020014
:109040004B4202001746020019460200F14B020093
:10905000F74B0200B75002002F720200A164020019
:10906000074F02000F4F0200174F02000B5D020076
:109070008394020067970200F79702005F9802004E
:10908000D7990200335B0200979A0200A39E020068
:1090900089A002003FA102003B1202006BA2020065
:1090A000CBA3020009A402000BA402000DA402003D
:1090B0000FA4020011A40200000000000000000044
:1090C00013A4020015A4020017A402003D2402000C
:1090D00019A402001BA402001DA40200000000004D
:1090E0000000000000000000000000000000000080
:1090F0000000000000000000000000000000000070
:10910000000000000000000000000000000000005F
:10911000000000000000000000000000000000004F
:10912000000000000000000000000000000000003F
:10913000000000000000000000000000000000002F
:10914000000000000000000000000000000000001F
:10915000000000000000000000000000000000000F
:1091600000000000000000000000000000000000FF
:1091700000000000000000000000000000000000EF
:1091800000000000000000000000000000000000DF
:1091900000000000000000000000000000000000CF
:1091A00000000000000000000000000000000000BF
:1091B00000000000000000000000000000000000AF
:1091C000000000000000000000000000000000009F
:1091D000000000000000000000000000000000008F
:1091E000000000000000000000000000000000007F
:1091F000000000000000000000000000000000006F
:1092000081B000F5E0700268914203D343681A44CC
:10921000914202D380680028F5D101B07047DFF891
:109220006817086890B94FF4805048604FF4803256
:109230004FF0FF308A60C86008610420DFF84C27D7
:10924000DFF84C374861C2F8BC010B600120704761
:1092500001F1080313F0070F0EBF0023C3F1080349
:1092600003F007031944D21A8161C26042F001037E
:109270004B60091D28238B50DFF80C170A69C26167
:1092800070472DE9FC4B074601F1080010F0070F6D
:109290000FBF8946C0F1080000F0070001EB00098C
:1092A00002F1080111F0070F06D002F10800C0F129
:1092B000080000F0070002441546A5EB090009EB81
:1092C0000306A0EB030B43F00303C9F80430AE42DE
:1092D00028BF01F0FFF92879C10758BF01F0FAF95A
:1092E000BBF1100F38BF01F0F5F9B869854207D11D
:1092F000F8685844F860BE6140F00100706050E1C9
:10930000786985420AD1B8688344C7F808B07E619D
:109310004BF00100706046F80BB042E1686800F065
:109320000301012940F0AB80C008C0000190C008D3
:109330001F2839D8AC68D5F80C800090454508BF87
:1093400001F0C8F9A54208BF01F0C4F968680099A6
:10935000C008C000B0EBC10F18BF01F0BBF9009905
:1093600007F1280000EBC100844206D03A6994421C
:10937000C0F08080E168A9427CD1A04506D1009868
:109380003968012282409143396075E0804506D0FA
:10939000386980456ED3D8F80800A8426AD1C4F86D
:1093A0000C80C8F8084067E0EC68D5F81880AC423B
:1093B0000CD0A8683969884222D3C168A94204BF89
:1093C000A168A9421CD1C460A0601BE005F1140291
:1093D000146834B905F1100214689CB101E01A4612
:1093E000146804F114031968002902BF04F1100382
:1093F00018680028F3D139698A4228BF106001D269
:1094000001F068F9B8F1000F36D0E96907F59870F6
:1094100000EB81000268954208D10460A4B9E869B4
:109420007968012282409143796025E0386980455E
:1094300008D3D8F81000A84214BFC8F81440C8F8E0
:10944000104001E001F046F9B4B139698C4211D302
:10945000C4F81880286928B1884226BF2061846139
:1094600001F038F9686938B13969884202D360611E
:10947000846101E001F02EF901982D188344686899
:109480004008400068604BF0010171604FEADB0466
:1094900046F80BB01F2C23D807F1280000EBC408B6
:1094A0004546BBF1100F38BF01F014F9386820FAB7
:1094B00004F1C90705D4012101FA04F404433C6016
:1094C00007E0D8F80800396988422CBF054601F04A
:1094D00001F9C8F80860EE60B560C6F80C8060E07D
:1094E0005FEA1B2008BF002123D0B0F5803F28BFD2
:1094F0001F211ED2A0F58072120C02F008029040CB
:10950000A0F58051090C01F004018840A0F58043CA
:109510001B0CC2F10E0203F00203521AD21A984039
:1095200002EBD032D01D2BFA00F101F0010101EB6A
:10953000420107F5987202EB8100F161002272612D
:1095400032617A6822FA01F3DB0707D4012303FAB8
:1095500001F1114379600660B0611DE002681F29C6
:109560001DBF4908C1F119010BFA01F1594600E08C
:1095700002465068C008C000584516D002F11003DA
:10958000CC0F03EB8403490018680028F0D1386938
:10959000834204D31E60B261F660B66001E001F060
:1095A00099F809F10800BDE8F68B396990688A429C
:1095B00028BF8842F3D3C6609660B060F260002096
:1095C000B061EEE72DE9FE4F04468B46A5692E46B5
:1095D000904699463146FFF713FEA8F1280201682C
:1095E000406801EB000AAAF1270111F007000EBF45
:1095F0000021C1F1080101F007010AEB0100A0F10F
:109600002F0706F11000874238BF374607F11800D0
:1096100001905946002000902046FFF719FE07F1FF
:10962000080010F0070F18BF01F054F81B207860F5
:1096300007F1080104F5E07090E80C5081E80C5047
:10964000C0F800B0C0F80480C0F80C9081600198A8
:10965000009900E0001D07224260491C00F1080249
:109660005245F7D30129D8BF01F034F8B74200F0D2
:109670009580BF1B301D311DC05940084000C851A6
:1096800047F0010171604FEAD70BF751BBF11F0F93
:1096900021D804EBCB0000F12805A846102F38BFD5
:1096A00001F018F8206820FA0BF1C90705D4012150
:1096B00001FA0BF10843206006E0A868216988429E
:1096C0002CBF804601F006F8AE60C8F80C60C6F802
:1096D0000880F5606FE0380A08BF002123D0B0F59C
:1096E000803F28BF1F211ED2A0F58072120C02F00D
:1096F00008029040A0F58051090C01F00401884057
:10970000A0F580431B0CC2F10E0203F00203521AB3
:10971000D21A984002EBD032D01D27FA00F101F0A6
:10972000010101EB420104EB8102002302F5987074
:10973000F16173613361626822FA01F3DB0707D4D8
:10974000012303FA01F1114361600660B0611DE07D
:1097500002681F291DBF4908C1F1190107FA01F16B
:10976000394600E002465068C008C000B84216D032
:1097700002F11003C80F03EB8003490018680028AA
:10978000F0D12069834204D31E60B261F660B560F7
:1097900011E003B0BDE8F04F00F09CBF0BE0216981
:1097A00090688A4228BF8842F3D3C6609560B06053
:1097B000F2600020B06103B0BDE8F08F2DE9F04108
:1097C000714F05463868884608B9FFF728FDB96823
:1097D00001EB08002F30491E20EA010188457DD2A7
:1097E00005F5D876B06828B1326889188A4275D2F2
:1097F000884273D300F0AEFF01001CBF0C6811F16A
:10980000010F6BD03068201805F5D87230605368AE
:10981000984238BF18467060A86960BB286908B1D3
:10982000814200D22961316174610020F06105F14B
:109830002802386868624FF0FF3028620020D2604A
:10984000926002F1080353611361801C10322028DA
:10985000F5D34E48854208BFA4F1280228D055F818
:10986000040CC00805EBC002A2F108000A19121A84
:10987000283A01461CE005F5E070024600E09268D7
:109880007AB3136857683B449942F8D1137B1F079A
:1098900027D4AB691768BB4223D3D2F804C067440E
:1098A000BB421ED2A444C2F804C0E868A9692218C9
:1098B0002846FFF7CDFC1FE08068C0B103689342E3
:1098C000FAD1027B130712D4026801604368E418DE
:1098D000446043462846BDE8F041D2E40020BDE89C
:1098E000F0812A69914238BF29610A19E5E700230E
:1098F00022462846FFF766FEE8688045EED2A0EBD8
:109900000800A969E86001EB0802AA6140F00100C3
:10991000506048F00300486001F10800BDE8F081A4
:1099200038B4194B1A6882B94FF480525A604FF418
:1099300080344FF0FF329C60DA601A610422134CCD
:10994000134D5A61C4F8BC211D6011F1400F17D2AC
:109950008269AAB1C368283199420BD200F5E0713F
:109960000C68A24203D34D682C44A24202D38968FA
:109970000029F5D1C16999423CBF4FF0FF31C16167
:1099800032BC002070470000305D002050540020A1
:109990006859883C2DE9F84F00258946090AC9F124
:1099A000000B08BF002323D0B1F5803F28BF1F2341
:1099B0001ED2A1F58072120C02F008029140A1F5AE
:1099C00080531B0C03F004039940A1F58044240C40
:1099D000C2F10E0204F00204D21A121BA14002EBE3
:1099E000D132D11D29FA01F303F0010303EB420345
:1099F000074607F5987858F8230030B31F2B0FBFA0
:109A00004C465C08C4F1190409FA04F4AC46594602
:109A100000E064004268D208D200A2EB09028A4248
:109A200003D21100054600F06881426910304FEA08
:109A3000D47B50F82B00002A1CBF82429446002899
:109A4000E7D18B466046B0BBBDBB012000FA03F3F3
:109A50005B00584203437868034000F04D81584250
:109A600003405B1E180B00F01000C340590901F0C1
:109A70000801CB409A0802F00402D3405C0804F0CD
:109A800002040818E3401018C3F3400620183044BD
:109A9000F3401B1858F823000DE008464168C90838
:109AA000C900A1EB090159453CBF8B460546016938
:109AB0000029F2D140690028F0D1002D00F01C816E
:109AC000B868A0EB0900834580F0168138698542AB
:109AD000C0F010816868C008C00009EB0B01884223
:109AE00018BF00F0F7FD05EB0906B54280F00281D2
:109AF000EC68D5F818A0AC420CD0A8683969884247
:109B000022D3C168A94204BFA168A9421CD1C46084
:109B1000A0601BE005F11402146834B905F11002CD
:109B200014689CB101E01A46146804F11403196822
:109B3000002902BF04F1100318680028F3D1396925
:109B40008A4228BF106001D200F0C4FDBAF1000FB4
:109B500036D0E96908EB81000268954209D10460BA
:109B6000200014D1E869796801228240914379602C
:109B700026E03869824508D3DAF81000A84214BFFD
:109B8000CAF81440CAF8104001E000F0A3FDBCB1CF
:109B90003869844212D3C4F818A0286930B13969F1
:109BA000884226BF2061846100F094FD686938B165
:109BB0003969884202D36061846101E000F08AFD66
:109BC000BBF1100F0CD2D94449F003006860291D85
:109BD000281D50F8090040F0010041F8090088E014
:109BE00049F0030068604BF0010070604FEADB0051
:109BF00046F80BB01F281DD807EBC00101F128045F
:109C0000396821FA00F2D207A34605D4012202FAEC
:109C100000F00843386006E0A068396988422CBF2C
:109C2000834600F057FDA660CBF80C60C6F808B07C
:109C3000F4605EE05FEA1B2008BF002123D0B0F58E
:109C4000803F28BF1F211ED2A0F58072120C02F0A7
:109C500008029040A0F58051090C01F004018840F1
:109C6000A0F580431B0CC2F10E0203F00203521A4E
:109C7000D21A984002EBD032D01D2BFA00F101F03D
:109C8000010101EB4201F16100227261326108EBD6
:109C900081007A6822FA01F3DB0707D4012303FA73
:109CA00001F1114379600660B0611DE002681F296F
:109CB0001DBF4908C1F119010BFA01F1594600E035
:109CC00002465068C008C000584518D002F1100381
:109CD000CC0F03EB8403490018680028F0D13869E1
:109CE000834204D31E60B261F660B66001E000F00A
:109CF000F1FC13E100F0EEFC0DE18B46A3E63969BF
:109D000090688A4228BF8842F1D3C6609660B060EE
:109D1000F2600020B061ECE72DE9F84F0646884676
:109D2000716848420140491E080B00F01000C14014
:109D30004A0902F00802D1408B0803F00403D9401D
:109D40004D0805F002051018E9401818C1F3400449
:109D5000281806F5987A2044E14009185AF821108D
:109D60004868C008C0000D46A0EB080909E001469C
:109D70004868C008C000A0EB080048453CBF8146C9
:109D80000D4608690028F2D149690029F0D13069EF
:109D90008542C0F0BE806868C00808EB090BC000AF
:109DA000584518BF00F096FC05EB0800854200906E
:109DB00080F0AF80EF68AC69AF420CD0A868316921
:109DC000884222D3C168A94204BFB968A9421CD104
:109DD000C760B8601BE005F11402176837B905F1D8
:109DE000100217689FB101E01A46176807F11403C3
:109DF0001968002902BF07F1100318680028F3D181
:109E000031698A4228BF106001D200F063FC002C47
:109E100031D0E9690AEB81000268954208D10760F8
:109E20008FB9E8697168012282409143716022E034
:109E30003069844205D32069A84214BF6761276155
:109E400001E000F047FCB7B13069874211D3BC6133
:109E5000286930B13169884226BF3861876100F0D6
:109E600039FC686938B13169884202D37861876109
:109E700001E000F02FFCB9F1100F0BD24BF0030002
:109E80006860291D281D50F80B0040F0010041F8C2
:109E90000B003DE048F00301696049F00100291D15
:109EA00041F80800009840F80990D6F808804FEA79
:109EB000D80BBBF1200F28BF00F00CFCB8F1000F4D
:109EC00022D006EBCB00776900F12804A246B8F156
:109ED000100F38BF00F0FEFB306820FA0BF1C90705
:109EE00005D4012101FA0BF10843306006E0A068B7
:109EF000316988422CBF824600F0ECFBA760CAF8AB
:109F00000C70C7F808A0FC60C6F808900098706153
:109F100004E000F0DFFB0020BDE8F28F05F108004F
:109F2000BDE8F28F2DE9FE4F0546AFF30080F52D19
:109F3000DFF89C6780F004810B2D31BF10250B35B5
:109F4000ED08ED003068EC08E04010F0030F46D05B
:109F5000C04300F00100041906F1280000EBC4081A
:109F6000E700D8F808506868C008C000B84218BFB9
:109F700000F0B0FBD5F80890454508BF00F0AAFBFB
:109F80004D4508BF00F0A6FB6868C008C000B84295
:109F900018BF00F09FFBC84507D13168012000FAC7
:109FA00004F421EA040434600DE03069814508D3EB
:109FB000D9F80C00A84204D1C8F80890C9F80C8060
:109FC00001E000F087FB47F003006860291D281DB1
:109FD00005F10804C05940F00100C851F8E0B1682B
:109FE000A94280F0BE80002800F0A1804FF0010857
:109FF00008FA04F1490000FA04F4484201430C4015
:10A0000060420440641E200B00F01000C44061094F
:10A0100001F00801CC40A20802F00402D440630819
:10A0200003F002030818DC401018C4F340071818A6
:10A030003818FC40241806F1280000EBC40AE70099
:10A04000DAF80890D9F80400C008C000B84218BF78
:10A0500000F040FBD9F808B0D14508BF00F03AFB4A
:10A06000D94508BF00F036FBD9F80400C008C0008D
:10A07000B84218BF00F02EFBDA4506D1316808FA65
:10A0800004F421EA040434600DE03069834508D308
:10A09000DBF80C00484504D1CAF808B0CBF80CA096
:10A0A00001E000F017FB45F00300C9F804007F1B36
:10A0B00009F1040147F00100485109EB0500019046
:10A0C000C751B4684FEAD40ABAF1200F28BF00F094
:10A0D00001FB34B3CDF800A006F12800756900EB50
:10A0E000CA0AD346102C38BF00F0F4FA3168009841
:10A0F00021FA00F2D30704D408FA00F008433060D4
:10A1000007E0DAF80800316988422CBF834600F086
:10A11000E1FACAF80850CBF80C50C5F808B0C5F8F9
:10A120000CA0B76009F108040198706150E07068F4
:10A13000C0B329463046FFF7EFFD040011D047E0D9
:10A1400015F1400F28BF4FF0FF350AD20B35ED084F
:10A150007068ED0028B129463046FFF71BFC04006B
:10A1600036D1B068A8421DD3411B726910290AD3A9
:10A1700050197061B16041F001034360415045F0F6
:10A18000030555600BE00021B1607161131D40F0C3
:10A1900003015160111D095841F00101195002F1EC
:10A1A000080415E0F06885420DD2401BB169F060EB
:10A1B0004A19B26140F00100506045F003054D605E
:10A1C00001F1080404E029463046FFF7F7FA044697
:10A1D000AFF300802046FFF7EEBA002800D17047A9
:10A1E0002DE9FC47A0F10805AFF30080DFF8E0643B
:10A1F00032699542C0F05982686800F00301012974
:10A2000000F05382C1084FEAC109C10705EB0908F4
:10A2100039D42C6810F0030F00F0498260420544E5
:10A220009542A144C0F041827069854200F0C78028
:10A23000E408202C5ED2D5F80CA0AF68554508BFC5
:10A2400000F048FABD4208BF00F044FA6868C00850
:10A25000C000B0EBC40F18BF00F03CFA06F12800B4
:10A2600000EBC400874205D031698F423FD3F968C3
:10A27000A9423CD1BA452CD13068012101FA04F43D
:10A2800020EA04043460454580F00F82D8F8044089
:10A29000E00740F10A82A00700F16881B0698045BB
:10A2A00040F0A080F068B5618144C6F80C9049F098
:10A2B000010068607069854202D100207061B06061
:10A2C000F069484580F0F38100213046FFF728FB14
:10A2D000EDE1824506D03069824508D3DAF80800FE
:10A2E000A84204D1C7F80CA0CAF80870CBE700F068
:10A2F000F1F9C8E7EC68AF69AC420BD0A8689042AE
:10A3000023D3C168A94204BFA168A9421DD1C4607A
:10A31000A0601CE005F114031C6834B905F11003BA
:10A320001C68A4B101E063461C6804F1140CDCF85D
:10A330000010002902BF04F1100CDCF80000002816
:10A34000F1D1934228BF196001D200F0C3F9002F68
:10A3500099D0E96906F5987000EB81000268954292
:10A3600009D10460200011D1E8697168012282409E
:10A370009143716087E73069874205D33869A84205
:10A3800014BF7C613C6101E000F0A4F9002C3FF4B3
:10A390007AAF31698C42AAD3A761286928B1884273
:10A3A00026BF2061846100F095F9686900283FF4B8
:10A3B0006AAF316988429AD36061846163E798F833
:10A3C000040000F0030003287FF45DAFC6F8089096
:10A3D00049F00101D8F8040040084000C8F8040022
:10A3E00069600AE0706980450AD1B068756181448E
:10A3F000C6F8089049F00100686045F8099056E1F8
:10A40000E408E400A144E408202C3AD2D8F80CA0D7
:10A41000D8F80870D04508BF00F05CF9B84508BF0F
:10A4200000F058F9D8F80400C008C000B0EBC40F21
:10A4300018BF00F04FF906F1280000EBC400874276
:10A4400007D031698F42C0F08480F968414540F0FF
:10A450008080BA4507D13068012101FA04F420EA6E
:10A460000404346077E0824506D031698A4570D3B0
:10A47000DAF8080040456CD1C7F80CA0CAF808709B
:10A4800069E0D8F80C40D8F8187044450DD0D8F8D9
:10A4900008003169884222D3C168414504BFA168E0
:10A4A00041451CD1C460A0601BE008F1140214688F
:10A4B00034B908F1100214689CB101E01A4614681E
:10A4C00004F114031968002902BF04F1100318688D
:10A4D0000028F3D131698A4228BF106001D200F010
:10A4E000F9F8002F37D0D8F81C1006F5987000EB5B
:10A4F0008100026890450AD10460200012D1D8F88A
:10A500001C007168012282409143716023E0306930
:10A51000874205D33869404514BF7C613C6101E046
:10A5200000F0D8F8BCB131698C4212D3A761D8F8D9
:10A53000100028B1884226BF2061846100F0CAF86B
:10A54000D8F8140038B13169884202D3606184615F
:10A5500001E000F0BFF849F00100686045F809909B
:10A56000706985420BD1C6F80890A0E064086400C9
:10A57000C8F8044049F00100686045F809904FEAC6
:10A58000D907202F22D206F1280000EBC704A046ED
:10A59000B9F1100F38BF00F09DF8306820FA07F1CC
:10A5A000C90705D4012101FA07F70743376006E020
:10A5B000A068316988422CBF804600F08BF8A56006
:10A5C000C8F80C50C5F80880EC6070E05FEA19200C
:10A5D00008BF002123D0B0F5803F28BF1F211ED225
:10A5E000A0F58072120C02F008029040A0F5805194
:10A5F000090C01F004018840A0F580431B0CC2F156
:10A600000E0203F00203521AD21A984002EBD03223
:10A61000D01D29FA00F101F0010101EB420106F51C
:10A62000987202EB810000226A612A61E961726816
:10A6300022FA01F3DB0707D4012303FA01F11143E6
:10A6400071600560A8611DE002681F291DBF4908EF
:10A65000C1F1190109FA01F1494600E002465068CA
:10A66000C008C000484526D002F11003CC0F03EB10
:10A670008403490018680028F0D13069834204D36C
:10A680001D60AA61ED60AD6001E000F023F8306A62
:10A69000401E30620BD1D6F8C80100E08068002867
:10A6A000FCD14FF0FF30306201E000F013F8AFF35F
:10A6B0000080BDE8F387316990688A4228BF8842EC
:10A6C000E3D3C5609560A860EA600020A861DEE77A
:10A6D00050540020012000F053B8F0B40246106836
:10A6E00095681318506803EB5004C00721D54D44FA
:10A6F0001FE0F0BC02F10C00704713F8017B05F875
:10A70000017B491EF9D1A0B1B60813F8011B06F070
:10A710000306032E08BF13F8016B01EB0621494223
:10A72000801C294405D011F8016B05F8016B401E0F
:10A73000F9D1A342DDD013F8016B16F0030104BF79
:10A7400013F8011BC91C30090F28DAD113F8010BCB
:10A750000F30D6E70749086808B10020704706485F
:10A76000C008C00008600549C908C900091A01608D
:10A77000704700BF6C5E00208F8E002088AE0020E6
:10A780002021090326311820ABBEF9E72DE9F84F47
:10A7900074A7A2B0D7E90045CDE900452C9EDFF8AB
:10A7A000307C04918DF843605FF000016FA40D913F
:10A7B00012944FF0FF368246904699460FE0C3460A
:10A7C0002C461BF8011B0498D0470028049000F089
:10A7D000B2800D98401C641E0D90F2D1A84498F8E8
:10A7E0000000252807D100210791089109910A91BD
:10A7F0000B910C910DE06A463146404600F0F4FFA3
:10A80000050001D10D98B5E0D9D50125E6E741F065
:10A81000010118F8010F2028F9D023280CD02B288B
:10A8200004D02D2805D0302809D086E041F002015F
:10A83000EFE741F00401ECE741F00801E9E741F0FE
:10A840001001E6E700200F900AE00F98B84205DA01
:10A8500000EB800302EB4302303A0F9208F101084B
:10A8600098F80020A2F130000A28EED398F80000F2
:10A870002E2818BF0E9629D118F8010F2A280BD1BF
:10A88000D9F80000C9F8000008F1010850F8042BBD
:10A89000C9F800000E9219E02D280CBF18F8010B22
:10A8A000002000220E920BE040B90E9ABA4205DA5F
:10A8B00002EB820403EB4403303B0E9308F10108E2
:10A8C00098F80030A3F130020A2AEDD3ADF8401019
:10A8D000129898F8001000F091FF08B118F8010BD9
:10A8E0008DF842009DF84200682804BF98F80010D7
:10A8F000682903D162208DF8420008E06C2804BF6B
:10A9000098F800006C2804D171218DF8421008F1EC
:10A91000010813A806904A4618F8013B02A95046C0
:10A9200000F068F838B913AA02A9504600F0CAF935
:10A9300000287FF554AF30461CE02A2882D1D9F890
:10A940000020C9F8002052F8040BC9F800200028A4
:10A950000F9003D540420F9041F0040108F1010827
:10A9600084E700000000000000000000686A6C74CA
:10A970007A4C000023B0BDE8F08F622820D0682810
:10A9800011D06A2803D06C2827D0712825D10868F7
:10A99000C01D20F007000860D0E9002308300860DF
:10A9A000194610467047002A0A680A60106803D0EA
:10A9B000121D0A6000B217E0121D0A6080B217E093
:10A9C000002A0A680A60106803D0121D0A6040B2AB
:10A9D0000AE0121D0A60C0B20AE0002A0A680A6092
:10A9E000106803D0121D0A60C1177047121D0A605B
:10A9F000002170477CB50D4611461C462E69B4F106
:10AA0000250200F04D811C3A00F08680121F022AB8
:10AA100040F282800E3A00F00781521F5AD0093A64
:10AA20007AD0921E16D0521E35D0521E022A73D9E9
:10AA3000121F30D0521F00F09A80521E4AD0521E70
:10AA400000F0E480D21E00F0FD80921E42D0D21EA3
:10AA500040D02BE195F83A206C2A09D06869421C55
:10AA60006A610A680A6052F8043B0A60335427E1BD
:10AA70000A680A6052F8043B0A60002100930191C1
:10AA80004FF0FF322A6329466A4600F096F9002803
:10AA900040F1168101E195F83A000122FFF76DFFC0
:10AAA000C5E900010023994204DA6869411C696123
:10AAB0002D210DE0288F810704D56869411C69614B
:10AAC0002B2105E0C00722D56869411C696120215E
:10AAD00031541CE095F83A000022FFF74EFFC5E91B
:10AAE000000195F83800010711D5D5E900230020B1
:10AAF000834208BF82420AD044F02000782806D161
:10AB0000686930213154401C411C6961345421462C
:10AB100068693044E86083E00868C01D20F00700E1
:10AB20000860D0E9002308300860C5E90023D5E9B2
:10AB30000001C80F04D06869411C69612D210DE036
:10AB4000288F810704D56869411C69612B2105E0C4
:10AB5000C00704D56869411C6961202131546869C6
:10AB60003044E8602146284600F032FAA8E005F1BA
:10AB70003A02507820B14FF0FF340FF6243070E0E5
:10AB80001078622808D0682824D06A2812D06C284F
:10AB90002ED071280ED02BE00A680A6052F8040B00
:10ABA0000A6020B94FF0FF340FF60C3059E0E96A23
:10ABB000017085E00A680A6052F8040B0A6020B947
:10ABC0004FF0FF340FF6F0204BE0EA6AD317C0E9EC
:10ABD000002375E00A680A6052F8040B0A6020B985
:10ABE0004FF0FF340FF6D0203BE0E96A018067E0C8
:10ABF0000A680A6052F8040B0A6020B94FF0FF346B
:10AC00000FF6B4202DE0E96A016059E00A680A6095
:10AC100052F8040B0A600021C5E90001EE607821BA
:10AC2000284600F029F94BE06C2285F83A200B68A1
:10AC30000B6053F8042B0B6052BB4FF0FF340FF640
:10AC4000AC200EE095F83A206C2AF0D00868086035
:10AC500050F8044B0860EC603CB94FF0FF340FF63D
:10AC6000702000F0E9FD201A76BD2E6B002E04D571
:10AC7000204600F001FE044608E03246002120464E
:10AC800000F024FE002814BF041B3446AC6117E01A
:10AC9000294600F092F8002812D54FF0FF3076BD1B
:10ACA0006869411C69612521315409E06969481CC2
:10ACB000686125227254210002D0411C696134541C
:10ACC000002076BD2DE9F0410E460546716B706996
:10ACD000B46A091A306A091AB069091A706A091A3D
:10ACE000F069091A96F838000C1B410790460DD4FC
:10ACF000002C0BDD2746B0682021A8470028B06053
:10AD000057D0F06A401C7F1EF062F4D1736942464E
:10AD10003146284600F0ACFC00284AD1376A002FA3
:10AD20000ADDB0683021A8470028B06041D0F06A41
:10AD3000401C7F1EF062F4D1B369F26831462846A8
:10AD400000F096FCA8BB776A002F09DDB0683021BF
:10AD5000A847B06068B3F06A401C7F1EF062F5D16E
:10AD6000F068B169F36942183146284600F080FC6A
:10AD7000F8B9B76A002F09DDB0683021A847B06084
:10AD8000B8B1F06A401C7F1EF062F5D196F8380029
:10AD900041070BD5002C09DDB0682021A847B06021
:10ADA00038B1F06A401C641EF062F5D10020BDE8A5
:10ADB000F0814FF0FF30BDE8F0812DE9F8470D46F6
:10ADC000A3B02F6B002F8146904648BF6FF000471D
:10ADD00000F0A8FD696B40180FF62C118128D1E90D
:10ADE0000023CDE9012328BF4FF0FF303ED20024DD
:10ADF000002F2FDDD8F8001001AA684600F0F6FCFD
:10AE00000646002E35D4D8F8000008B9761E30D496
:10AE1000B7421FDB6869301881280AD300206863B5
:10AE200003AA29464846FFF74DFF040012D400202C
:10AE3000686103A8D5F814A032466946504400F072
:10AE400085FDB244C5F814A058F8040B002818BFBB
:10AE5000BF1BCDD12CB903AA29464846FFF732FFC4
:10AE6000044614B9002068616863204624B0BDE838
:10AE7000F0874FF0FF34F8E72DE9FC4707468A4694
:10AE80003E69BAF16F0F08BF082405D04AF02001CF
:10AE9000782914BF0A2410243C25D7E90023BAF1ED
:10AEA000640F18BFBAF1690F9046994606D1002188
:10AEB0008B4203DAD8F1000869EB4909002081458B
:10AEC00008BF80451FD1386BE8B9082C4CD197F8E2
:10AED0003800010748D530203B2586F83B0043E089
:10AEE00000280ED597F8380000F01400102808D17B
:10AEF0007A6B7869121A386A121A511A0029C8BF77
:10AF00003962BDE8F3878DF800A0404649462246E5
:10AF1000E31700F07BFD3032D0B26D1E3A28019568
:10AF200004DB9DF80000A0F151018A1872554046DB
:10AF300049462246E31700F069FD80468946002015
:10AF4000814508BF804503D0F86871198842DCD379
:10AF5000082C09D197F83800010705D5715D302913
:10AF600002D06D1E30207055C5F13C01B9617019D9
:10AF7000F860386B8142B3DA411A39624FF6EF70EC
:10AF8000398F01403987BDE8F3872DE9D043064664
:10AF90000F4614464FF00008DFF8389412E0E0073F
:10AFA00007D542464B463046394600F04FFE06462E
:10AFB0000F464046494642464B4600F047FE641065
:10AFC00080468946002CEAD130463946BDE8D08318
:10AFD0002DE9F34F054641F020048DB0D5E90089F5
:10AFE000612C02AE09D0286B002848BF062003D48C
:10AFF00008BF672C01D101202863D5E90023580040
:10B000004015401C0ED119030CD00320A8619DF8F7
:10B01000380061381A2802D20FF2F46111E00FF201
:10B02000F4610EE058004015401C0FD119030DD1FA
:10B030000320A8619DF8380061381A2814D30FF254
:10B04000DC61E868032200F081FCD3E1194621F0BD
:10B050000043B3F5801F10460DD20027BB4208BF46
:10B06000BA42019703D111E00FF2AC61E9E701AAFE
:10B0700000F0C6FE0AE0DFF8607307EB1352DFF85A
:10B080005C3301921940DFF858331943C5E90001D8
:10B09000612C0ED1E86830210170811CE9609DF8B7
:10B0A000381061290CBF7821582141706869801CD3
:10B0B0006861D5E900AB2BF0004300202AF00002C4
:10B0C000834204BF8242002300F05A81612C40F089
:10B0D000A980286B00284CBF2120401C00904046CE
:10B0E000009F7F1C49460022002300F0C1FED94684
:10B0F00001988DF8082038BF89F00049001F0190A1
:10B10000002FD0460DF1090040F3498140F2FF7154
:10B11000DFF8D0B20C910646404649460022002393
:10B1200000F0C4FE80F03A814800400D00F11C029E
:10B1300010D0002A0EDD0C98824205DB09F0004099
:10B1400040EA0B01002013E0A448084040EA025105
:10B1500040460DE029F00043002028F00002834221
:10B1600008BF82420FBF40461C22404600F0BCFE92
:10B170008046894600F05AFFFF1F002F044609DD74
:10B1800000F076FF02460B464046494600F082FF3B
:10B1900080468946F01D072104E004F00F0200F804
:10B1A000012D2411002C01DD491EF6D5491E5CBF7E
:10B1B000002200F8012DF9D5ECE00020194602AA82
:10B1C0000A4400E05B1E12F80149491E8442F9D08E
:10B1D0000F2804D10DF10900425C521C4254002991
:10B1E00004D50198001D02AE5B1C0190591E12D4BB
:10B1F0009DF838007218147804F130085FFA88F46A
:10B20000392CC4BFA0F13A04A044491E02F80189B8
:10B21000F1D58DF83800286B002840F1B080591E18
:10B220002963ACE0404649460022002300F020FE9E
:10B23000019938BF89F0004947F2975041436A4A63
:10B2400091FBF2F20192D2F1070204DD4046494639
:10B25000FFF79BFE0AE0524200206449FFF795FE8B
:10B2600002460B464046494600F086FF8046662C63
:10B27000286BDFF87CB106BF019F0A3706273F180D
:10B28000142FC8BF142730208DF8080089460DF10F
:10B29000090000E03046002F34DD064640464946AE
:10B2A00001F08EF801460A4606F1080304200A263A
:10B2B000B2FBF6F606EB860EA2EB4E02303203F836
:10B2C000012C0A22B6FBF2F202EB820EA6EB4E062E
:10B2D0003036401E03F8026DE9D1083F002F03F11C
:10B2E0000806D7DD084601F07FF802460B464046C7
:10B2F000494600F0CFFE00225B4600F0A7FC8046E6
:10B300008946CBE70DF10901401A0DF1090604E069
:10B310000199491E401E0191761C31783029F7D0E1
:10B32000662C02D10199491C03E0652C0CBF012158
:10B3300000212B6BCB189842B8BF431E002B1ED4A4
:10B34000834204DAF05C3528A8BF392000DA3020C7
:10B350001946721E02EB010800E05B1E18F8019905
:10B36000491E8145F9D0392802D1705C401C7054C7
:10B37000002904D50198401C16465B1C01900198D9
:10B3800000B200901BB29DF838103246284600F0FB
:10B3900035F82FE0C61D002F3FF7BEAE30460DF149
:10B3A0000901401A009903468842C8BF0B46002B8A
:10B3B0000DF109063FF52FAF8342BFF6FEAE0DF14A
:10B3C0000900C05C07287FF7F8AE0F20F6E6000002
:10B3D000CBCCCC0C0000244002FCFFFFFFFF0F8011
:10B3E0000000E03F0000F07FA08601000000F03F79
:10B3F00084D797410FB0BDE8F08F00002DE9F847E2
:10B4000083B006468A461746984600F0F1F9B8F12F
:10B41000000F406A356B90F8009002DC4FF0010895
:10B42000BFA7BDF930404AF02000662808BF641C61
:10B4300015D0672840F0848014F1040FC0F2868094
:10B44000AC4280F2838096F83800641C010702D475
:10B45000A845B8BF454620B22D1A48BF00250FFAAF
:10B4600084FAF068B169BAF1000F25DC4A1C302378
:10B470004354002D03DC96F83800010703D5F0682B
:10B4800000F80290521C15EB0A0FB8BF6C4220B2B4
:10B49000441941424445B8BFA046B26171620FFAF7
:10B4A00088F5F561F068B3692A463946184400F01A
:10B4B0004DFA641BB462C4E022B29045084417DA26
:10B4C0004246394600F042FAB0694044B061AAEB06
:10B4D0000801002D716203DC96F838100A0705D5C3
:10B4E000F16801F80090F069401CF061B562A8E0D5
:10B4F000394600F02BFAB069002D5044A8EB04083F
:10B5000003DC96F838100A0703D5F16801F80090BB
:10B51000401CB0610FFA88F08542F068B369B8BF8B
:10B52000A8460FFA88F207EB0A01184400F00EFA59
:10B53000B0690FFA88F10844B061681A706280E05F
:10B54000BAF1610F14D14FF0700A16E0A84504DA81
:10B5500096F838100A0758BF45466D1E48BF0025AB
:10B56000BAF1670F14BF4FF0450A4FF0650A04E0C7
:10B57000BAF1410F08BF4FF0500AB169F368481C97
:10B58000B061002D17F8012B5A5403DC96F83810DF
:10B590000A071BD5F168431CB36101F80090002D28
:10B5A00014DDA8F101080FFA88F08542F068B8BFF1
:10B5B000A8460FFA88F23946184400F0C7F9B06976
:10B5C0000FFA88F108446D1AB0617562F068B169CC
:10B5D0000844002C80F800A003D42B214170811C6A
:10B5E00003E02D2141706442811C00206A460AE07C
:10B5F00023460A2493FBF4F404EB8405A3EB4503F0
:10B6000002F8013B401C24B2002CF1DC012806DCCE
:10B610004AF02002652A04BF302201F8012B48B904
:10B62000302001F8010B07E0401E1DF800203032E9
:10B6300001F8012B0028F7DCF068B2691044091A00
:10B64000F16196F8380000F0140010280DD17169EE
:10B65000B0694118706A4118F0694118B06A411820
:10B66000706B8142BCBF411A316204B0BDE8F08703
:10B67000F8B505460E4617461C46002074B117F86B
:10B68000011BB068A847B06030B1F06A401CF0629E
:10B690000020641EF3D1F2BD4FF0FF30F2BD000078
:10B6A0007072696E74665F733A20256E20646973E8
:10B6B000616C6C6F776564007072696E74663A20B5
:10B6C00062616420256E20617267756D656E74001D
:10B6D0007072696E74665F733A20626164202573CC
:10B6E00020617267756D656E740000007072696E1E
:10B6F00074665F733A2062616420256C7320617206
:10B7000067756D656E7400000000000000000000A9
:10B710006E616E004E414E00696E6600494E4600F5
:10B7200030000B78012B70B505460C460AD14068F5
:10B730004E6803687168DB6898476868036831463B
:10B74000DB689847002368686360C4E904332370AA
:10B7500003682146DB68BDE870401847FFE74138C1
:10B760001A288041C00F7047A0F10901052901D3B3
:10B77000202801D10120704700207047A0F141012D
:10B780001A2938BF203070471A48704730B45368C0
:10B79000D418042B09DA41B1057804F8015B10F8DC
:10B7A000015B15B15B1C491EF3E7536030BC704769
:10B7B00038B514461D4661B1FFF7E8FF61686A6B52
:10B7C000204690476FF00102811A02D0491E03D033
:10B7D00005E06FF0010032BD4FF0FF3032BD0021B7
:10B7E000616032BDDA6B1047024BE1E7014BF9E7CC
:10B7F00001487047943700205C3700200278C9B2B6
:10B800008A421AB11CBF10F8012FF9E718BF0020B7
:10B81000704700F5805210B55368B3F5806F09DAB0
:10B82000946800EB830021440133446091605360CD
:10B83000002010BD0120FCE780B500B906A0054935
:10B840000B681BB122220021984701E0FEF742FF5E
:10B85000222002BD705E0020636F6E737472616996
:10B860006E742068616E646C65723A206261642057
:10B870006D6573736167650000F10103810704D092
:10B8800010F8011B89B18107FAD10268B2F10131C8
:10B89000914311F0803F04BF50F8042FF6E710F8F1
:10B8A000011B11B110F8011BFBE7C01A7047B1F57D
:10B8B000807F02D34FF0FF30704701700120704746
:10B8C0000078401E8041C043C00F7047C9B2830753
:10B8D00006D0521E22D310F8013B9942F7D11FE047
:10B8E000083A13D302F1040241EA012141EA01417D
:10B8F00050F8043B121F21BF4B40A3F1013C2CEA3E
:10B90000030C1CF0803FF3D0C9B2001F083210F8BE
:10B91000013B521E28BF91EA030FF8D818BF01203F
:10B92000401E704780B5FFF72FFF006C02BD002955
:10B930000ADB00F580535B688B4205DD00EB81007C
:10B9400043681360002070470120704762B38B0783
:10B9500008D0521E11F8013B00F8013B00F0248092
:10B960008B07F6D1830740F0208000BF103A07D341
:10B9700030B4B1E83810103AA0E83810F9D230BC31
:10B98000530724BFB1E80810A0E8081044BF51F8DD
:10B99000043B40F8043BD20724BF31F8022B20F8C7
:10B9A000022B44BF0B7803707047121F17D35B0044
:10B9B00009D151F8043B20F8023B1B0C121F20F860
:10B9C000023BF6D20BE051F8043B00F8013B1B0AA6
:10B9D00020F8023B1B0C121F00F8013BF3D238BFCA
:10B9E000121D521E24BF11F8013B00F8013BF8D88C
:10B9F00070478268521C8260426832B10268531CF0
:10BA0000036011704168491E41607047B3BBD9B1F2
:10BA1000B2F5803F7DD2022A1ED98C46B1FBF2F1ED
:10BA200002FB11C31B0443EA1043B3FBF2FC02FB0D
:10BA30001C3380B240EA0343B3FBF2F002FB103246
:10BA400040EA0C4000237047022A05D98446B0FB27
:10BA5000F2F002FB10C270474AB105D100F00102BA
:10BA600049085FEA3000704700220023704700F069
:10BA7000C9BC0B000200002100207047904271EB0E
:10BA8000030CF6D3B3F5803F2FD2F0B5B3FA83F7AA
:10BA9000B1FA81F4A7F10F0E3D1B5340CEF1200601
:10BAA00002FA0EF2F3415340B5F10F0746D80F3CAE
:10BAB0002C444140C4F12006A040F1414140B1FB7B
:10BAC000F3F603FB1611A2FB0645001BA94102D2A7
:10BAD000761E8018594180EA010221FA0EF362FABB
:10BAE0000EF200215A403046F0BD30B4B1FBF3FCF9
:10BAF00003FB1C11A2FB0C45001BA94103D2ACF1B6
:10BB0000010C8018594130BC02460B4660460021AA
:10BB10007047B2F1807F65D3F0B5B2FA82F7B1FA1F
:10BB200081F4C7F10F063D1B22FA06F307F1110E4F
:10BB3000F24120355A40B5F10F07B8D94140C4F160
:10BB40002006A040F1414140B1FBF3FC03FB1C1176
:10BB5000A2FB0C45001BA94103D2BCF1010C8018CB
:10BB600059410F2F12D30F3FC90341EA5041B1FB96
:10BB7000F3F603FB1611A2FB0645D4EBC030A94136
:10BB800002D2761E8018594146EACC3C07B34140A8
:10BB9000C7F12006B840F1414140B1FBF3F603FB89
:10BBA0001611A2FB0645001BA94102D2761E801881
:10BBB000594180EA010221FA0EF3C7F1200462FA2A
:10BBC0000EF20CFA07F05A402CFA04F13043F0BDA3
:10BBD00080EA010221FA0EF3002162FA0EF26046B9
:10BBE0005A40F0BD8C46B1FBF2F102FB11C31B02BF
:10BBF00043EA1063B3FBF2FC02FB1C331B024CEA6A
:10BC0000002043EA1063B3FBF2FC02FB1C331B026F
:10BC10004CEA002043EA1063B3FBF2FC02FB1C3346
:10BC20001B024CEA002043EA1063B3FBF2FC02FB68
:10BC30001C324CEA002000237047036A23B9C06914
:10BC4000B0FA80F04009704700207047B0B581EA33
:10BC5000030C0CF0004C40F2FF7515EA11541DBFA7
:10BC600015EA1357AC42AF4239E0E41923EA4553D1
:10BC700043F48013C90241F0004141EA505EC7021B
:10BC80001100A7FB020200284FF00000EEFB01208C
:10BC90004FF00001E3FB072118BF42F001024018FA
:10BCA00000214941E3FB0E01A4F580640F0302D299
:10BCB00052004041494154F101046CDD470872F1E2
:10BCC000004250F1000051EB0451A1F580115CBF1E
:10BCD00041EA0C01B0BD4CEA05510020B0BD05EAB7
:10BCE0001357AC4214BFAF4241E050EA410E1CBFB3
:10BCF00052EA430E02E061460020B0BD24423C44BB
:10BD00001BD15FEA070EF6D0090302BF01460020EF
:10BD1000AEF1140EB1FA81F7AEEB070401FA07FE9B
:10BD20000C37C7F1200100FA07F7C8404EEA000EB1
:10BD300023EA455343F48013A2E733F00043B3FAF8
:10BD400083F704BFB2FA82FE77440B3FE41BB7F1DE
:10BD5000200E2FBF02FA0EF3BB40C7F1200E22FACD
:10BD60000EFE38BF43EA0E03BA40641C82E750EA75
:10BD7000410E14BF52EA430E6FF000014FF400175A
:10BD800017EB430F8ABF194617EB410FB5E74CEA93
:10BD900005510020B0BDD4F10104B4F120070FDA41
:10BDA000C4F12007520828BF42F0010210FA07F53B
:10BDB00001FA07F7E1BF2A43E0403843E1400FE0D2
:10BDC000352C98DCC7F1200452EA400220FA07F231
:10BDD00018BF42F0010231FA07F0A1400A430021E6
:10BDE00072F1004250F1000051EB0C01B0BD03684C
:10BDF00010B4DC690022A44601235DF8044B6047BF
:10BE000010B5144600F002F8226010BDC1F30A53C9
:10BE100043B14A0012F5001F28D2A3F2FE32A1EB73
:10BE20000251704750EA410C20D001F0004C31EA39
:10BE30000C01B1FA81F204BFB0FA80F3D2180B3AC8
:10BE4000B2F120032CBF00FA03F1914041EA0C014A
:10BE50003EBFC2F1200C20FA0CF31943904052422D
:10BE600040F2FD33D21A01EB0351704700227047B4
:10BE70004FF4001C1CEB410F94BF1CEB430F09E077
:10BE800041EA030C50EA4C0C52EA0C0C03D29942E2
:10BE900008BF9042704714BF8B42824270470EB475
:10BEA00083B004AB019303B003B070474FF4001CA0
:10BEB0001CEB410F94BF1CEB430F09E041EA030C5C
:10BEC00050EA4C0C52EA0C0C03D28B4208BF82425F
:10BED000704714BF994290427047C3695940036A42
:10BEE000C161013B03627047124254D440F2FF7CAF
:10BEF0001CEA11530FD0634531D09B1863453CBFFA
:10BF000001EB0251704701F0004141EA0C51002061
:10BF100000F07ABA704750EA410320D001F0004C9B
:10BF200091EA0C011CD0B1FA81F30B3B9A420DD976
:10BF3000D21A994051EA0C01C3F1200C20FA0CFCF2
:10BF400061449840531C40F2FF7CD7E7914041EA9E
:10BF50000C01C2F1200C20FA0CF3194390407047F9
:10BF6000B0FA80F31533202BE0D3202AEED3203A09
:10BF7000203B9A4209D9D21A00FA03F141EA0C0196
:10BF80000020531C40F2FF7CB8E700FA02F141EABE
:10BF90000C0100207047524240F2FF7C1CEA115312
:10BFA0000DD06345DBD0B2EB030C3CBFA1EB0251DB
:10BFB00070470CF1010221EA035141F4801150EA6B
:10BFC000410CCCD001F0004C352A27DC30B481EA9A
:10BFD0000C01B2F1200309DAC2F12003044601FA90
:10BFE00003F5D0402843D1409C400CE0C3F120022F
:10BFF000450020FA03F418BF44F0010421FA03F0CD
:10C0000091400C43002174F1004550F1000051EBC8
:10C010000C01244230BC7FF47BAF704761460020A6
:10C0200076E70268531C036011707047C1F30A532E
:10C0300040F2FE329B1A14DDD3F120034FEAE17285
:10C0400008DDC90241EA505141F00040D840801853
:10C050005040704703F2E13010B1D24382F000400B
:10C060007047002070478068036810229B6818475B
:10C07000C11768B14840401AB0FA80F29040D21C13
:10C08000C907C2F5846241EA025202EBD0214005A1
:10C090007047FEE770B44FF0004591EA030F40F19E
:10C0A000BF816B40841A71EB030603D2001BB141C0
:10C0B000121973414FF4001C1CEB410F34BF7CEB91
:10C0C000430442E00C0DA4EB1356352E4FDC45EA39
:10C0D000C323DB0A45EAC121C912B6F120050DDDF3
:10C0E00063FA05F6EB4086EA0305124218BF45F0F5
:10C0F0000105C01851F100010CD213E062FA06F5F7
:10C10000F2405540F3415A40B340F3405A40801842
:10C11000594107D349085FEA30005FEA350528BF77
:10C1200045F0010501F58011420875F1004250F11A
:10C13000000041EB04514E0016F5001F70BC38BFE3
:10C1400070470020090D090570471CEB410F10D204
:10C1500052EA43060BD0BCEB410F05D80C0DAB43A4
:10C16000661E342EB6DD02E0AB438018594170BC28
:10C17000704770BC7047FEE7F0B540F2FF7581EA8A
:10C18000030C0CF0004C15EA11541DBF15EA1357AF
:10C19000AC42AF42E5E0BC41C1F31301C3F313036A
:10C1A000801A994143F4801304D2641E400049412F
:10C1B00080185941C90241EA5051B1FBF3F603FB23
:10C1C0001611A2FB0675D7EBC020A94102D2761E3C
:10C1D00080185941C90241EA5051B1FBF3FE03FBFB
:10C1E0001E11A2FB0E75D7EBC020A94103D2AEF100
:10C1F000010E80185941890241EA9051760546EABC
:10C200008E2EB1FBF3F603FB1611A2FB0675D7EBDE
:10C210008020A94102D2761E80185941C90241EA04
:10C2200050514EEA060EB1FBF3F603FB1611A2FBCA
:10C230000675D7EBC020A94102D2761E801859415D
:10C24000C90241EA5051B1FBF3F703FB1711A2FBFE
:10C250000735D3EBC020A94167F100070CBF0042AE
:10C2600047F0010766F3D5274FEA1E31B80814F5E9
:10C27000806412DDBD0775F1004250EB0E5051EBAA
:10C28000045111F5801F5CBF41EA0C01F0BD4CF078
:10C290007F6141F0E0410020F0BDBD076D0840EA3C
:10C2A0000E5041F48011D4F10104B4F120060ADAF1
:10C2B000C4F120060200E04001FA06F3E140184311
:10C2C000B24015430EE0342C13DCC6F1200445EADD
:10C2D00040056D0820FA06F2154321FA06F0A14048
:10C2E0000D43002175F1004250F1000051EB0C01AB
:10C2F000F0BD00205FEA0C01F0BDCFB992185B41A0
:10C30000B3FA83F704BFB2FA82F6BF190B3FB7F155
:10C3100020062FBF02FA06F3BB40C7F1200622FA1F
:10C3200006F638BF3343BA401CB1E419641E33E744
:10C330007F4231F00041B1FA81F404BFB0FA80F6D7
:10C34000A4190B3CB4F120062FBF00FA06F1A1405E
:10C35000C4F1200620FA06F638BF3143A0403C1B4A
:10C360001AE7AC421ABF05EA1357AF4212E050EA8F
:10C3700041061CBF52EA4306BFE750EA4107304678
:10C3800061461CBF41EA0551F0BD52EA430C08BFAB
:10C39000C143F0BD00204FF4001616EB410F98BFCB
:10C3A00016EB430F08BF16EB410F24BFC14305E056
:10C3B00016EB430F0CBF61464CEA0551F0BDFEE79A
:10C3C000400D491840EA81200CD2490DA1F5806149
:10C3D000491C40F0004005DBD1F11F0154BFC840AB
:10C3E000C017704700207047014648B1B0FA80F18D
:10C3F0008840C91CC1F58461090501EBD0214005C5
:10C400007047FEE77047FEE70FB581B00020C046D9
:10C4100002492222425001B00FBD00007C5E002084
:10C42000841A71EB030604D26E40001BB14112194D
:10C4300073414FF4001C1CEB410F34BF7CEB4306EF
:10C4400082E00C0DA4EB1356362E7BDC012E45EA60
:10C45000C32341DC43EA525312BFD20292025B086B
:10C46000240545EAC12141EA5051D2EBC02099414F
:10C4700025D407D1B0FA80F610FA06F162D0002078
:10C48000203608E0B1FA81F6B140C6F1200220FA68
:10C4900002F21143B0404FEAF474B4EB465434F066
:10C4A00001064FEA74040AD8D6F50016760D04F09A
:10C4B0000044F04061FA06F25040F1404840C00AA2
:10C4C00040EA415021F0004128BF5FEA500550F199
:10C4D000000044EBD12135E0DB0A45EAC121C90A5D
:10C4E000B6F120050EDD42EA0242120CC5F120062B
:10C4F00003FA06F6EB4042EA06056D42984161F107
:10C5000000010DE062FA06F5F240554063FA06FCC0
:10C5100082EA0C02F3405A406D42904161EB030104
:10C5200011F4801F05D1641E620502D06D004041E8
:10C53000494121F48011430875F1004350F1000096
:10C5400041EB045170BC70471CEB410F15D223F036
:10C55000004352EA43060BD04FEA4C0CBCEB410FB0
:10C5600004D80C0D661E342EB7DDEBE7801A994116
:10C5700050EA410608BF0021E4E708BF1CEB430F67
:10C5800028BF6FF00001DDE70000000000000000A0
:10C5900028B100BF02A1800141F0010108477047A6
:10C5A0000338FDD87047000010B5040005D04FF4E3
:10C5B0007A70FFF7EDFF641EF9D110BDF8B50C4697
:10C5C00015461E4600F04CFF60B12860012702E0CE
:10C5D00045F827007F1C2146002000F041FF20B1D4
:10C5E000B742F5DB4FF0FF30F2BD3846F2BD10B573
:10C5F0000446FFF741F9401E06D4215C0D2912BF05
:10C600000A2900212154F6D0002010BD0CB410B529
:10C61000C0B004460A4642AB4FF48071684600F051
:10C6200043FF01461CB9684600F0F6FF08E0012C04
:10C6300004D10021684601F08CFA01E04FF0FF3090
:10C6400040B010BC5DF80CFB012908BF0FF680213B
:10C6500002D011B90FF68821D8E74FF0FF307047AC
:10C660000A460FF68C21D1E70A460FF6A421CDE742
:10C6700080B518B9BDE8024001F0F0BB012908BF40
:10C680004FF0FF3004D0022906D1506801F040FE7F
:10C69000BDE8024001F04BBC4FF0FF3002BD70B569
:10C6A000044601F073FE0546DFF8E86901F06EFE0E
:10C6B000401BB0F5FA6F06D296F8040118B1642059
:10C6C000FFF772FFF2E701F07FFE0FF6642100F042
:10C6D0000FF9002070BD70B501290446154602D13E
:10C6E00001F09DFE52E0022997A621D1686897A12A
:10C6F00001F0BAFE18B9204601F0AFFF46E06868C5
:10C70000314601F0B1FE28B9204601F091FE012C1E
:10C710003CD126E0686801783039042936D201F02E
:10C72000F7FD042832D20146204602F055F82DE0EC
:10C7300003292BD16868314601F096FEA0B9A8689C
:10C740001022002101F0E9FD0446200403D0A1B22B
:10C75000002001F0D6FF240C03D02146012001F077
:10C76000D0FF02F02AF811E0012655F826000178E2
:10C770003039042907D201F0CBFD042803D2014649
:10C78000204602F029F8761C022EEEDD002070BD56
:10C790007CB5002815462ED10129DFF800690DD19E
:10C7A0003088F189441CA142B8BFB489214602B047
:10C7B000BDE870400246002002F0F6B902290AD115
:10C7C00000F042F80446B0898442A4BFF089A04238
:10C7D00037DB2046EAE7032933D100F035F800F0D3
:10C7E00036F8B1898C42A2BFF289A242884228DB86
:10C7F0008242DBDA25E0022905D100F025F8BDE808
:10C80000764002F037BA032907D100F01DF800F096
:10C810001EF84FF0FF3201460DE0042911D100F05F
:10C8200013F800F014F80646E8681022002101F021
:10C8300074FD02463146204602B0BDE8704002F069
:10C84000BEB94FF0FF3076BD686801F061BD0446A7
:10C85000A86801F05DBD38B501290446154602D12E
:10C8600002F0EAFA42E0022923D16D68B8A100F093
:10C87000BCFA50B902F08DFC00280CBF0FF6BC01C9
:10C880000FF6DC0100F034F830E0287830380A2860
:10C890002CD2284601F03CFD0546002180B202F072
:10C8A0003DFC00282A4614BF0FF6F4010FF6CC0118
:10C8B00019E003291AD16868A6A101F0D5FDA8B92D
:10C8C000A868017830390A2910D201F021FD054607
:10C8D000002180B202F03EFC00282A460CBF0FF671
:10C8E000DC010FF6FC012046FFF790FE002032BD70
:10C8F00020468BE61CB5012905D102F09DFA01F016
:10C900004EFB002016BD02291BD1546892A120467F
:10C9100001F0AAFD10B902F08FFAF2E70FF2A07150
:10C92000204601F0A1FD0028E9D08CA1204601F0AD
:10C930009BFD30B902F080FA01F031FB01F030FBD1
:10C94000DFE74FF0FF3016BD2D6F00002D640000B3
:10C950002DE9F8410F46012FA1B040F3D5801446D0
:10C96000054666687EA100F005F9002842D1042F33
:10C970007CA638D1A06803236A467BA1FFF71EFE80
:10C98000032840F0DF80009801F0C2FCB0F5FA6F98
:10C99000A8BFA0F5FA600890019801F0B9FC401E0C
:10C9A0000790029801F0B4FC06900323E0686A4601
:10C9B0006EA1FFF703FE032862D1009801F0A8FCE6
:10C9C0000590019801F0A4FC0490029801F0A0FCED
:10C9D000039003A802F0ECFC002840F0AE8002F0C7
:10C9E00061FE0346A3E0022F4AD102F03FFD0FF69D
:10C9F00008039CE05EA100F0BDF868BB032FBFA652
:10CA00003ED1A4682046FEF737FF20283DD22021E2
:10CA1000684602F079FE2146684602F079FE02F08F
:10CA2000BCFE0446012C08BF02F0ABFE684601F0D4
:10CA3000D3FA002806D46B46324601212846FFF778
:10CA400003FE03E031462846FFF70EFE012C7DD1A0
:10CA5000012002F087FE79E00FF2646100F08AF8AD
:10CA600030B901F07DF90FF2A4730FF298725FE014
:10CA70000FF2A07100F07EF860B9032F0FF29C76E0
:10CA800060D100F002FA032800905BD201226946CF
:10CA9000002015E00FF28C7100F06CF8A8B9032F9C
:10CAA0000FF288764ED100F0F0F90090401F1A285E
:10CAB00048D20098DFF8E815C865012269460220CF
:10CAC00001F0EAFA002838D430E00FF2687100F083
:10CAD00051F8C8B9052F0FF2647633D1E068694682
:10CAE00002F07AFE206901A902F076FE0746002FC7
:10CAF00006DD394601A802F09EFE0099814208D069
:10CB000031462846FFF7ACFD4FF0FF3022B0BDE8BC
:10CB1000F081E06801F0FCFB804600F0B6F93B468E
:10CB200001AA414601F00DFB002806D5A368324654
:10CB300001212846FFF788FD08E031462846FFF727
:10CB400093FD03E031462846FFF78AFD0020DDE72C
:10CB50002D6300002D62000065780000616C6C00A0
:10CB600072746300525443002D0000003A0000002C
:10CB700069640000304601F077BC78B502299DB0A9
:10CB8000044633D155680FF2BC61DFF8146500F03C
:10CB90002CF960BB09A801F03BFA002115A802F0AE
:10CBA0006BFE0DA802F086FE0322A7A106A8FEF7E1
:10CBB000DDFE07220FF2946107A8FEF7D7FE02F010
:10CBC00071FD034606A907A8049105900DAD316ECD
:10CBD000DFF8D00402680391029215A90091019533
:10CBE00009AA0FF270612046FFF710FD82E097A1BD
:10CBF00000F0FBF828B902F055FD02460FF274610F
:10CC000060E093A100F0F1F840B9684601F000FA45
:10CC100000286FD16A460FF26C6116E08DA100F01A
:10CC2000E4F838B90021684602F026FE6A460FF2A1
:10CC300064610AE00FF26C6100F0D7F848B9684609
:10CC400002F038FE6A460FF264612046FFF7DEFC10
:10CC500050E00FF26C6100F0C8F818B9204602F0FD
:10CC600056FE47E00FF2606100F0BFF818B92046A9
:10CC700000F048FD3EE00FF2586100F0B6F810B940
:10CC80000FF2546134E00FF28C5100F0AEF860B94D
:10CC90000122694601F0E9F9002803D4009A0FF255
:10CCA0004C610FE00FF2745112E000F09CF898B95B
:10CCB00001226946022001F0D8F9002806D4009A22
:10CCC0000FF238612046FFF7A1FC13E00FF25C5130
:10CCD0002046FFF7C9FC0DE00FF2306100F085F847
:10CCE00040B9307E00280CBF0FF228610FF2386186
:10CCF000FFF7FEFD00201EB070BD0000494400009B
:10CD000002F0D2BE38B50129144602D102F0C8FFA4
:10CD100029E0022914D16068B8A101F0A5FB10B97F
:10CD200002F0C1FF1FE060680178343902291AD28D
:10CD300001F0EEFA011F022915D202F0D3FF12E032
:10CD4000032910D1012554F825000178343902292E
:10CD500006D201F0DDFA011F022938BF02F0C2FF3E
:10CD60006D1C022DEFDD002032BDBFF34F8FCE4989
:10CD7000CE480A6802F4E06202430A60BFF34F8FB4
:10CD800000BFFDE780B5012002F0ECFC002002BDF1
:10CD9000F8B50229044624D155680FF22C3100F071
:10CDA00024F8F0B10FF264510FF29856BC4F00F026
:10CDB0001CF820B9387633460FF280520DE000F0AF
:10CDC00012F870B9012000900122694601F064F95F
:10CDD0000120787633460FF2544201212046FFF7B6
:10CDE00033FC0020F2BD0FF23C41284601F03CBB71
:10CDF000F8B50229044625D1D2F80450B2A1FFF7B4
:10CE0000F4FFF8B10FF204510FF24056A44FFFF7B0
:10CE1000ECFF28B90120387633460FF220520DE09E
:10CE2000FFF7E1FF70B9009001226946012001F08F
:10CE300033F90020787633460FF2F0320121204694
:10CE4000FFF702FC0020F2BD34470000727463005B
:10CE5000696400006370750070B50429A0B01446C1
:10CE600010D1606801F054FA054600F00EF800EBAE
:10CE70000536E068694602F0AFFC82B2694630468A
:10CE800002F0ADF9002020B070BDA06801F040BAFA
:10CE90002DE9F0410129054602DC4FF0FF300DE09D
:10CEA000506801F035FA04000AD102F0F9FF224679
:10CEB0000FF2BC412846FFF7A9FB0020BDE8F08136
:10CEC000012C04D102F0D9FF02F0DCFFEFE7022CC5
:10CED00004D102F0D2FF02F0DCFFE8E7032C41F2BC
:10CEE000813641F2941740F2A46817D102F0C5FFD1
:10CEF00002F0C8FF4046FFF74BFB02F0C5FF4FF4BE
:10CF00004870FFF745FB02F0C4FF3846FFF740FBCF
:10CF100002F0B8FF3046FFF747FBC6E7042C14D1F8
:10CF200002F0ABFF02F0B5FF4046FFF731FB02F025
:10CF3000B2FF4FF44870FFF72BFB02F0A3FF384617
:10CF4000FFF726FB02F0A5FFE4E722460FF20841B7
:10CF50002846FFF75BFBA0E72DE9FC4105460024CE
:10CF60000FF21C48524E49A70C20604332584AB178
:10CF7000002C12BF4146326839462846FFF746FB6F
:10CF8000641CF1E742A12846FFF740FB0020BDE802
:10CF9000F6812DE9F8430446894616469846002551
:10CFA00000E06D1C0C20684308EB00073968F9B1FC
:10CFB000306801F059FA0028F3D16CB938790128AA
:10CFC0000FD102F0DEFBBB6832464946002098478D
:10CFD0002FA000F010FB09E07879012808BF02F0CB
:10CFE000D0FBBB683246494620469847002001E006
:10CFF0004FF0FF30BDE8F283000000002D6100001B
:10D0000038B504468AB00D46012C01BF2878422865
:10D0100069784D2904D12946012002F0C0FF33E090
:10D020002846FFF7E4FA002C29460CBF0FF25830CF
:10D030000FF2603000F0DFFA0A236A4616A1284694
:10D04000FFF7BCFA0546002D1EDD194B00F034F841
:10D05000002819D5174803681BB100F02DF80028E7
:10D0600012D50098FEF708FC02280DD30FF23431D8
:10D07000FFF73EFC009A0FF280312046FFF7C6FA18
:10D080000FF28831FFF734FC0BB030BD2573000080
:10D090000D0A0000F437002020000000485D002049
:10D0A000B8350020B02F00200CED00E00400FA0598
:10D0B000B8340020505E00206A462946204668E7C2
:10D0C0007464617461000000736461746100000045
:10D0D0004F4B202573203A2025730D0A00000000D5
:10D0E0004552524F52202573203A2025730D0A00D5
:10D0F0004552524F52202573203A20496E76616C7A
:10D10000696420506172616D657465720D0A00007A
:10D110004552524F52202573203A2046756E637453
:10D12000696F6E204661696C7572650D0A000000BA
:10D13000646675206F6B0D0A000000005732355190
:10D140003235364A562C2073756363657373667582
:10D150006C6C79206572617365642E0D0A000000A5
:10D16000573235513235364A562C206E6F74206551
:10D1700072617365642E0D0A0000000053656374CC
:10D180006F722025642C20737563636573736675F5
:10D190006C6C79206572617365642E0D0A00000065
:10D1A000536563746F722025642C206E6F74206544
:10D1B00072617365642E0D0A00000000426C6F639B
:10D1C0006B2025642C207375636365737366756CBF
:10D1D0006C79206572617365642E0D0A0000000091
:10D1E000426C6F636B2025642C206E6F7420657217
:10D1F000617365642E0D0A00436C65617265642E6F
:10D200000000000054444154410000005361766521
:10D21000640000006D6F6465000000004D4F4445E0
:10D2200000000000706175736500000050415553A7
:10D230004500000064636667000000004443464701
:10D2400000000000696E666F000000003530304459
:10D2500050530000494E464F2C25732C25732C2526
:10D26000732C25732C25733A25732C25732C257369
:10D27000000000004F4B20525443203A2025730DEC
:10D280000A0000004F4B204944203A2025730D0A24
:10D29000000000004F4B20435055203A2025730DCD
:10D2A0000A0000006370755F696400004F4B204303
:10D2B00050555F4944203A2025730D0A00000000B4
:10D2C0006661756C74000000756172740000000086
:10D2D00074696D65720000004F4B2054494D4552F2
:10D2E000203A203130300D0A000000004F4B204D15
:10D2F0004F4445203A2025640D0A00004F4B205032
:10D3000041555345203A2025640D0A00747269671F
:10D31000676572004F4B2054495252474552203A9C
:10D32000204F4E0D0A0000004F4B205452494747F2
:10D330004552203A204F46460A0A000054524947B7
:10D3400047455200454E41424C45440044495341F3
:10D35000424C454400000000696E76616C696420AF
:10D36000666972655F6D6F646520282564290A000F
:10D3700066697265203A206F6B282564290A0000CF
:10D380002C202573000000003E3E2025730D0A0D61
:10D390000A000000424C453E3E2025730D0A0D0A4E
:10D3A000000000000D0A2D2D2D2D2D2D2D2D2D2DA4
:10D3B0002D2D2D2D2D2D2D2D2D2D2D2D2D2D2D2D9D
:10D3C0002D2D2D2D2D2D2D2D2D2D2D2D2D2D2D2D8D
:10D3D0002D2D2D2D2D2D2D2D2D2D2D2D2D2D2D2D7D
:10D3E0002D2D2D2D2D2D2D2D2D2D2D2D2D2D2D2D6D
:10D3F0002D2D2D2D0D0A00002573203A206E6F74FF
:10D4000020646566696E65642E0D0A00232323235C
:10D4100023232323232323232323232323232323DC
:10D4200023232323232323232323232323232323CC
:10D4300023232323232323232323232323232323BC
:10D4400023232323232323232323232323232323AC
:10D45000232323232323232323230D0A0000000057
:10D4600038B504000D4609D0204602F0CDFD044435
:10D47000207848B90B4A0021116032BD0948046880
:10D48000002CF1D1002032BD2946204602F0CDFD0E
:10D490002118087810B1002201F8012B2046014A1A
:10D4A000116032BD645E002008B584B00023039390
:10D4B00000290EBF01930190491E0291009301A91A
:10D4C00004AB074878441830FDF760F9019909B1B9
:10D4D00000220A70002858BF039805B000BD00BFA5
:10D4E00013E5FFFF00000000000000000000000046
:10D4F00010B5040008D000BF99A14FF47A4041F064
:10D5000001018847641EF6D110BD38B50178884CFA
:10D5100011B1022934D031BD684602F06EFE9DF88B
:10D52000001082A000F067F8608882499DF8002012
:10D53000401C608001F5A1657F2A688802D150B344
:10D54000401E1BE00D2A18BF0A2A0CD100220A54E3
:10D550000120287002F0D0FE00206880606C002856
:10D5600019DD002116E0B0F5807FA4BF002068809F
:10D570006A889DF8000088546888401C688031BD26
:10D58000616C082907DA04EBC10200235360491CCF
:10D5900040689060616431BD38B58AB00DF110000B
:10D5A00071A1644C1822FEF7E1F94FF480700190EC
:10D5B00004F20C614FF480600291039004F20C5568
:10D5C000009507235C4A694604A802F0B7FD04F5FC
:10D5D000A06100220A720A604A6018B102F0C6FE19
:10D5E0004FF0FF300BB030BD52487047514900201A
:10D5F00081F8080570470EB400B5C0B0024641ABD3
:10D600004FF480716846FFF74FFF0146684600F00F
:10D6100003F840B05DF810FB2DE9F041444D06469B
:10D62000686C00288846C8BF002047DCEFF30580FF
:10D63000F8B14048002400F5A06105E0375D0244E0
:10D64000641C82F800714B6044450BDA4A680F682D
:10D65000531CB3F5806FA8BF0023BB42EED1A86C6A
:10D66000401CA864002CC4BF062002F045FE2046E2
:10D6700024E02878012803D1A96C491CA9641BE087
:10D6800001202870002700E07F1C47450BDAF05D81
:10D6900002F072FE0400F7D0A86C401CA86402E0FF
:10D6A0000120FFF725FF02F0FFFD0028F8D0002041
:10D6B00028700CB9404601E04FF0FF30BDE8F08122
:10D6C00038B51C4C04F5A06507E02868401C2860AC
:10D6D000B0F5806FA4BF0020286028686968884280
:10D6E0000DD0204490F8000102F046FE0028ECD056
:10D6F0000F48816C491C81644FF0FF3032BD00201F
:10D7000032BD0000F8B504465FF000050BA6084FD7
:10D7100008E007EBC5008368426831462046FEF703
:10D7200075FF6D1C786C8542F3DBF1BD256300004D
:10D73000385B0020444600200BD50100554152546F
:10D740005F4552524F52203A2025642C2025640D0B
:10D750000A000000000000000000000000000000BF
:10D760000338FDD8704700000500000004000000E9
:10D77000FFFFFFFFFFFFFFFF0000000000E0D701F9
:10D7800028B10FF2BC51800141F0010108477047F8
:10D7900000B5C3B011208DF80000DFF8A8240FF207
:10D7A000DC4103A802F0FAFD03A8FEF765F81F2884
:10D7B000C8BF1F2082B203A968467CDF08B102F00F
:10D7C0000DFE01A800210022C0E9001210203C211A
:10D7D000ADF80610ADF804004FF4C871ADF808209C
:10D7E000ADF80A1001A87ADF08B102F0F7FD43B0E6
:10D7F00000BD02F0F3BD70B504462078D0B9A28A0E
:10D800001546022D16DBDFF8406421693046FEF72D
:10D810009DF80020705506F58071A08A08600120EF
:10D820004871087908B901220A710220BDE87040E8
:10D8300002F062BD70BD1CB5DFF81004DFF81044C3
:10D84000019001A904F1200002F0D9FD08B102F015
:10D85000C5FDDFF8000400906946201D02F0FEFEC1
:10D8600008B102F0BBFD13BD007840B9DFF8E0233A
:10D8700010883B2176DF002818BF02F0AFBD70474B
:10D8800002F0ACBD00B587B01C21684601F03CFF3A
:10D89000002000904FF4A0314FF4F020029001914D
:10D8A00000200321ADF80E008DF810008DF80C104B
:10D8B000DFF8A403DFF8A41305900691684602F090
:10D8C000CEFF08B102F08AFD07B000BD704780B5F9
:10D8D0000321DFF88C0303F01DF918B1BDE8024005
:10D8E00002F07CBD01BD38B5DFF8645304462188E1
:10D8F000288810290CD0112921D0132939D02129A9
:10D900002ED03B293FD0522938D056293BD031BDAB
:10D91000DFF85023116811B9012003F016FB0FF254
:10D920006C30FFF768FEA188298005F1200002F025
:10D9300078FD08B102F052FD03F056FB31BD042022
:10D9400003F003FB4FF6FF7028800FF25430FFF70F
:10D9500052FEFFF7BCFFBC49002081F8040131BD35
:10D960000FF2E4321088ADF800006946A0888FDF1E
:10D970000CE00023002285217FDF07E00023002246
:10D980000021B1DF02E0A088132176DF08B102F0A8
:10D9900025FD31BD80B503F0C7FB08B102F01EFDC7
:10D9A000002000906946012003F05CFC08B102F001
:10D9B00015FD684603F0AFFC08B102F00FFD01BD94
:10D9C000A3484B8802889A4202BF0A8840F6772310
:10D9D0009A4202D18988CA1E4280704710B5A24C73
:10D9E000A249204603F0F0FC08B102F0F7FCF72151
:10D9F000204603F0FFFC18B1BDE8104002F0EEBC79
:10DA000010BD18B5ABB0AC21684601F07DFE022018
:10DA10008DF8000000219648914C00788DF8021096
:10DA2000012807BF06218DF8031005228DF8032079
:10DA30000121ADF84C10012204F2344114918DF80B
:10DA40007C201FA9402201280CBF002044F2506016
:10DA50000861CA60874888626946204602F0E5FF8F
:10DA600008B102F0BBFC0121204602F0DBFF2CB024
:10DA700010BD10B5744C04F584721021C02003F061
:10DA80007FFD08B102F0AAFCFFF784FFFFF780FEDC
:10DA9000FFF7A4FFFFF7CFFEFFF7B3FFFFF7F2FE9C
:10DAA0000A20FFF76DFEFFF712FF04F582700021D8
:10DAB00001808170002010BD634870476248D0F833
:10DAC000000170476049002081F805017047F0B5FA
:10DAD0000446694815460278C1B00AB908202CE00E
:10DAE0008078012811D14FF4807301AA204603F0F9
:10DAF00069FD002807DD01AA0A211154401C01AC70
:10DB0000ADF8000003E000201BE0ADF80010002697
:10DB1000012D4F4F09D100F016F870B9BDF8000083
:10DB20000FE04FF47A70FFF72BFE00F00CF813288B
:10DB3000F3D1761C332EF4D30D2002F017FC4FF0F6
:10DB4000FF3041B0F0BD3B886A462146381D02F0E7
:10DB5000EEBD38B504460D46FDF78EFE81B22A466D
:10DB60002046BDE83840B2E70CB40A4610B5364945
:10DB7000044691F80401C0B028B9082002F0F6FB71
:10DB80004FF0FF300EE042AB4FF480716846FFF774
:10DB90008BFC0028D8BF002004DD81B222466846F5
:10DBA000FFF795FF40B010BC5DF80CFB10B50446C4
:10DBB00086B00020207004A86DDF10B14FF0FF3058
:10DBC00015E09DF811009DF81210039002919DF848
:10DBD00013009DF814100190CDF800109DF8153039
:10DBE0009DF8162034A1204602F0D8FB002006B094
:10DBF00010BD000078B589B037A0154D3DA6FFF7E0
:10DC0000FAFC00242246314601A802F0C7FB01A815
:10DC1000FDF732FEADF800006A462B8801A9281DE9
:10DC200002F085FD40B9641C142CEBDB3CA0FFF72F
:10DC3000E2FC00200AB070BD0246214630A0FFF78A
:10DC4000DAFCF3E7D3350020F4370020F3D70100E6
:10DC5000C02F0020F7D7010069D8010081D801004A
:10DC6000EC2F0020545E0020B05D0020C1D90100DF
:10DC7000845E0020CDD80100F838002053575F4162
:10DC80004952424147202D2025730000424C453E19
:10DC90003E20636F6E6E65637465642E0D0A00002E
:10DCA000424C453E3E20646973636F6E6E656374DB
:10DCB00065642E0D0A000000253032583A253032B6
:10DCC000583A253032583A253032583A25303258B1
:10DCD0003A253032580000007379735F626C655FDB
:10DCE000746573742829202D2073746172740D0A71
:10DCF00000000000746573742D25640D0A00000097
:10DD0000626C655F6E75735F646174615F73656E8D
:10DD10006428256429202D3E2025640D0A0000007A
:10DD20007379735F626C655F746573742829202D45
:10DD30002073746F700D0A000000000000000000E6
:10DD40000338FDD87047000000000000000000000C
:10DD500028B10FF29C41800141F001010847704752
:10DD60002DE9F84F90B0054600F010FBBA4FBB49C3
:10DD7000D1F8009080467868002400280DD53868D6
:10DD80007C60401C38603D61D9F80800323096282C
:10DD9000F86055D39638F86052E006D101207860DB
:10DDA00001210E2001F0BAF917E0411E0B2902D221
:10DDB000401C786044E04FF0FF3610D10D207860B1
:10DDC00003F098FC009001961022396902910396A5
:10DDD00069464FF4604001F002FA044630E00D2835
:10DDE00003D103244EF2100A04E04DF6C04104248E
:10DDF00001EB801A4FF0000B10E0FD6809F11000F4
:10DE0000102250F825100DEB0B10FDF79FFD6D1C37
:10DE1000962D28BF0025FD600BF1010BA345ECDB1F
:10DE200022016946504601F0DAF904467868401C40
:10DE30003328786004DB7E60B868002848BF3E6005
:10DE4000404600F0AEFA02460FF250310FF23C307D
:10DE5000FFF7D1FB204611B0BDE8F08F2DE9F84166
:10DE600089B08046102205A94FF4604001F0E1F826
:10DE7000002835D4079B059A0FF234310FF24C3548
:10DE80004046FEF7C3FB4620FFF762FF4EF2100745
:10DE9000962405AE102205A9384601F0CAF80028DC
:10DEA0001ED4B6F90C00B6F90230BDF91420049066
:10DEB0002946B6F90A00039002901037B6F9060019
:10DEC0000190B6F9040000904046FEF79FFB462003
:10DED000FFF73EFF641EDDD100200AB0BDE8F081EF
:10DEE0004FF0FF30F9E718B5A1B044F25441C30137
:10DEF000ADF80010ADF8020003F560431228B9BF79
:10DF0000802284247022742401A9184601F091F81B
:10DF1000002806D4012221466846FFF7D8FD0028D4
:10DF200002D54FF0FF3000E0002022B010BD38B520
:10DF300000282CD501F031FC012818D1464CA068EE
:10DF4000002805D52068401C00212060A1601CE04D
:10DF5000FFF7C9FFA068401C1328A06015DB6168AB
:10DF60004FF0FF300029A0600FD520600DE00025A4
:10DF70002846FFF7B8FF32244FF47A70FFF7E8FE27
:10DF8000641EF9D16D1C132DF2DB002032BD132865
:10DF900002D34FF0FF3032BDBDE83240A3E700E0CE
:10DFA00000BF4FF0FF30704780B501464FF4F0726C
:10DFB0004FF4704001F066F9002800D569E0BDE833
:10DFC000044000210F2001F0A9B801464FF4F0727F
:10DFD0004FF4704001F070B910B50446FDF74CFCE9
:10DFE000202802D300F07FF805E000210F2001F087
:10DFF00095F8002800D535E02146194801F088FB46
:10E000002146BDE8104020224FF4704001F0E7B8EF
:10E0100010B5044600202070202221464FF47040A5
:10E0200001F007F8002800D51CE02078FF2804BF85
:10E030006178FF290BD1A078FF2804BFE178FF2980
:10E0400005D104A001682160052002F08FF90020AD
:10E0500010BD0000585858009C2F0020203600208A
:10E06000D33500204FF0FF3010BD80B510283EBFE3
:10E0700013185B1E102B02D300F035F809E04FF2A5
:10E08000200303EB8000BDE808409204120C00F06E
:10E09000D0BF4FF0FF3002BD70B504461646102CBD
:10E0A0003EBF3019401E1028F8B00D4602D300F0D4
:10E0B0001AF804E06846FFF777FF002802D54FF012
:10E0C000FF300EE0002007E06946021901EB8201F3
:10E0D00055F820200A62401CB042F5D36846FFF78D
:10E0E00074FF78B070BD072002F040B938B5034620
:10E0F0001546032B38BF412DA0B00C4602D3FFF7C5
:10E10000F2FF13E04FF260008022694600EB8310BB
:10E1100001F0B8F8002809D40098854206D12946B4
:10E1200002A801F088FB0199884202D04FF0FF302D
:10E1300005E02A4602A92046FDF708FC002021B090
:10E1400030BDF8B504460D461F46032C3CBF781978
:10E150004128F8B0164602D3FFF7C5FF04E0684631
:10E16000FFF722FF002802D54FF0FF300CE00DEB47
:10E17000C4106D0800EB45003A4631466030FDF7AB
:10E18000E5FB6846FFF721FF79B0F0BD2573203A23
:10E19000202564206D732E0D0A00000073617665E2
:10E1A0005F747269676765725F6461746100000023
:10E1B000426174746572793D25642C2054726967DC
:10E1C0006765723D25640D0A0000000025642C255A
:10E1D000642C25642C25642C25642C25642C256452
:10E1E0000D0A000000000000000000000000000018
:10E1F0000338FDD8704700002DE9FC4F83B00E4670
:10E2000017460BB100221A608046444600E0641CA9
:10E21000207803F0B1FA0028F9D120782D2816BF14
:10E220002B2814F801BB4FF02B0B002F019603D4C1
:10E23000012F01D0252F04DB002E47D0C6F8008027
:10E2400044E0002F0ADD102F04BF2078302802BFE1
:10E25000617841F0200178290ED10AE02078302839
:10E2600018BF0A2708D1607840F02000782802D132
:10E270001027A41C00E00827029400E0641C20780A
:10E280003028FBD04FF0000925A02646CA468DF85D
:10E29000000007E09DF80050451BCA46EDB207FBA1
:10E2A0000959641C207803F071FA00BF1CA30146D1
:10E2B0003A461846FDF70AFB0028EBD10299A14225
:10E2C000484605D1019808B1C0F8008000201CE044
:10E2D0001DA1A61BC95D761A002E0FD405DC451BB7
:10E2E00003D3B5FBF7F1514508D0FEF78DF804983C
:10E2F00008B1012101604FF0FF3003E0BBF12D0FA9
:10E3000008BF4042019901B10C6005B0BDE8F08F33
:10E31000FFE700230A2200216EE700BF00236BE71E
:10E32000303132333435363738396162636465668B
:10E330006768696A6B6C6D6E6F70717273747576F5
:10E340007778797A0000000000002115110E0D0C7D
:10E350000B0B0A0A0909090909080808080808082E
:10E360000707070707070707070707070700000052
:10E370001149124A01200860012111484160816061
:10E380002021116001220260002070470D480068C2
:10E390007047884201D3401A7047C1F1807140181C
:10E3A000704708490968814201D3081A7047C0F1D3
:10E3B00080700818704700000800004008150140F0
:10E3C000001001400415014011DF0849B120086028
:10E3D000BFF34F8F064907480A6802F4E062024320
:10E3E0000A60BFF34F8F00BFFDE700BF1C05004070
:10E3F0000CED00E00400FA05E0B5002008210190D2
:10E4000000914FF4007300220021164803F008FB2E
:10E410000EBD0B4601460822124803F035BB1149D8
:10E42000498800F0D9B90F484088112100F0E9B9B6
:10E4300038B50C4D04466888411E8941C90F2046F5
:10E4400000F0CAF9002802D54FF0FF3032BD6988CC
:10E45000204600F0C1F90546012C08BF00F0ADF9D7
:10E46000284632BD745D002081EA00039B0717D166
:10E47000820707D010F8012B11F8013BBAB19A427C
:10E48000F6D014E002680B689A42A2F1013301BF92
:10E49000934313F0803F50F8042F51F8043FF3D01A
:10E4A00010F8012B11F8013B0AB19A42F8D0D01AAA
:10E4B00070470000000000000000000000000000A5
:10E4C00028B10FF20C41800141F00101084770476B
:10E4D00010B5044600F0F6FF20600020207103F024
:10E4E0000CF96071DFF890030188E18010BD90F9AC
:10E4F00004100329BCBF41796529BEBFC08840F222
:10E50000FF11884201DB00207047012070473EB5B3
:10E510000546FFF7ECFF012833D06946DFF85C03BE
:10E5200000F0B9FC00F02FF81024BDF8040000281A
:10E5300004BFBDF8060000281DD000F071F800F0FF
:10E5400022F8BDF80200BDF80030000300EB0340E4
:10E55000BDF8043000EB0320BDF806300822294640
:10E5600000EBC30000F065FD2846FFF7C0FF01285F
:10E5700007D0641ED9D14FF6FF70E8804FF0FF300E
:10E580003EBD00203EBD012300222021684600F050
:10E5900066BC38B584B00546FFF72EFF002848BF9B
:10E5A0004FF0FF303AD402A80821019000914FF4B7
:10E5B000007302220021B14803F032FA04002DD486
:10E5C00002A8FFF7A4FF002C0CBFBDF80E0000202E
:10E5D00000F098F974B99DF90C0010F1010F09D001
:10E5E00000218DF80C10012D04BF02A8FFF711FFC8
:10E5F00000F016F802A8FFF76BFF0120012D8DF83F
:10E600000C000AD1002102A8FFF703FF00F008F870
:10E61000002000F007F800F003F8002005B030BD3E
:10E6200046204DE71CB504466846FFF751FF2346D8
:10E6300008226946914803F027FA16BD1CB5044626
:10E640006846FFF745FF02218DF80410ADF806403B
:10E6500000216846FFF7DDFE16BD38B5874D04463C
:10E66000688802280CBF03210221204600F0B4F87C
:10E67000002802D54FF0FF3032BD69882046BDE842
:10E680003440A9E00000000070B5064686B00C4694
:10E69000154668090002EB0000EB043003F0F803B4
:10E6A000082204A9181800F0C4FCFFF7B9FF9DF96F
:10E6B000140010F1010F21D0022804980CD100F0B1
:10E6C000EBFFBDF816109DF8152002910192009005
:10E6D0002B4622466BA10EE000F0DEFFBDF81610BF
:10E6E0009DF815200190039102922B469DF914008C
:10E6F0006DA1009022463046FDF788FF002006B04D
:10E7000070BD2DE9F84FA2B08846060345F244419A
:10E710000001ADF804104FF0010A4FF0FF3B002557
:10E7200000904FF6FF7901AF18EA0A0F4FEA4B0B42
:10E7300036D0009828187880802202A9304600F050
:10E7400078FC002836D40A244FF47A70FFF7B8FE1C
:10E75000641EF9D1002101A800EBC10082884A455E
:10E7600004BFC088484502D0491C1029F3DB10299A
:10E7700003DA788840F44040788018EA0B0F03D120
:10E78000788840F400407880C900091D002289B2D1
:10E7900001A8FFF79CF900280CD47888010405D45F
:10E7A00080366D1C202D4FEA4A0ABDDB002023B0C5
:10E7B000BDE8F08F4FF0FF30F9E780B545F24440F7
:10E7C0004FF6FF71ADF80000ADF8021000220421F1
:10E7D0006846FFF77CF902BD38B50C4658B90025EC
:10E7E0002A4621460020FFF74FFF6D1CB5F5007F3C
:10E7F000F6D3002032BD2046BDE834404FF6FF710D
:10E800007FE7F8B502280C4609D21D4800F02AF827
:10E8100048BF05F580654FF4806600271EE0042898
:10E820000AD2164800F01EF8B5F5806FB8BF05F59E
:10E8300080654FF40066F0E74FF0FF30F2BD28121C
:10E8400005EBD0514912A5EB41220020FFF71CFF38
:10E850006D1CB542A8BFA5F580657F1CA742EEDB05
:10E860000020F2BD41888288C08802EB011200EBD3
:10E8700042152D1B70470000485D0020605D0020A0
:10E88000745D0020256425303364202074696D6533
:10E890005B545D203A2020257320253364202054CA
:10E8A0003A25640D0A0000002564253033642020D9
:10E8B00074696D655B25645D203A202025732025F1
:10E8C00033642020423A25640D0A00000000000055
:10E8D0000338FDD870470000000000000000000071
:10E8E00028B10FF24C51800141F0010108477047F7
:10E8F00010B5040005D04FF47A70FFF7F1FF641EE5
:10E90000F9D110BD1CB5411C88B240F2FF129042F3
:10E9100000DA00B901214FF4FF7000900123A04CF0
:10E92000102289B2204603F031FA21889D4A916570
:10E9300016BD38B501469A4D1022284603F04BFA11
:10E94000040004BF288900280BD1A98A28888142A5
:10E9500007D003F074FB29880FF2C430A982FEF7B8
:10E960004AFE204632BD00002DE9F04F8C4B8BB0A3
:10E970009C89A142A1BF0A92DB890A9A934205DAD7
:10E98000072001F0F3FC4FF0FF3082E081460025C4
:10E9900000248A4601E00AF1010A8148C189491C24
:10E9A0008A4508BFB0F80CA00FF28831524648469D
:10E9B000FDF72CFE00260027300300EB0A404FF045
:10E9C000000B00EB0728102206A908EB0B1000F043
:10E9D00030FBBDF9182012F1010F04BFBDF91A0078
:10E9E00010F1010F23D1BDF91C0010F1010F04BF7C
:10E9F000BDF91E0010F1010F19D1BDF9200010F171
:10EA0000010F01BFBDF9220010F1010FBDF9240073
:10EA100010F1010F0BD1641C022C25DD11271026EB
:10EA2000002D27DDC6A14846FDF7F0FD22E0BDF927
:10EA30002430BDF926000FF25C3104930590002CC0
:10EA4000BDF92030BDF9220002930390C8BF002415
:10EA5000BDF91C30BDF91E00009301904846BDF978
:10EA60001A30FDF7D3FD6D1C0BF1010BBBF1100F3C
:10EA7000A9DB7F1C102F9FDB761C102E9BDB0A98D6
:10EA8000824588D14FEA0502CCA14846FDF7BEFD7C
:10EA900000200BB0BDE8F08F38B5FFF777FC0446D7
:10EAA00040F6B83502E0FFF771FC04462046FFF758
:10EAB00078FCA8420BD201F03BFC0021012003F0BE
:10EAC00036FB0128EFD00120FFF712FFEEE731BD42
:10EAD0002DE9FE4F324DA8890F468742A2BF029210
:10EAE000E989914206DA072001F040FC4FF0FF303F
:10EAF0004EE07F1CE989B8B2491C8842C5A008BF16
:10EB0000AF891FFA87F94946FEF775FD0026ADF873
:10EB10000070B046ADF80280002400E014B901F0A6
:10EB20009EF903E0032C08BF01F09BF9ADF8044007
:10EB30004FF0000A01F0FCFB0021012003F0F7FA7E
:10EB40000AEBCA00ADF8060000230122B1B2684604
:10EB500003F0A7FA83464620FFF7C2FE761CBBF1FE
:10EB6000840F17D30AF1010ABAF1010FE2DD641C28
:10EB7000A4B2102CD2DB08F101081FFA88F010288B
:10EB8000C8DB02988145B4D1002003F0FDFA0020D3
:10EB9000BDE8FE8FFFF780FF1024A046E7E70000E6
:10EBA000485D0020B8350020002808BFFFF7DCBE14
:10EBB000012808BFFFF78CBF4FF0FF3070472DE9E9
:10EBC000F845A2B00C4644F25341ADF8001090460F
:10EBD0006101ADF80410ADF8020021030127002502
:10EBE000002601EB004A18EA070F24D006EBD67086
:10EBF0004010F3010AEB002003F0800380220DF1A6
:10EC00000601181800F015FABDF8060080B100F0F2
:10EC100078F803DB0F2C08BF1F2E02D100F063F839
:10EC2000012500F067F80A20FFF762FE65B902E0EF
:10EC30004620FFF755FEBDF804007F00761C401CFF
:10EC40001F2EADF80400CEDD85B9BDF8020040F4FA
:10EC50000040ADF802000022BDF8040040F400407E
:10EC6000ADF8040006216846FEF731FF002023B00E
:10EC7000BDE8F085F8B5A2B0044644F25340ADF8C3
:10EC80000000ADF802400020ADF804000026240486
:10EC9000002740F2FF1580220DF10601204600F00A
:10ECA000C8F9BDF8060078B100F02BF801DBAF42DF
:10ECB00002D100F018F8012600F01CF80A20FFF736
:10ECC00017FE30000CD102E04620FFF709FEBDF828
:10ECD000040080347F1C401CAF42ADF80400DADD34
:10ECE000002023B0F0BDBDF8021041F40041ADF8A2
:10ECF000021070470001801D81B200226846FEF7B5
:10ED0000E6BE00204FF6FF730DF106010201895A9D
:10ED1000994202D0401C0828F6DB08287047000002
:10ED200073646174615F626C6F636B203A20256469
:10ED30000D0A0000626C6F636B2025640D0A0000F1
:10ED400053545245414D5F454E44212121212121FB
:10ED500021212121212121212121212121212121A3
:10ED60002121212121212121212121212121212193
:10ED70002121212121212121212121212121212183
:10ED80002121212121212121212121212121210D87
:10ED90000A000000253032642C253032642C2530E6
:10EDA00032642C253032642C253032642C253032EC
:10EDB000642C253032642C25640D0A00454E442114
:10EDC0002121212121212121212121212121212133
:10EDD0002121212121212121212121212121212123
:10EDE0002121212121212121212121212121212113
:10EDF0002121212121212121212121212121212103
:10EE000021212121212121212121282564290D0AC7
:10EE10000000000073656E7420626C6F636B203AB3
:10EE20002025640D0A000000000000000000000022
:10EE30000338FDD87047000038B500241BA5002119
:10EE4000A0B200F06BF921462846FEF7D4FB641C03
:10EE50000E2CF4DB1AA0BDE83240FEF7CCBB10B597
:10EE6000C4880CB1641E14E04C1E818811B1491E87
:10EE700081800EE00F218180418811B1491E4180BF
:10EE800007E00F21418001888A4234BF491E591E84
:10EE90000180C48010BD02880A8042884A8082882E
:10EEA0008A80C088C8807047000000004572617386
:10EEB000652025645F736563746F720D0A0000003E
:10EEC000457261736520646F6E650D0A0000000075
:10EED00028B10FF21C41800141F001010847704741
:10EEE0001FB5069C0091019202930394002269468B
:10EEF000001D03F03CFA04B010BDF8B511F1010F8C
:10EF00000CBF531C531D092B01DB0720F1E0C3F19B
:10EF10000805DFF86443261DEFB26D1CF05511F1B2
:10EF2000010F0FD0EFB2080EF0556D1CEFB2080CB8
:10EF3000F0556D1CEFB2080AF0556D1C201DEEB2A5
:10EF40006D1C8155100006D0211DEEB200206D1CF5
:10EF50008855521EF8D11846F2BD1CB50A4600214C
:10EF600000911218DFF810434042204400F10C01D8
:10EF70000023D2B2DFF80403FFF7B2FF18B101F0AB
:10EF8000F5F94FF0FF3016BDF8B51D4614460246A0
:10EF900008182918C9B2DFF8E06200915242B71888
:10EFA000C2B207F1940307F10C01DFF8D002FFF7BA
:10EFB00097FF00B19DE02CB12A4606F1940120464E
:10EFC000FCF7C4FC0020F2BD10B5DFF8AC426620AF
:10EFD000A07200219920E0720220FFF7BEFFB0B9B5
:10EFE00000F0F3F8204600F072F880B9A078C1076D
:10EFF0000ED400F083F850B900F0E7F8204600F096
:10F0000066F800F0E2F8A078C10701D40320E1E03F
:10F01000002010BD10B5044603224FF0FF319020B0
:10F02000FFF76BFF2246BDE8104002230021C0B26B
:10F03000AAE770B50C46154640F201118D4206460E
:10F0400005DA06F0FF01C1F58071914201D2072077
:10F050000AE0802D12DD00F018F8802322460021FE
:10F06000C0B2FFF791FF20B101F080F94FF0FF30FF
:10F0700070BD00F0AAF88034803D803600F005F8BD
:10F08000EBB22246BDE87040D0E7002231461320A3
:10F0900033E779490620FFE7C872002101205CE7C9
:10F0A0000A4680B5411E03290BD2754B724918449C
:10F0B000012310F8010CC8720021BDE800500120A6
:10F0C00062E7072001F052F94FF0FF3002BDF8B5BA
:10F0D00004460025684E6A4F785DF072012362197C
:10F0E00000210120FFF750FF18B96D1C032DF3DB41
:10F0F000F2BD01F03BF94FF0FF30F2BD5E49B720A1
:10F10000CAE780B569460120FFF7CAFF002806BF9D
:10F110009DF8000010F00100012002BD38B5044642
:10F12000B4F5005F0D46A8BF07200CDAFFF7B1FF6A
:10F1300048B900F04AF8002221032120FFF7DDFE44
:10F1400000F045F800B100E01AE001F00FF94FF0CF
:10F15000FF3032BD38B50446B4F5007F0D46A8BF78
:10F1600007200CDAFFF795FF48B900F02EF80022CF
:10F170002104DC20FFF7C1FE00F029F800B1E4E72C
:10F180002DB900F022F8FFF7BCFF0128F9D00020CC
:10F1900032BD10B50446FFF77CFF50B900F015F8FA
:10F1A00000224FF0FF31C720FFF7A7FE00F00FF855
:10F1B00000B10FE02CB900F008F8FFF7A2FF01281A
:10F1C000F9D0002010BDB8B20544462080E60021E9
:10F1D000C0B2C2E601F0CAF84FF0FF3010BD2DE911
:10F1E000F0410646154640F2011085420C4605DA0C
:10F1F00006F0FF00C0F58070A84201D207202CE085
:10F20000FFF747FF002828D1FFF7DFFF802DDFF849
:10F21000688017DD00F02CF80746802200F023F804
:10F220008021F8B2FFF799FEB8B9FFF7CEFFFFF7DC
:10F2300068FF0028F9D1FFF72CFFFFF7C6FF8034E5
:10F24000803D803600F014F80646AAB200F00BF8B4
:10F25000E9B2F0B2FFF781FE18B101F087F84FF084
:10F26000FF30BDE8F081214608F10C00FCF76EBBD1
:10F2700000223146122040E6AC570020A83500207D
:10F28000EC360020F8B504460D46164604E0FFF7BC
:10F290009AFFF61B14FA87F4B0B260B18128ACBFB4
:10F2A00080273746BAB229462046FFF7C2FE00281B
:10F2B000EDD54FF0FF30F2BDF8B504460D461646C9
:10F2C00004E0FFF780FFF61B14FA87F4B0B260B1D8
:10F2D0008128ACBF80273746BAB229462046FFF7BF
:10F2E0007EFF0028EDD54FF0FF30F2BD000000009A
:10F2F0000338FDD870470000002101E0491C0A389E
:10F300000A28FBDA40EA0110C0B2704701090A225C
:10F3100000F00F0012FB01007047C5E030B585B06A
:10F320000446002008218DF80800019103AD0095E6
:10F3300000F096F860B10020206118210120E06003
:10F3400061610020A060606020604FF0FF302DE020
:10F35000687800F07F00FFF7D9FF20609DF80E006D
:10F3600000F07F00FFF7D2FF60609DF80F0000F013
:10F370003F00FFF7CBFFA060287900F03F00FFF7C8
:10F38000C5FFE0609DF81100FFF7C0FF00F0070027
:10F39000A0619DF8120000F01F00FFF7B7FF401EAC
:10F3A0002061E879FFF7B2FF6061002005B030BD51
:10F3B00030B585B0044600208DF808008DF80C00AB
:10F3C00003AD2068FFF798FF68706068FFF794FF4F
:10F3D0008DF80E00A068FFF78FFF8DF80F00E06832
:10F3E000FFF78AFF2871A069FFF786FF8DF81100EB
:10F3F0002069401CFFF780FF8DF812006069FFF75D
:10F400007BFF8DF8130003A9082000F03FF880B9B6
:10F41000A52000F02BF800280BD420490120887685
:10F420001F480168CA0544BF81F480710160002053
:10F4300001E04FF0FF3005B030BD00B585B02C20A5
:10F44000012103AA8DF808000191009200F008F84C
:10F4500000280CBF9DF80C004FF0FF3005B000BD38
:10F46000012302AA51210F4803F058B800B585B016
:10F470002C218DF808108DF80C0003A9012000F054
:10F4800005F808B14FF0FF3005B000BD01900091C4
:10F49000012302AA5121034803F055B8B8350020D2
:10F4A000545E00204436002080B5FFF7C6FF0028D8
:10F4B00002D54FF0FF3002BDA52801D1012002BDC9
:10F4C000002002BD00B58BB06846FFF727FF6846F5
:10F4D00000F002F80BB000BDF8B505468CB02F69FE
:10F4E000EE686C6974A168463022FCF73FFA04F5B7
:10F4F000FA64611E40F26D13880803FB0103642067
:10F50000B1FBF0F29A1A4FF4C873B1FBF3F15DF856
:10F5100027008A188218012F11D914F0030F06D181
:10F520006420B4FBF0F0642101FB104030B9B4FB5F
:10F53000F3F34FF4C87000FB134404B9521CB6181F
:10F5400051496C68AB688E193C204FF461614443AB
:10F5500028684E4A01FB0343C31802FB06363046B7
:10F560000DB0F0BD10F0030F14D16421B0FBF1F128
:10F57000642202FB110159B94FF4C873B0FBF3F3D5
:10F580004FF4C87101FB1300401E8041C00F70474B
:10F5900001207047002070472DE9F0413B493C4E67
:10F5A000B0FBF1F501FB15003C22B0FBF2F23C216F
:10F5B00001FB1202B2614FF46161B0FBF1F201FB99
:10F5C00012003C23B0FBF3F0F0610721281DB0FBD3
:10F5D000F1F1C1EBC101401A3262306340F2B277FF
:10F5E00040F26D144FF4B77809E0854225D300F05E
:10F5F00033F8012814BF204640462D1A7F1C00F026
:10F600002BF801280CBF40462046EEE7B46A304490
:10F61000005D854218D300F01FF8012814BF0020B8
:10F620000C203044005D641C2D1AB46200F014F804
:10F6300001280CBF0C200020E8E7A7F5FA60F06273
:10F6400075630020B062F1E700206D1CB063756245
:10F6500006F11800BDE8F081384683E71FB5016860
:10F660000C4C03914168029181680191C16800913D
:10F67000036942691CA15B1C02F5FA62204600F096
:10F680008DFE204604B010BDC506F5FF8051010077
:10F69000442B0020C45C002080B5FFF77DFFBDE84F
:10F6A0000240DBE700B58BB06846FFF737FE6846DF
:10F6B000FFF7D4FF0BB000BD000000001F000000EA
:10F6C0003B0000005A000000780000009700000096
:10F6D000B5000000D4000000F3000000110100009C
:10F6E000300100004E010000253034642D253032F9
:10F6F000642D2530326420253032643A253032645E
:10F700003A25303264000000002202F051BFFEE7CB
:10F710005FEA000C80EA01039B0715D1830706D03E
:10F7200011F8013B00F8013BB3B18307F8D10A6837
:10F73000B2F1013323EA020313F0803F02BF40F825
:10F74000042B51F8042FF3E711F8013B00F8013BBB
:10F7500013B111F8013BF9E76046704780B502F03C
:10F760004DFF14E080B5002807BF00230C4900239B
:10F770000C4942F21072012002F05AFF0A4A01219C
:10F7800004E080B502F098FF074A0021117018B11B
:10F7900000F0ECFD4FF0FF3002BD034800787047E9
:10F7A000D99902002F1F0200855E0020A0F13002CF
:10F7B0000A2A81B038BF30380CD3A0F14103062BA0
:10F7C00038BF373806D3A0F16101062934BF573856
:10F7D0004FF0FF3001B07047F8B504460D460026E3
:10F7E000207870B1617861B1FFF7E0FF074660787B
:10F7F000FFF7DCFF00EB071005F8010BA41C761CDB
:10F80000EEE73046F2BDFEE718B50021174A0B4679
:10F8100008205C08DB07234644BF154C6340401EAC
:10F82000F7D142F82130491CB1F5807FEFD311495F
:10F830000120086011BD70B50D460E4904460868E8
:10F840004FF0FF3608B9FFF7DFFF0020074908E057
:10F85000225C724002F0FF0251F8223083EA162641
:10F86000401CA842F4D3F04370BD0000505000206B
:10F870002083B8ED445E00201FB50C4612494A684B
:10F88000029220B1D1F8002011A100F087FD6CB1E7
:10F890009DF808009DF80910019000919DF80A302C
:10F8A0009DF80B200CA1204600F078FD002004B04C
:10F8B00010BD000080B505490A684B6809A100F039
:10F8C0006DFD002002BD000000010010600000106E
:10F8D0006E52462578000000256325632563256365
:10F8E000000000002530385825303858000000004E
:10F8F00030B5134B1C68202C08DA0C2565431D44D9
:10F90000641C1C6045F8040F6960AA6030BD2DE9D5
:10F91000FC410B4D0FF22C0804462E1D002709E078
:10F92000B06800904146736856F80C2B2046FCF7EF
:10F930006DFE7F1C28688742F2DB0020BDE8F6815F
:10F94000285600206661756C74203A2025642C20AE
:10F9500025642C2025640D0A000000000000000032
:10F9600010B5040008D000BF95A14FF47A4041F0D3
:10F9700001018847641EF6D110BD00002DE9F04F4B
:10F9800099B04FF0000818901791144616931698E6
:10F99000804561D26078179915904144A078149001
:10F9A000E07813902079129060791190A279E37930
:10F9B000267A677A94F80AC094F80BE094F80C5011
:10F9C00094F80D9094F80EA094F80FB05FA01091E9
:10F9D00021780F911899F9B1CDF838B0CDF834A04D
:10F9E000CDF830900B9505920693CDF828E0CDF830
:10F9F00024C008970796119A12990F9B04920391BD
:10FA0000139A1499029201910146159A00920020CE
:10FA1000109AFEF7A9F81BE0CDF834B0CDF830A06D
:10FA2000CDF82C900A95049205931199129A03919E
:10FA30000292CDF824E01399149A01910092CDF826
:10FA400020C0159B0F9A109907970696FDF7D3FDD6
:10FA5000103408F110089AE7002019B0BDE8F08FC3
:10FA600070B504460129C0B088BF4FF0FF3019D8E7
:10FA70000D0300264FF480726946284602F04DFEC1
:10FA800000280ED44FF480736A4631022046FFF7F7
:10FA900075FF0120FFF764FF761C102E05F58075B9
:10FAA000E8DB002040B070BD2DE9F84F0D46032D76
:10FAB000C0B0834616460CD1706822A1FEF7D4FC74
:10FAC00038B9B068FEF724FC01465846FFF7C8FF76
:10FAD00034E001270FF270080FF2CC092BE056F842
:10FAE0002700FEF715FC8246BAF1000F25D45246D6
:10FAF00049465846FCF78AFD002404EB0A104FF4EF
:10FB0000807269460002FFF794FA60B94FF480737F
:10FB10006A4621025846FFF731FF0120FFF720FF18
:10FB2000641C102CE9DB681E874203DA4146584604
:10FB3000FCF76CFD7F1CAF42D1DB002041B0BDE87B
:10FB4000F08F00002D6900000D0A000025303458A8
:10FB5000203A2025303258202530325820253032A6
:10FB60005820253032582025303258202530325840
:10FB700020253032582025303258202D2025303293
:10FB80005820253032582025303258202530325820
:10FB90002025303258202530325820253032582048
:10FBA000253032580D0A0000536563746F722025AA
:10FBB000643A0D0A0A000000000000000000000086
:10FBC0000338FDD870470000E0B5002010210190F7
:10FBD00000914FF48073042200213C4801F020FF83
:10FBE00000200EBD10B50446FEF7D0FB241838489F
:10FBF0008462002010BD00007FB5354C20780128BC
:10FC000008BF4FF0FF303CD0FFF75CFC6060002085
:10FC10002081FEF7BBFB2F4E05463068962802D2A6
:10FC2000002161811DE0A16A2846FEF7B2FB00F5C4
:10FC3000E8405B306081B4F90A00401D0B2810D306
:10FC40006068FFF729FDB4F90A10238BE28A02915C
:10FC500031680191618B00914FEA000141A0FDF7ED
:10FC6000CAFCA56201F046FDA0811B480188E18124
:10FC70001A49088820821A480188618200200121DF
:10FC8000217004B070BD10B50346114C1022211D27
:10FC900004F1140001F0F8FE08B90021217010BD34
:10FCA0000B48C08A1EE038B50948C18A04290CBF38
:10FCB000052504250224284600F014F8042D0CBF65
:10FCC00005250425641EF6D1002032BD0C5C002001
:10FCD000F85B0020B83500203A5B0020DE370020BA
:10FCE0005E5D00202DE9F04389B0804600240FF2CC
:10FCF000A0092602002506EB08362701102205A9D7
:10FD0000A819FFF796F9059810F1010F22D0BDF858
:10FD10001800D8B90598FFF7BFFC0346BDF82200CC
:10FD2000BDF8201004900391BDF81E00BDF81C1012
:10FD3000029001914146BDF91A000090E81005EBD0
:10FD4000107007EB20124846FDF755FC1035B5F54D
:10FD5000807FD3DB641C102CCBDB002009B0BDE816
:10FD6000F08300002573203A206C6F6E6720696E67
:10FD700074657276616C202825642C2025642C2003
:10FD800025642C20256429202D3E2025640D0A00A1
:10FD900025642530336420202573202025642C2001
:10FDA00025642C2025642C2025642C2025640D0A34
:10FDB0000000000000000000000000000000000043
:10FDC00030B5039D049C41EA420141EA830141EAC6
:10FDD0000521414A41EA044142F8201030BDE0B516
:10FDE00000210191009100230122012105E0E0B5ED
:10FDF0000B460021002201910092FFF7E1FF07BDB1
:10FE000080B536480178012908D100211920FFF773
:10FE1000EEFF00211A20FFF7EAFF05E01920FFF7A7
:10FE2000DEFF1A20FFF7DBFF00210320FFF7DFFFD3
:10FE30001F20FFF7D4FF1E20FFF7D1FF1D20FFF783
:10FE4000CEFF00210220FFF7D2FF00211B20FFF789
:10FE5000CEFF00211C20FFF7CAFF002002BD204971
:10FE600000E020494FF00070086070471C4900E036
:10FE70001C494FF080600860704719494FF00040FE
:10FE800008607047164900E016494FF0804008604E
:10FE90007047134900E013494FF000500860704765
:10FEA00010484FF0804101604FF0005101604FF069
:10FEB00000410160704700000B480068C00E02E07E
:10FEC00009480068000F00F001007047064800680C
:10FED000C008F8E70000000000070050845E002022
:10FEE000080500500C05005010050050F8B50446F8
:10FEF0000D46A2F10C07A0B0394605F10C00FFF742
:10FF00009AFCA9683BA6884207D000BF3BA33246B3
:10FF100000212046FCF798FB25E06868042804D3FC
:10FF200031462046FCF79CFB1DE000973A46A86846
:10FF3000019005F10C0102A8FBF718FD686807F1B4
:10FF400008036A460021FEF7FCF8002807D408A33E
:10FF5000324601212046FCF777FB002005E03146C0
:10FF60002046FCF781FB4FF0FF3021B0F0BD0000D0
:10FF70005345540080B50846111F001D02F008FDCE
:10FF8000002002BD80B50846A2F10803C18800F137
:10FF9000080280889BB202F013FD002002BD10B55C
:10FFA0004B88012B07D040F20114A34206D0B3F5D1
:10FFB000817F06D008E0BDE8104097E7BDE810401B
:10FFC000D8E7BDE81040DDE74FF0FF3010BD44F644
:10FFD0004252028089B20122FDF779BDE0B54FF4AB
:10FFE0008071ADF80210ADF8040006216846FFF7F5
:10FFF000EEFF0EBD4443464700000000435243203D
:020000040002F8
:100000004572726F7200000070B4044604E015F887
:10001000016BB34203D1641C23781BB10D462A78CF
:10002000002AF4D1201A70BC704770B4044600E076
:10003000641C23783BB10D462A78002AF8D015F8C5
:10004000016BB342F8D1201A70BC704718B4047821
:100050009A4B1B5D1BB118BC001D02F0E2BE18BC20
:100060000C3003F056B91CB50178954C002942D0EC
:10007000022928D060D2017AD9B14168097804F107
:10008000180003F08BFA20B101218DF800100190C7
:1000900006E0206A616A081A05D000208DF8000089
:1000A0006846A16B8847206AA18B626A101A814258
:1000B00006D3012204F13D01201DFFF7C7FF13BD48
:1000C0000120207013BD8DF80010C06822797B4993
:1000D0000190885C38B1012204F13D0104F108006F
:1000E00002F09FFE25E0012204F13D0104F1100021
:1000F00003F00FF91DE004F13C0104F1280003F0C6
:1001000060FA98B921796D48405C38B1012204F158
:100110003C0104F1080002F032FE13BD012204F19B
:100120003C0104F1100003F073F813BD03208DF8B7
:1001300000006846A16B884713BD00002DE9F04719
:100140005F4D06460C0088B01F46AA6308BF072013
:1001500050D06268216892B205F1180003F00AFAE3
:10016000002847D1E268A16892B205F1280003F0A7
:1001700001FA00283ED100BF53A191E81C57684600
:1001800080E81C5771690691307C8DF81C70401E08
:100190008041C043C00F8DF81400707C00B10E2068
:1001A0008DF81500474AF0680290B06803903168F6
:1001B0000191694670680090281D03F02EFAC8B9B5
:1001C0002870306810F1010F13D02A793B49885C00
:1001D00038B1012205F13D0105F1080002F021FED0
:1001E00008E0012205F13D0105F1100003F091F84E
:1001F00000E0002008B0BDE8F08770B5304C2678EC
:10020000014604F1180003F0DCF90546BEB10021F7
:1002100021702A482179405C38B1012204F13D0166
:1002200004F1080002F0FDFD06E0012204F13D01A9
:1002300004F1100003F06DF808B100F0CFF8284683
:1002400070BD70B501461E4D05F1280003F0A6F9FA
:10025000040027D12979194E705C20B105F10800FE
:1002600002F0D6FD03E005F1100003F016F8C8B95E
:1002700005F13C0105F1280003F0A3F990B92979B3
:10028000705C38B1012205F13C0105F1080002F073
:1002900076FD06E0012205F13C0105F1100002F0B7
:1002A000B7FF0446204670BD0548016B406B411AFC
:1002B000481E8041C00F704700000000045E00200F
:1002C0001C37002067000200FFFFFFFFFFFFFFFF5A
:1002D000FFFFFFFFFFFFFFFF000000000000000026
:1002E0000000D601060100001F480021016441649E
:1002F0008166C166002070471B494A6C01EB82038E
:10030000521C082A986428BF00224A6400207047C3
:1003100015490A6C486C824201D10020704701EBFC
:1003200082004830521C082A28BF00220A64704705
:100330000D48016C406C814200D1704780B5FFF7D9
:10034000E7FFBDE8024003F0A5B907498A6EC86E11
:10035000824201D10020704701EBC200521C082AE2
:1003600028BF00228A6670476C5A00200149486500
:1003700070470000B835002038B5044600252046F7
:10038000FFF75FFF48B1042807D10120FDF7B0F85F
:100390006D1CB5F5FA7FF2DB0D2032BD0CB430B523
:1003A00083B0044606A802900A46002501940095F1
:1003B00002AB01A9084878441E30FAF7E7F9019921
:1003C0000D7000284EBF04460198041B204603B060
:1003D00030BC5DF80CFB00BF4BBCFFFF18B583B011
:1003E000694600220023002481E81C0002906A462E
:1003F000002144F20100FFF77BFA04B010BD002891
:1004000018BF002901D10E2070470278DE2A01D1E1
:100410000820704709684160DE2101704FF6FF71C6
:1004200007E008B90E2070470278DE2A01D00820C4
:1004300070474180002070470246107A58B15088BA
:10044000002166DF08B91172704711281CBF51687E
:100450000847012010727047F8B505460C0018BF18
:10046000002D84B04FD02078DE284CD1A988608838
:10047000814204BF2046FFF7DFFF2888012805D00E
:10048000112839D051280FD005B0F0BD287A0128A5
:1004900002BFA9886088814235D1012020722046A0
:1004A000FFF7CAFF05B0F0BDA8886188884204BF85
:1004B000A879022827D1A87B04281CBF0628052874
:1004C00021D16846002100220023002680E84E004A
:1004D0004FF4C0700227ADF804008DF80070A87BBF
:1004E000052808BFADF80410A8886946B0DF50B1F0
:1004F0006168884705B0F0BDA8886188884204BF5C
:100500004FF6FF70608005B0F0BDFEE730B50546E0
:100510000C4687B0A18868696A4603F025F918215E
:1005200001A8FFF7F1F80295A088ADF80C0000983B
:1005300004902989E088884204BF218A022913D1C6
:10054000009808B304F1120003F038F920B10099C3
:1005500001200870022102E00099087003218DF843
:100560000410A96981B10DE0A98988420CD1A9695B
:1005700051B100208DF8040004F112020592208A86
:10058000ADF8180001A8884707B030BD38B505465A
:100590000C0018BF002D8AB05ED02888102805D026
:1005A000502836D057283AD00BB030BD00200090EC
:1005B0006A46A988606903F0D7F802A800210022E2
:1005C000C0E9001201A80221ADF808100390ADF8AF
:1005D0000A202189A88802AAADDF00283CD1A069A1
:1005E000002839D0039803F0E9F8A8B3009808B1BF
:1005F00001210170182104A8FFF786F802208DF868
:1006000010000594A888ADF818000098079004A879
:1006100020E029462046FFF779FF0BB030BDA988BE
:1006200060696A4603F0A0F8B0B900980178002923
:100630001CBFA06900280FD0182101A8FFF764F89B
:1006400001208DF804000294A888ADF80C000098F1
:10065000049001A8A16988470BB030BDF0B500BF78
:100660004DA292E8E8008DB0040009A880E8E800F7
:1006700014BF00290E2058D00868A061214609A89F
:1006800062DF002851D120788DF802000121ADF8F9
:100690000010A21C69460120A8DF002845D12021B6
:1006A00001A8FFF731F80220ADF80400F42021780A
:1006B000ADF808008DF8061001219DF81100ADF885
:1006C0000A1040F00C008DF811008DF810108DF814
:1006D00015108DF8161004F10C02608801A903F0C2
:1006E00073F810BB202101A8FFF70EF80320ADF826
:1006F0000400F4202178ADF808008DF806100121DF
:100700009DF81100ADF80A1040F010008DF81100AE
:100710008DF810108DF815108DF816108DF8171033
:10072000221D608801A903F04FF80DB0F0BDF0B5AF
:10073000040085B00D4616461F4608BF0E2029D07E
:1007400060696A46394603F00FF818BB4FF6FF712F
:100750008F421ABF0098002805201BD0007810B9DE
:10076000082005B0F0BD3188F529A8BF072011DAAF
:1007700001A80021002200238C4680E80E10A088EA
:10078000ADF80400049501208DF80600039601A938
:100790003846AEDF05B0F0BD9ECADC240EE5A9E008
:1007A00093F3A3B50000406EF8B486881746BC19D1
:1007B000B24228BF3746F51BC2881F4607EB020C22
:1007C000934228BF1746D61B4A8803889A4224BF03
:1007D0004088904209D38888A84228BF844204D325
:1007E000C888B04228BF844502D2F2BC00207047BE
:1007F000F2BC0120704738B5804A04461089A1B286
:1008000088422BD17E4D107C297B88420FD202F189
:100810001201A0B275DF30B111281CBFA9690029EF
:100820001CD0884731BD107C401C107431BD0021A4
:100830001174287C48B13B21A0B276DF002818BF94
:10084000082802D0A96901B18847696931B100203F
:100850008DF80000ADF802406846884731BDF8B514
:10086000010001D10E20F2BD91E8FC10644880E83F
:10087000FC10624C04600868A8B17ADFB8B9096856
:1008800020460822FBF762F84FF6FF70208104F142
:100890002000E06000215B4A04F10C0003F0FEF848
:1008A00028B10320F2BD20467BDF0028ECD0F2BD4A
:1008B0001CB50B460246597A514C71B9187A00287A
:1008C00058680CBF6168A16803F0FAF800281CBFE3
:1008D000A16900290CD0884713BD002018726169F6
:1008E00031B101208DF80000ADF80220684688473C
:1008F00013BD2DE9FC4104462088102807D011289B
:100900002FD0122861D050283ED0BDE8F381E07B83
:10091000A58801286FD1394E394F30894FF6FF78BD
:10092000404519D100203074358106F1120031465E
:100930000822FBF70BF8434640F2F31204F11001D2
:1009400006F11200FFF730FF7074F889002852D1C9
:1009500006F1080128464BE0B96900294BD0042074
:1009600030E0264DA1882889884244D1E86803F008
:10097000D7F800281FBF22498969002988474FF608
:10098000FF702881BDE8F3811D4DE088E989884228
:1009900004BF208A022801BFA788184E3089B842B8
:1009A00029D104F1120002F009FF18B106F1080183
:1009B00038461DE0F06803F0B3F800281CBFA969B1
:1009C000002918D0BDE8FC4108470C4DA6882889AD
:1009D000B04210D14FF6FF7340F2F31204F1080158
:1009E00005F11200FFF7E0FE687405F108013046DA
:1009F000BDE8FC415CE7BDE8F3810000885B0020B6
:100A0000E45C0020F7070200417949B100F22E4171
:100A1000087828B98978481E8041C043C00F7047C4
:100A20000020704780F830107047F8B504460D007C
:100A300018BF002C01D10E20F2BD05F17A0001781B
:100A4000012904BF807F012831D005F19C07786817
:100A500004281CBF3968042929D00020A07005F1A2
:100A60007801201D2C22FAF781FF04F124060020D2
:100A700030730721B8683061F868706104F58267E7
:100A80004FF6FF70B8823F6104F2264003F06AF827
:100A9000207818B904F15002FF21117104F15500BA
:100AA0003860307801280CBFEE201F2001E00720BD
:100AB000F2BDB88004F2144204F15501284603F057
:100AC00094F928BB04F23121B96004F21C42307859
:100AD00001280CBFEE201F20B88105F13C0003F077
:100AE00084F9A8B904F150000121417004F13C02DD
:100AF000A169B184012131760021F1610170606941
:100B0000306204F1540072DF10B90120207000201F
:100B1000F2BD00002DE9FC4105460F46287810B9CA
:100B20000820BDE8F68105F22648AF70072140464F
:100B300003F018F8A87905F5826605F1240410B1D0
:100B4000A978012906D0E87968B1A878012818BFEA
:100B5000022808D1216921B1012070770820884737
:100B600001E000207077F07D002804BF317E00296D
:100B70000DD1707E002804BFB17E002907D1F07E20
:100B800028B9317F481E8041C043C00F00E00120DA
:100B90007F1E032F18D8DFE807F002090F13AA7988
:100BA00022B1217811B938B101200EE0E97900298C
:100BB0001CBF0028022008D1287A08B1032004E0D5
:100BC000687A08B1042000E00020A870216981B192
:100BD000A878032818BF04280BD16A794AB1B07FDE
:100BE00038B9002285F830240120F07707208847A3
:100BF00001E00020F077182105F13C00FEF784FDAC
:100C00000120207605F15007A06801281CBF0228AA
:100C100001207870207828B1616801291CBF022961
:100C20000121B97000213970A978042943D8DFE87F
:100C300001F074030F1F5100012060730020306128
:100C40002062C4F81C80022020768020A08434E03A
:100C50000221002814BF0720032020766173286931
:100C6000A08400203061C4F81C80E868206224E081
:100C7000696921620028A969A18414BF06200120A6
:100C800020762846FFF7C0FE90B10220387001227E
:100C9000B188306803F0E5F908B10421017005F16D
:100CA0003C02314605F1540072DF20B9052000E016
:100CB000032060733661A87888B3316905F13C027E
:100CC00005F1540072DF78BB217B387973DF30B3D4
:100CD000BDE8F681E96921620028296AA18414BF70
:100CE0000620012020762846FFF78EFE98B10220CC
:100CF00038700122B188306803F0B3F908B10421DB
:100D0000017005F13C02314605F1540072DF002804
:100D1000D1D10620CDE70420CBE700206073216904
:100D200009B1607B88470020BDE8F6811CB50C4600
:100D30000188102904D0112909D0262914D013BD07
:100D4000C17B01292BD18088A4F8240413BD04F2AF
:100D5000244100228A7280880988884204BF207951
:100D600000281CD101210FE0007A012818BF0228B9
:100D700015D1A078401C81B24CF6CD424A43910C6B
:100D800001EB8101401AC1B22046FFF7C3FE0028E3
:100D90001CBFA16B002902D0BDE81C40084713BD51
:100DA00010B5040008D000BF8DA14FF47A4041F087
:100DB00001018847641EF6D110BDFEB50022CDE9C1
:100DC0000022012842D1022000900190FFF74EF846
:100DD0006420FFF7E5FFFFF74BF800F05BF803F046
:100DE0004FF9FFF743F86420FFF7DAFFFFF740F809
:100DF00000F050F803F044F9022600275DF8275070
:100E000015F0010418BFFFF72AF815F0020518BF06
:100E1000FFF72CF86420FFF7C3FF0CB1FFF721F8B0
:100E20000DB1FFF725F800F035F803F029F97F1C24
:100E3000022FE3DB761EE0D104244FF4FA70FFF7B3
:100E4000AFFF03F01DF9641EF7D1BFE7022804D1FC
:100E50000120009002210191B8E7042810D1FFF78A
:100E600005F8FEF7FCFF4D4C02E003F009F930BF36
:100E7000A07E0028F9D0FEF7FBFFFEF7F2FFF7BDDA
:100E8000032802D100900321E5E7052808BF0120CF
:100E90009AD0F7BD4FF4C87082E780B53DE080B5C9
:100EA0004DE03F480168491C0160C80748BFFEF794
:100EB000D6BFFEF7DBBF3A480178CA0748BFFEF746
:100EC000D0BFFEF7D5BF36480168491C016003203A
:100ED000B1FBF0F000EB4000091A012908BFFEF752
:100EE000C5BF70472E4800680321B0FBF1F101EB4C
:100EF0004101401A012808BFFEF7BABF70472848D1
:100F00000168491C01600320B1FBF0F000EB4000D8
:100F1000091A012900D0704780B5FEF7A7FFBDE888
:100F20000140FEF79CBF1E4800680321B0FBF1F1B1
:100F300001EB4101401A012800D0704780B5FEF74F
:100F400097FFBDE80140FEF78CBF10B50446FEF7E1
:100F50008FFFFEF786FF012C20461249124A18D057
:100F6000022C02D11149124A13E0032C02D111497B
:100F7000114A0EE0042C02D11049114A09E0052C57
:100F800002D11049104A04E0062C06BF0F49104A4E
:100F90000120104B9A605960186010BDB8350020D0
:100FA000585E00205FFE010063FE01006DFE01003F
:100FB00071FE01009B0E02009F0E0200A30E0200B4
:100FC000B70E0200C70E0200E50E0200FF0E02007F
:100FD000270F02009C3500200000000000000000E8
:100FE0000338FDD87047000080B50D48017801290D
:100FF00007D1FEF7D2FB20B90A49012081F804018C
:1010000001BDFEF7CAFB012805D1BDE80440C82197
:10101000002003F0D5B8BDE802400920FFF76CB905
:10102000845E0020F43700202028014604DA73484B
:10103000C84000F001007047402808DA0122A1F101
:10104000200012FA00F018BF0120C0B27047012042
:10105000704700001FB5044678A1684603F0D5F834
:1010600002E0684603F0E2F8029A3AB15168126869
:10107000204690470028F4D1112000E0002004B061
:1010800010BD00001FB504466FA1684603F0BDF80F
:1010900006E05168126820469047684603F0C6F89B
:1010A000029A002AF5D11FBD80B51620FFF7BCFFBC
:1010B00028B942F20100BDE80240FFF78FB950485D
:1010C00000784009082803D2EC21C140C80702D4A7
:1010D00042F20200EFE74B49886820B10A6842F407
:1010E00080020A6001BD48494FF48000086001BDDC
:1010F00080B51620FFF798FF28B9BDE8024042F2FC
:101100000100FFF76BB93F49886820B10A6822F4F3
:1011100080020A6001BD3D494FF480000860BFF3C2
:101120004F8FBFF36F8F01BD3EB5394D287808B1A1
:1011300008203EBD0121A970FFF78CFF112820D0A7
:101140000020FFF79FFF00BF45A00168019100222A
:101150008DF80020684603F079F82E4901A810DFC9
:101160000446401E8041C00F00F034F80CB1204608
:101170003EBD0020A8706870FFF796FF0120FFF7C2
:1011800081FF00203EBD38B5214D287808B90820E0
:1011900032BD0121A9700120FFF75CFF112817D093
:1011A0000220FFF76FFF00208DF80000684603F073
:1011B0004DF811DF0446002000F00CF80CB1204679
:1011C00032BD0020A870FFF793FF0320FFF75AFFFE
:1011D000002032BD28709DF8000003F053B80C4881
:1011E000817809B9082070470078002818BFFFF7F8
:1011F000CABF99E70648007870470000FC06FFBDAB
:1012000016E400E0EC5D002000E100E080E100E099
:10121000805E0020F1F80100E0B500BF0DA1684636
:1012200002F0F3FF05E0486809688847684602F065
:10123000FDFF02990029F6D107BDEDE7A49E02004B
:10124000B49E020008000000B49E0200C49E02008A
:1012500008000000C49E0200D49E020008000000A6
:10126000020000053EB50B00044601D10E203EBD34
:1012700040481860002168460022002580E82600CA
:10128000012006218DF800408DF80200ADF8041011
:1012900069461A68202069DF00F037F801208DF8D0
:1012A000010069461A68402069DF00F02EF8F72037
:1012B0008DF80040ADF8020069461A68232069DF06
:1012C000684600210022002480E8160001208DF8E5
:1012D000000069461A6869DF00F011F84FF4B06049
:1012E000009069461A68A12069DF00F008F88DF8BF
:1012F000001069461A68A02069DF00203EBD6846DC
:101300000021002280E81600704768460021002274
:1013100080E82600704760DF10B9174A012111707C
:1013200070470000144900B50878ADF5017D88B913
:1013300003E0052818BFFFF751F80DF5017D00BD4A
:101340005168126804A8904701A802F06FFF039A41
:10135000002AF5D14FF4FA70ADF80000694604A8F0
:1013600061DF0028E5D100BF04A101A802F04DFF14
:10137000EDE70000B82A0020835E00208CA0020068
:10138000ACA0020008000000F72101801721418075
:10139000002101714171FB2181711B21C1717047D5
:1013A00030B400BF6EA284B0D2E90045CDE900455B
:1013B000ADF80010ADF8021067A1D1E90023CDE926
:1013C0000223694602AA21E008B90E207047016194
:1013D000F72101804180FB210171F721C180172194
:1013E000018100218172C172FB2101731B214173B4
:1013F0000020704708B90E207047A1F11702E12ABA
:1014000001D30720704701800020704790DF04B0AF
:1014100030BC7047F0B502468BB0908800280C466F
:1014200040F09880118810290BD0112919D0232958
:1014300000F07D8024295DD03A2916D055293AD074
:101440007FE0A01D21798171D27B012A03D0022A7D
:1014500003D1628800E022880280C079884270D27D
:101460006CE0A01DFFF790FF6BE0A51D5089298857
:10147000884228BF0846688068881728B8BF1720A8
:101480006880216900291CBF687900280FD000BF3F
:1014900035A10020D1E90023CDE90023ADF80200F9
:1014A00069466888ADF8040020462269904700200C
:1014B0006871287145E0D088A21D17281188B8BF2F
:1014C0001720884228BF0846508000201071B5DFE1
:1014D0005179002935D12069002832D024A100207B
:1014E000D1E90067CDE90067ADF802005088ADF89A
:1014F000040017E0111D68462C22FAF737FABDF8F0
:101500000010BDF8040004EBC10250732069C0B1A3
:1015100019A3D3E90067CDE90067ADF80210507B4D
:101520008DF80400694622692046904709E0A01D15
:1015300012898179D2B2914288BF11460020FFF70B
:101540002FFFA07A30B1E1880020A5DF10B9A0728A
:101550000120E0720BB0F0BD0000000000000000B0
:101560000000000000000000770A000000000000FA
:10157000770A0000000000007ADA00000000000096
:1015800012F003030FD1094B9A6001F1010C4FEAED
:10159000CC4C02EB1C42DA6000225A701A70588060
:1015A000998000207047072070470000C05D002030
:1015B00080B5FAF761F9801C032190FBF1F08000FF
:1015C00002BD00002DE9FC420500144618BF002CA6
:1015D00089461E4603D0FFF7EBFF864241DA002022
:1015E0003DE0021D954249DB9CF800209208B25C68
:1015F0000A5438469CF800709CF801203F0107F01F
:10160000300747EA22171A19F75D0F541F197F7820
:101610009278BF0007F03C0747EAA217401CF75D2D
:101620000F54401C1F19E41CBF7807F03F07F65DFC
:101630000E54401C1AE01A192D01527805F030059D
:1016400045EA22151A19755DCD55527802F00F0240
:1016500016F822300B54401C3D220A54401CBDE8B1
:10166000F6822B462146354600240020471CA9F16E
:101670000202944203EB040C0BA6B2DB4C45EEDAFB
:101680009CF80050AD08725D0A54781CA9F1010263
:101690009CF800509442CED105F003052D01725DF7
:1016A000CA553D220A54D6E75137535466696A67D2
:1016B00068775A306E5770715573494A364C4142BB
:1016C000797A444345334748753459784D39504FFA
:1016D0006164386272566F586B6C6D313246763584
:1016E0004B52634E74652B2F000000001F490860A9
:1016F000002070471D48006870477CB51C481B4E91
:1017000001786424012940F2C67512D1FEF7DEFB90
:10171000012813D1306840F6C411884201D36320F8
:1017200076BDA8420ED3A0F2C67044434FF4FF70BA
:101730000FE0306840F64C11884201D3642076BD3A
:10174000A84201D2002076BDA0F2C67044434FF4F7
:10175000C370B4FBF0F076BD04480168B1F5006FCA
:1017600002D204480122427570470000B42F0020C5
:10177000845E0020B835002010B50446FAF704F85E
:1017800001462046096ABDE81040084710B50446E6
:10179000F9F7FAFF01462046896ABDE8104008477C
:1017A00028B10FF28C31800141F0010108477047E8
:1017B000C1888289491CC18089B2914210D100211F
:1017C000C1808188C289491C818089B2914207D138
:1017D00000218180428841898A4208BF491C41809A
:1017E00070472DE9F44F94B08B4606464FF4805075
:1017F000318A90FBF1FA0AEBDA704FEA60084FF099
:10180000FF30039001904FF0000904A8AAF1010AEB
:101810000024009013E00021039128790228C8BF1A
:10182000641C00F0A3F808FB0030FDF702FC00F098
:1018300098F841D1C24600F08DF801200190AAEB42
:10184000090008286BDA009800254F4606E0029A46
:1018500005A98B5C022BC8BF641C7F1CBA455DDBED
:101860006801029004A8029901440091308A3388EB
:101870004FEA0B3C02460CEB034307FB0030FDF73D
:10188000D8FB009801686D1C11F1010F05F00105EE
:10189000DDD1B089A6F802B07F1E97FBF0F1B180D0
:1018A00000FB117704A8F78000EB4511328A1498E9
:1018B000FAF74CF800202EE0287902280198C8BFDA
:1018C000641C10F1010F21D1308A3388024607EBE6
:1018D000034704A90AFB0070FDF7ABFB00F041F8D9
:1018E00008BFC146A7D0328A149804A9FAF72EF887
:1018F0009DF814000228C8BF641C022C0ADD0020D9
:10190000A6F802B0B080F080012004E0C14600F0EB
:1019100021F894E7022015B0BDE8F08F00900398FD
:1019200010F1010F04AD7FF47CAF00F01FF809FB4C
:101930000030FDF77EFB00F014F87FF46CAFB08947
:10194000A6F802B099FBF0F100FB1199B180A6F85E
:101950000690D9E7AAEB090000EBD07009EB60080C
:1019600070470098016811F1010F7047308A338881
:101970004FEA0B37024607EB034304A97047F8B55B
:10198000C2B005460C460027698902A800EBC716BD
:101990007918324689B22846FFF723FF4DF8270011
:1019A00080B17F1C022FEFDB0020A880E880009828
:1019B000022811D10198022817D122980299884251
:1019C00020D214E024B12A8A31462046F9F7BEFF1E
:1019D0002846FFF7EDFE1DE001281DD101990129E0
:1019E0000ED168896880012018E0012814D124B143
:1019F0002A8A02A92046F9F7A9FF6889401C08E055
:101A0000022909D124B12A8A22A92046F9F79EFF8A
:101A100068896880002001E04FF0FF3043B0F0BDDE
:101A20002DE9FE460A9C212CBFBF1D4605FB04F391
:101A300041F20106B34202DA0E2A164605DD0720FE
:101A4000FEF794FC4FF0FF301CE0DDF82C908A4646
:101A50000746142102F086F8A7F800A0002038817C
:101A60007E814FF4807090FBF4F0B8814946B889CC
:101A700095FBF0F0F8817D823C82384603B0BDE8EA
:101A8000F0467CE7BDE8FE86F8B505460C46288999
:101A9000012816461F4605D1FDF733FB012811D05A
:101AA00002202881A988002904BFE88800280FD1D6
:101AB000288948B968883946FDF730FB012F07D1DE
:101AC000012028811120F2BD022804BF00202881B6
:101AD000FCF75CFC074668882B88000300EB03409A
:101AE000AB88214600EB03202C8AEB88B2B203FBC3
:101AF0000400FDF774FB04464620FFF751FEFCF797
:101B000045FC3946FCF745FCC928084E02D330880D
:101B1000401C30802846FFF74BFE0CB90020F2BD78
:101B20003088401C30802046F2BD00005E5D002001
:101B30000338FDD8704700000000000000000000DE
:101B400028B10FF25C31800141F001010847704774
:101B5000C1884289491CC18089B291421BD30021AE
:101B6000C1808188491C818089B2102913DB002142
:101B700081804188491C418089B210290BDB0021FA
:101B800041800188491C018089B2C289521C91425E
:101B9000A4BF81890180002070477FB504461503EA
:101BA000668905EB0145761E05EB032512E000F082
:101BB000B4F8009911F1010F04BF019810F1010F61
:101BC0001ED1029911F1010F04BF039810F1010F0A
:101BD00016D1761E002E0FD4208A1022694606FBED
:101BE0000050FDF726FA0028E1D54FF0FF3005E060
:101BF000761CE680002001E00020E08004B070BD8B
:101C00006089401E8642F3D1E6802046FFF7A0FFA0
:101C1000F0E72DE9FF4216468946370304460F25B3
:101C200007EB09471022694607EB0520FDF701FA8B
:101C3000002819D400F071F8009810F1010F04BFCA
:101C4000019911F1010F12D1029810F1010F04BF97
:101C5000039911F1010F0AD16D1EE3D50020A08078
:101C6000E08004B0BDE8F0824FF0FF30F9E7A580D6
:101C70002B46324649462046FFF78FFFF1E7F8B57D
:101C80000D4684B004460F272E041022694606EB49
:101C90000730FDF7CEF9002819D400F03EF800987F
:101CA00010F1010F04BF019911F1010F12D1029837
:101CB00010F1010F04BF039911F1010F0AD17F1E2A
:101CC000E3D500206080A080E08005B0F0BD4FF03B
:101CD000FF30FAE767803A4629462046FFF799FF2A
:101CE000F3E7F8B504464FF0FF35A689374607E01D
:101CF00000F013F80099A9423CBF0D463E467F1CF8
:101D0000E089B84207DB042269463804FDF791F9FF
:101D10000028EDD5B9E03046F2BD462010E7DFB52A
:101D200006464FF6F074B78912E0FFF7F6FF009908
:101D300011F1010F04BF019810F1010F07D10299B1
:101D400011F1010F04BF039810F1010F0ED07F1C99
:101D5000F089B84210DB1022694604EB0740FDF71A
:101D600068F90028E1D54FF0FF300DE037803946A3
:101D70003046FFF784FF07E03046FFF7B2FF3080C0
:101D800000207080B080F08004B0D0BD2DE9F0411B
:101D90000E46069C054617469846122101F0E2FEC3
:101DA00000202881002E4FF4807090FBF7F06881AE
:101DB0002F82A5F80C80EC8103D52846FFF7AFFFF2
:101DC00000E02E80288800050021000CFDF7A6F910
:101DD0000020BDE8F081F8B505460E4628890128A7
:101DE000144605D1FDF78DF901281CD00220288169
:101DF000A988002904BFE88800281CD12889B0B927
:101E0000EB8969882A889A4208BF0F2901EB0210E2
:101E100002D10121102002E0401C012180B2FDF717
:101E20007DF9012028811120FEF7A0FA2DE002287B
:101E300004BF00202881FCF7A9FA07466B88288890
:101E400031461B03AE8803EB0043E888A2B203EBE4
:101E5000062300FB04342046FDF7C1F90446FCF7D5
:101E600095FA3946FCF795FAC9280A4E02D330880C
:101E7000401C3080FFF751FF2846FFF769FE0CB980
:101E80000020F2BD3088401C30804FF0FF30F2BDA2
:101E9000000000005E5D0020000000000000000067
:101EA0000338FDD87047000010B56F4C6060A1602A
:101EB000E260236110BD000038B56B4C606890B3E0
:101EC00021696A4D91ED000AAA6CDFED660A60EEA9
:101ED000200AFCEEE00A10EE900A904238BF10464D
:101EE000A86443F69821E86C401C8842E86405D356
:101EF0000020E86402F00EFA0020A86461680A88F5
:101F000020885D3A0F2A0BD2401C208042F22931F2
:101F100080B2884207DBBDE832400320FEF7ECB90F
:101F200008B10020208031BD51494861704770B52B
:101F30004E4C4F4D2068401CC107206041D54D4894
:101F4000017801295DD0686802F014FA0646E06B5A
:101F5000308040F6FF7188420CBF0120401CE063D6
:101F6000206C18B1328844490A433280207D18B170
:101F7000318841F4804104E0607D18B1318841F43A
:101F800000513180B01C02F052FA88B9FCF7FEF91A
:101F9000E860B01C696988470446E868FCF701FA04
:101FA0002969401828613CB1E0B202F099FA03E0D7
:101FB000308840F4805030806868BDE8704002F09E
:101FC000DBB92968884203D30A31296002F0C2F8DC
:101FD000A868804729480168002912D4284A106857
:101FE000002804D4BDE870400020FBF7B9BE2548A6
:101FF0000168002905D4BDE870404FF0FF30FBF7C1
:1020000096BF70BD80B51021962002F08DF9184A58
:10201000506010B94FF0FF3002BD14484D214160AF
:1020200057218160FFF798FB0A21022002F0C8F8CF
:102030000320FEF78AFF02F0AFFA002002BD0B4931
:102040000A686423B2FBF3F3642000FB13234D2BD7
:1020500002D24D32D21A02E06432D21A4D324A60B4
:10206000704700000000C842885D0020B83500209D
:102070001C360020845E00200080FFFF9C2F002083
:10208000A02F0020A42F0020CB074CBF0923002342
:10209000D380C1F34303C1F3431193805180108077
:1020A00070472DE9F04104463C4F208878809846DF
:1020B000B980154660882388000300EB0340A3889D
:1020C000E4880E2600EB03207E22B91D06FB0400E7
:1020D000FCF7AFFF002807D4B7F90610002904BFAA
:1020E000B7F90800002802D14FF0FF300EE0012DB3
:1020F00004D100F035F84643B61D00E08426424680
:10210000B1B23846BDE8F041FBF7E1BCBDE8F08173
:102110007CB515460C461E466A46FFF7B5FF3346AA
:102120002A4644F400416846FFF7BBFF76BD38B548
:1021300004461B481B4A13680D46016899420DD09E
:10214000FEF703F90168042906D14068010C2B460B
:10215000224680B2FFF7DCFF012032BD002032BDF5
:1021600010B500203E210D4A02EB4103B3F90640B1
:1021700014F1010F02D1401C491EF5D50721B0FB17
:10218000F1F0C0F1090010BD024604484FF6FF719E
:10219000418081800621FBF79ABC00002434002096
:1021A000D45A0020D85A00202DE9FC4704460F4697
:1021B0002179DFF8CCA24FF02C0818FB01F00AEBD4
:1021C00000051646287F994610B10820BDE8F6871D
:1021D0000FF2CC22206852F8211002F020FA10B140
:1021E0001120BDE8F6872E60C5F804903A783B7B55
:1021F000A448012101FA02F2012BD4BF426002601F
:10220000A14A97F800C042F82C107B78FF2B06D02B
:1022100001FA03F64660032642F8236001E04FF01E
:10222000FF3397F802C0BCF1FF0F1ABF002642F837
:102230002C604FF0FF3C94F804E0BE7818FB0EFED3
:10224000D6448EF81F60FE78FF2E07D001FA06F6FE
:102250000660032097F803E042F82E002079FA7810
:1022600018FB00F05044827720683A7800F5A060AF
:102270008260C360C0F810C0BA6842627A7B3B7B60
:10228000521E9241D243D20F012B09D00AD3032B05
:1022900003D038BF42F0040204E042F0060201E03D
:1022A00042F00202426522797B7918FB02F80AEBC0
:1022B000080282F8203001602868D0B120683A799D
:1022C000000300165201002802D4704B1A5405E096
:1022D0006F4B00F00F00184400F8042C2268120322
:1022E000121606D402F01F006A4B8140520943F8CF
:1022F000221000206877012028770020BDE8F687AB
:1023000038B400F5A36210688DF800008B69486A44
:10231000984203D29DF800304C6923544B6A91F8DF
:1023200028005B1C4B625C1C48B10869844298BF62
:10233000204608618869844298BF20468861086900
:10234000844203D2C868005D50600DE08D69AC42E4
:1023500003D291F82000506006E0834204D3AB42E0
:1023600032BC8041C00F704732BC01207047F8B5C5
:102370000579434C2C2313FB05F52C440025667F7F
:102380000EB11120F2BD23680BB10126667704F16E
:102390000C0391E8C05083E8C050A37F84F8285014
:1023A000FF2B04D0012606FA03F3364E736012B1F8
:1023B0006577062540E00668656206F541720420EF
:1023C0005060C6F80851D6F808010090009B486894
:1023D00000281ABF0B68187894F82000C6F81C056E
:1023E0004868022804D309684878C6F81C0506E046
:1023F000C868022824BF94F82010C6F81C1520686D
:1024000010B10421116017E0D6F808010028FBD0B4
:10241000C6F80851D6F808010090304600992146C8
:10242000FFF76EFF0028EFD1A07FFF2804D0012125
:1024300001FA00F0134908602846F2BD1CB51648A1
:102440000F4C00210160006800900099134821465C
:10245000FFF756FF90B9A07FFF2804D0012101FAB1
:1024600000F00849086000206077207261682268E7
:1024700004F1080002B0BDE81040104713BD000091
:10248000245C0020080500500007005000E400E034
:1024900018ED00E000E100E00831024000300240A9
:1024A0003D2402001CB5049C0094001D02F01BFB9F
:1024B00016BD00007FB504460D4616464FEA0D00D6
:1024C00037A11022F9F752FA009501960023002255
:1024D0006946204602F0D4FB20B1FDF747FF4FF0DC
:1024E000FF3003E0201D02F02CF9002004B070BD85
:1024F00010B5094C082209212046FFF7DBFF30B94F
:102500000622072104F11000FFF7D4FF18B1FDF7F0
:102510002DFF4FF0FF3010BD3436002038B5044693
:10252000012000900D462046FFF7BCFF30B9059B07
:10253000049A2946201D02F0EFFA18B1FDF716FFA4
:102540004FF0FF3032BDF0B585B00024002501AE5C
:1025500005E0102C18DA575D3755641C6D1C9D4240
:10256000F7DB0B9A0A9B002595420FDA102CBFBFB0
:102570005F5D3755641C6D1CF6DB05E0FDF7F6FE6C
:102580004FF0FF3005B0F0BD0720F7E701220092C1
:10259000E3B201AAFFF786FF0028EFD1F2E70000BF
:1025A00000000000000000000000680602010000BA
:1025B00000B500BF130096469446103928BFA0E826
:1025C0000C50FAD85FEA417C28BF0CC048BF40F8E5
:1025D000042BC90728BF20F8022B48BF00F8012BA5
:1025E00000BDFEE7B0F5A07F07D13A49087808B9E9
:1025F00002224A708868496808477047E0B500BF02
:1026000038A00021D0E90023CDE900238DF8011086
:102610008DF8021004218DF800102F4A2FA0694672
:1026200002F0A2FB10B92B4A0121517003B000BD8A
:102630002DE9FC4704460F46380091461E4608BF68
:102640000E2037D0012C07D14FF00108214D6878BA
:1026500050B90820BDE8F687200008BF4FF4807805
:10266000F4D00720BDE8F68703280FF2700A05D1E1
:10267000504602F0EBFB0220687001E0022802D114
:10268000504602F0E7FB2C706F60AE6001200090B6
:1026900043464A460021504602F0FAFB6878022879
:1026A000504602D102F0CEFB01E002F0BEFB032057
:1026B00068700020BDE8F68710B5064C61780329E4
:1026C00005D100BF05A002F0C1FB0221617000200E
:1026D00010BD0000F85D0020E525020000900040DC
:1026E000010400000000000600000000704780B5F3
:1026F00000222D492D4802F025FC18B1FDF736FEC9
:102700004FF0FF3002BD10B5284C00E041DF2046FD
:1027100002F09AFC0028F9D110BD80B51346B0F53F
:10272000CE2F3EBF1A18521EB2F5CE2F06D200F0A1
:102730001EF802F012FC18B1FDF718FE4FF0FF3042
:1027400002BD80B51346B0F5CE2F3EBF1A18521EFB
:10275000B2F5CE2F08D20022009200F008F802F065
:102760001FFC18B1FDF702FE4FF0FF3002BD0A4614
:1027700000F5C8310D48704780B50A46B0F5CE2F38
:102780003EBF00EB0231491EB1F5CE2F08D200F555
:10279000C8310023054802F033FC18B1FDF7E6FD0F
:1027A0004FF0FF3002BD0000ACA00200E037002077
:1027B00080B5DFF8C003DFF8C0230168D2F8000459
:1027C000814228BF00F0BFF9002002BDDFF8A80356
:1027D000D0F80C14890AA0F80A14704780B5014695
:1027E0004FF4B2624FF4CC20FFF797FFBDE80140F1
:1027F000FFF789BF10B5044601214FF4CC20FFF745
:10280000BBFFFFF780FF4FF4B26221464FF4CC20AC
:10281000FFF797FFBDE81040FFF775BFF8B5ADF5BE
:10282000B26D07460C4615466846FFF7D7FF4FF6D0
:10283000FF718F42E2AE07D0B7802FB9CE48D0F8F3
:102840000C14E291FFF7C2FF2CB12A462146E4A8FE
:10285000F9F77CF8F5806846FFF7CCFF0DF5A06D21
:1028600025B0F0BD18B55968C44BCA689A4215D155
:10287000C34C616842688368002904BFA0680028CF
:1028800003D00021217011BD521C10785B1E01067F
:10289000FAD4511C01206160A360207011BD30B5D5
:1028A0000A46ADF54F7D014604A802F04AFC00F04F
:1028B0004AF8B448B24C03904FF44771002020709E
:1028C0006060A06008A8FCF71FFF4FF4477108A8DC
:1028D000FCF71AFF08AAAC49684602F0F6FE30B3CE
:1028E0009DF88C0100281EBF63ADA879002826D072
:1028F000A268616804A802F024FC00F024F84FF4F8
:10290000B27165A8FCF700FF65AA9C49684602F011
:10291000DCFE20B90FF28020FAF76DFE07E0286F89
:102920009A49884206D348F20100FDF757FB4FF061
:10293000FF3005E09049C1F80C04FFF747FF002085
:102940000DF54F7D30BD684604A91022F9F70EB889
:1029500080B58F4908804FF46C30C860FFF736FFB0
:10296000BDE80140DCE080B5ADF5B26D6846FFF72B
:1029700035FFE29810F1010F06D07F49C1F80C0431
:10298000BDF88C03FFF7E4FF0DF5A06D25B000BD89
:1029900038B504460D46FFF782FF00280FD476486D
:1029A000D0F80C140FF20C20FAF725FE2A46214627
:1029B0000020FFF733FFBDE832400020C8E731BDFB
:1029C0002DE9F84FDFF8B08108F2044593462A88D4
:1029D000814690421F4618BF4FF0FF3045D1C1F3EA
:1029E0000E06CC0BB246BAF1070F08BF012405D082
:1029F00026B949460FF2DC10FAF7FDFD012000FA76
:102A000006F6688830422FD159463A4608EBCA107C
:102A1000F8F79CFFA8883F18AF80688806436E804F
:102A2000E88881450DD12888A968800210FA87F0CE
:102A3000884216D100F01BF8FFF765FE00F02FF872
:102A400012E0B6B2FF2E0CD100F011F82888401C1D
:102A500028800022002180B2FFF7E0FE00F060F83D
:102A600002E00CB100F06FF80020BDE8F28F70B505
:102A7000414C04F204452888EE6810F0030F06EB81
:102A8000802605D101213046FFF776FEFFF73BFE99
:102A9000AA8821463046FFF754FE002070BD38B5A5
:102AA000ADF5B26D6846E2ADFFF798FE4FF0FF342A
:102AB000EA88E294E4A917A8F8F758FFE8880E908E
:102AC0000F900146E4A8FCF7B6FE324DE96810907D
:102AD00014911591286900F5C830FCF7ACFEE9683F
:102AE00009911290002113900A90089104910120FD
:102AF00001210B90059101A85821FCF79CFE009044
:102B00006846FFF777FE2C600120FDF767FA0FF2A9
:102B1000D000FAF770FD0DF5A06D002025B030BD96
:102B2000E0B51C4800210181C18040F20313114926
:102B30000A68ADF8023002F59672026006218088BC
:102B4000ADF8040011E0E0B50A4912480A6881882E
:102B5000ADF8041002F5967202604FF48273C088DB
:102B6000ADF80600ADF8023008216846FDF72FFAEF
:102B70000EBD0000B8350020882B0020407F0200E9
:102B8000E05D002065280200608002000140020034
:102B90008C2F0020882F002070625F6465636F6453
:102BA000652829202D3E206661696C65642E0D0A1A
:102BB0000000000050444655203A206170705F7359
:102BC000697A652C2025642062797465732E0D0A5C
:102BD0000000000050444655203A2025640D0A00AC
:102BE00050444655203A2066696E69736865642EC4
:102BF0000D0A000018B40A6812F1010F0BD001236E
:102C000003FA02F2DFF854341A60DFF854340C6827
:102C1000032243F824204A6812F1010F04D0DFF8A0
:102C20004044002344F822300268886902F22453A9
:102C300018604C7D087D04439C6448680B6802F270
:102C40000C542360A060087D01281ED1886810F113
:102C5000010F04D0DFF80844002344F82030C8688E
:102C600010F1010F0BD0012303FA00F0DFF8EC3371
:102C70001860DFF8EC33CC68032043F8240002F539
:102C8000A1628868C9681160906011BC704700003B
:102C9000F8B504460E462179DFF8C803174601EB64
:102CA000C10200EB820595F8200008B10820F2BDB2
:102CB0000FF2C832206852F8211001F0B0FC08B1C0
:102CC0001120F2BD31462046FFF794FF6F60306956
:102CD00028606868002845D02068317F0022C0F84D
:102CE00010214901D0F8102100920022009BC0F869
:102CF0002021D0F8202100920022009BC0F824213E
:102D0000D0F8242100920022009BC0F84421D0F882
:102D1000442100920022009BC0F85821D0F858218D
:102D20000092009BDFF84023C0F804230003001644
:102D3000002803D4DFF83423115406E0DFF83023F1
:102D400000F00F00104400F8041C21680903091664
:102D500008D4012201F01F00DFF81833824049092E
:102D600043F8212021680820C1F800050020A8614F
:102D7000E8616861012085F820000020F2BD78B488
:102D80000479DFF8E03204EBC40503EB850301F0BE
:102D90006045B5F1005F1C462AD15B695BBB62618F
:102DA000A1600021056805F590731960186800900E
:102DB000009AC5F85811D5F858010090009A60693A
:102DC000A66805F24452166050600120A860606851
:102DD000D8B91A68501E80419A6BC043521E924166
:102DE000D243D20F52EAD070F3D03AB10F210AE0A9
:102DF00072BC1020704772BC112070470120E8603F
:102E0000986B0028FCD000226261084672BC7047B3
:102E10000079944900EBC00201EB82014B69581E16
:102E200081E02DE9F84103468E4E187900EBC0048D
:102E300006EB840C0F4607F06044B4F1005F1AD132
:102E4000DCF80400002538B1D3F800E00EF5417835
:102E50004FF40474C8F80440DCF818409CB1DCF866
:102E60001C505DB120B119684FF40470C1F804031F
:102E70001120BDE8F2811020BDE8F2810125CCF8D7
:102E80001010104604E0CCF81820CCF80C100020EC
:102E9000CCF81C000024196801F5887ECEF80040AB
:102EA000DEF8000000900098C1F84441D1F84401D8
:102EB0000090009801F234500760426015B901207B
:102EC000086005E0D1F8000240F02000C1F80002DF
:102ED0001A7902EBC2008300301DC058E0B9DEF859
:102EE0000010481E8041DEF83410C0434A1E924153
:102EF000D243DEF81410D20F491E8941C943C90FCD
:102F000042EAD0700843EAD006F11805EC5001B14E
:102F100003242AB10F2403E04FF40470C1F8040322
:102F20002046BDE8F2818041C043C00F704780B5A4
:102F300084B00346012002918DF80000019268469A
:102F400019685A680DE080B584B0024600208DF8FB
:102F5000000002910021906801905161684611685B
:102F60005268904705B000BD78B5044604F58876F0
:102F700085B00D467169D9B93068002836D0316006
:102F8000316800910098D4F83C15A86981422DD190
:102F9000EA68E86930B3D4F8003223F02003C4F8BB
:102FA0000032E869A8612869E8600020E8611AE059
:102FB0000020706170690090022000998DF8040073
:102FC0000021D4F88004C4F880040490D4F83C05AF
:102FD0000390E8680290A961E96101A829686A681C
:102FE000904703E0A8612846FFF7A1FF706B78B116
:102FF00000217163706B00900099A86940B10021B5
:10300000A961E9612846D4F83C15EA68FFF78FFF0B
:10301000306970B100213161306900900120009960
:10302000E060686928B104F23C5128460969FFF75D
:103030008AFFB06C60B10021B164B06C009000995F
:10304000686928B104F23C5128460969FFF77BFF03
:1030500006B070BD0349084886E700000805005027
:1030600000070050A05C00201003420000E400E0D4
:1030700018ED00E000E100E00020004055300200C3
:1030800018B40A6812F1010F0BD0012303FA02F2FF
:10309000DFF8BC341A60DFF8BC340C68032243F854
:1030A00024204A6812F1010F04D0DFF8A84400235D
:1030B00044F822300268886902F2245318604C7D7B
:1030C000087D04439C6448680B6802F20C54A060BD
:1030D0002360087D01281ED1886810F1010F04D0FB
:1030E000DFF87044002344F82030C86810F1010F65
:1030F0000BD0012303FA00F0DFF854341860DFF836
:103100005434CC68032043F8240002F5A162886897
:10311000C9681160906011BC704700002DE9FC4146
:1031200004460F4690462179DFF82C042C2212FB2E
:1031300001F2851805F12906707810B10820BDE864
:10314000F6810FF22C42206852F8211001F067FA44
:1031500000B19FE039462046FFF792FFC5F8048092
:1031600038692860686880B32068397F0022C0F819
:103170001C214901D0F81C2100920022009BC0F8BC
:103180004421D0F844210092009BDFF8D023C0F8FE
:10319000042300030016002803D4DFF8C4231154CD
:1031A00006E0DFF8C02300F00F00104400F8041C14
:1031B00021680903091608D4012201F01F00DFF875
:1031C000A8338240490943F8212021680420C1F82E
:1031D00000050020A861E86130706861012070700E
:1031E0000020BDE8F68181B00022C0F81C21D0F893
:1031F0001C210092009B8A680B6AD25CD1F820C027
:103200000CF1010CC1F820C0C0F81C2501B07047BA
:103210002DE9FC4104462C202579DFF83C3310FBD6
:1032200005F51D446869B8B96A61A960286285F826
:10323000280000262068C0F81C61D0F81C110091FD
:103240000121009A81602946FFF7CDFF686860B9C7
:10325000D4F800806F690FE01CE0D1F81C01002851
:10326000FBD00122CA60002068613046BDE8F681CB
:1032700029464046FFF7B7FF286A2168B842ECD2DA
:10328000D8F81C110029F3D195F828000028F7D0B0
:103290000F26E8E71120BDE8F6810279DFF8B812C1
:1032A0002C2010FB02F288184169A2E081B000686E
:1032B0000021C0F82411D0F8241100910021009AB7
:1032C000C0F80811D0F8081100910121009A01609E
:1032D00001B0704781B08A6952B90021C0F8081165
:1032E000D0F808110091009AD0F8180501B0704785
:1032F0000022C0F80821D0F808210092009B4A6AF9
:10330000D0F81805CB689854486A401C486201B050
:103310007047F8B506462C2034798F4B10FB04F427
:103320001F190023786828B1356805F541704FF4FE
:1033300001744460B86970B1FB6943B1786820B129
:1033400032684FF40171C2F804131120F2BD012359
:103350003961FA6103E0BA61F9607862F86197F85F
:103360002900034304BF3046FFF7A0FF78683168A7
:10337000002838D10022C1F84421D1F8440100903E
:103380000099326802F58471C869441EA441E4437F
:103390000868C96BE40F401E8041C0434D1EAD411B
:1033A000ED43ED0F45EAD0702043EAD055EA040022
:1033B00007D139461046FFF78DFF786AB969884210
:1033C000DFD30020B8610CB10320F2BD0DB10F2096
:1033D000F2BD97F829003168002807BF01224A6032
:1033E00001220A6003E04FF40170C1F804030020D9
:1033F000F2BD481E8041C043C00F704780B584B005
:103400000346012002918DF8000001926846196878
:103410005A680DE080B584B0024600208DF80000A7
:1034200002910021906801905161684611685268CC
:10343000904705B000BDF0B585B00D46044604F5D3
:10344000417704F584763868810523D5F06908B39F
:103450000021F16105F12802F06900904FF401703C
:1034600000997860507808B90121616002208DF8D8
:1034700004000021D4F88004C4F880040490A869F2
:103480000390E8680290A961E96101A829686A6867
:10349000904727E03968480724D5306810B329469B
:1034A0002046FFF717FFA869696A88421AD1E869C0
:1034B00040B1EA68696AA8612869E8600020E861AB
:1034C00068620CE005F12801487808B901216160C3
:1034D0004FF4017078600020EA68A861696A2846A4
:1034E000FFF78CFF7069B0B16869296A814207D221
:1034F00095F8280020B929462046FFF774FE0AE017
:1035000000217161706900900099686918B169695A
:103510002846FFF77FFFF06B98B10021F163F06B55
:103520000090009905F12801487808B10121216037
:10353000A86930B10021A9612846EA68696AFFF7E5
:103540005DFF05B0F0BD0449084874E700000000C5
:103550000805005000070050505C00208000020069
:1035600000E400E018ED00E000E100E00020004091
:103570004735020009B90E207047130004D0A2F1AC
:10358000010C1CEA020F01D0092070470160511E96
:10359000818000218160C16000207047836882883B
:1035A000D0F80CC0ACEB03039A4208D30368D0F800
:1035B0000CC002EA0C029954C168491CEBE70420D4
:1035C00070478268C3689A1A0BD00368D0F808C0A5
:1035D000828802EA0C0C13F80C300B708168491CCD
:1035E00001E00520704781600020704780B500E051
:1035F00080B584B002788DF800204368019382681A
:103600008DF80820C068174A039002EB81026846D3
:1036100091685268904705B000BD2DE9F84F88B019
:103620000378104C04EB83056A600E69AE604D7F31
:10363000E5546D4691E8C05F85E8C05F0493037868
:10364000E15C31B102B1084A6946001DFFF720FB79
:1036500005E002B1054A69460C30FFF75FFD09B08D
:10366000BDE8F08F045E0020ED350200F135020068
:1036700028B100BF3AA1800141F00101084770471D
:1036800010B5040005D04FF47A70FFF7F1FF641E07
:10369000F9D110BD38B5C0B000682D4C2D4D401E7D
:1036A000082852D8DFE800F005145151282F324085
:1036B0004800F9F799FF01466846FCF729F8F9F741
:1036C00095FF6846F8F7D8F802466946002010E0F2
:1036D000FAF7F4F90446FAF7EFF90146621C684676
:1036E000F8F734F9FAF7EEF9FAF7E8F9024669461D
:1036F0000120F9F785FC28E041F29410FFF7B8FFAC
:10370000FCF7C0FB21E0F9F7DBFF1EE043F6982051
:10371000FFF7B6FF0020A07595F80401012818BF37
:103720000420FDF712FC10E04FF47A70FFF7A8FFB9
:10373000206CFAF715FB08E04FF4FA60FFF7A0FFE2
:10374000012085F8040100F0D9FD002041B030BD12
:10375000B8350020F4370020000000000000000011
:103760000338FDD87047000038B5054614001EBF69
:1037700000202060002D01D0286808B90E2032BD3D
:10378000E888420800EB92729208B0EB820001D008
:10379000072032BD084602F0A5F9C0B2142801D1B5
:1037A000052032BD2979884201DB042032BDE98839
:1037B0002A68484310442060002032BD0078FFE7AB
:1037C00000F0010070470000F8B50F4690B00546C4
:1037D000B878164600B901208DF80E00032138880C
:1037E000ADF80C0001A8FBF78FFF787C401E00218C
:1037F00004288DF8041011D8DFE800F00D09070542
:103800000300222008E0122102E0312004E02121FF
:103810008DF8041002E011208DF80400B87C401EE1
:10382000002104288DF8051011D8DFE800F00D09FB
:1038300007050300222008E0122102E0312004E005
:1038400021218DF8051002E011208DF80500F87B8C
:103850009DF80610421E9241D24301F0F701D20FAB
:1038600041EAC2018DF8061001F0EF01387C421EDA
:103870009241D243D20F41EA02118DF8061001F0B5
:10388000FE013A7B501E8041C04341EAD0718DF861
:10389000061001F0F901387D002814BF0220012034
:1038A00041EA40018DF8061009A81C21FBF72CFF06
:1038B000787B10F0300F29D0032102A8FBF724FFFA
:1038C000F87C401E002104288DF8091011D8DFE88B
:1038D00000F00D0907050300222008E0122102E094
:1038E000312004E021218DF8091002E011208DF82B
:1038F00009009DF80A0000F0F90040F002008DF880
:103900000A00112102A88DF808100E90787B8DF81E
:10391000240004A8B97B8DF825101421FBF7F4FED0
:1039200003A8049001A90591B888ADF81C00B868F7
:1039300018B1F988ADF818100890BC69002C71D046
:1039400003216846FBF7E0FE2088ADF82C0000213B
:103950006088ADF82E0060680A90CDF834D0207BE6
:103960008DF80010401E042811D8DFE800F00D0982
:1039700007050300222008E0122102E0312004E0C4
:1039800021218DF8001002E011208DF80000B969A6
:10399000487B401E002204288DF8012011D8DFE862
:1039A00000F00D0907050300222008E0122102E0C3
:1039B000312004E021218DF8011002E011208DF862
:1039C0000100B869817A481E80419DF80210C04309
:1039D000C00F01F0F70141EAC0018DF8021001F0BB
:1039E000EF01B869C27A501E8041C043C00F41EA5E
:1039F00000118DF8021001F0FE01B869027A501E24
:103A00008041C04341EAD0718DF8021001F0F90104
:103A1000BA69907B002814BF0220012041EA4001CE
:103A20008DF80210F86900B10C90334604AA09A978
:103A30002846AADF11B0F0BD10B5DFF8244104F12B
:103A40001C0002F065F8D4E9022300211018594146
:103A5000D4E90423994206D828BF904203D2B0F19A
:103A60007F4061F1FF3110BD7CB504460D463C4EF0
:103A7000694606F17C0002F0A3F868B10470456065
:103A8000694606F17C0002F0C3F818B106F11C008B
:103A900002F042F8002076BD042076BD10B4130079
:103AA00008BF07200AD000684FF0FF34C0E9024485
:103AB000012918BF002142610161002010BC70473C
:103AC0002DE9FC410E46002105468DF80010904678
:103AD000684600F0BBFBD5E902234FF0FF3083427C
:103AE00008BF824208D1FFF7A7FF0027801979415C
:103AF000C5E90201012400E000249DF8000000F067
:103B0000C1FB14B90020BDE8F6812869C5F818800A
:103B100000B12E6129460020FFF7A6FFBDE8F6811F
:103B200038B5002105468DF80010684600F08EFB80
:103B3000D5E902234FF0FF30834207BF82420024C1
:103B4000C5E9020001249DF8000000F09BFB0CB9C0
:103B5000002032BD29460120FFF786FF32BD00005C
:103B6000B82A0020002202F0A1B878B405460C461D
:103B70002978012902BF68780028072045D01088DD
:103B8000861CB3422ED3012904D169784118891CBF
:103B90008B4227D31B1A9B1E9BB2ADF8003069469F
:103BA00010882044801C7DDF78BB2878022804D050
:103BB0006978BDF80060B14205D3BDF800108B42B2
:103BC000A8BF09210ADA0821012805D168788342B3
:103BD000A8BFADF8000001DAADF80030BDF8000074
:103BE000FF2802D372BC0C2070471388401CE0549D
:103BF0001088401C108080B221541188491C11800B
:103C0000BDF8000041181180002072BC70472DE9FA
:103C1000FC470A9FDDF82C803D881C4600230646A1
:103C20008A46964699461DE039889DF8002052182C
:103C30001018804538DB43B9491C3980012389B20B
:103C400004F801A03888401C388069463A8822442C
:103C500001A864DFE8B939889DF8000008183880A9
:103C600009F101093088814515DA706850F829009A
:103C700001900022694601A864DF50B99DF8000058
:103C80007045EDD1002B14BF00200220CCE7605519
:103C90000020BDE8F687002BFAD03888401B401E74
:103CA00081B2B1F5807FF2DB0C20BDE8F6872DE90B
:103CB000FC41089F099C01941646054698460097CA
:103CC0000222FFF7A4FF38B901940097434610225F
:103CD00031462846FFF79BFFBDE8F681F0B4148813
:103CE000A51DAB4238BF0C2014D30388062B10DB74
:103CF00040F68146B34203DB4FF6FF77BB4208D163
:103D00004588062D05DBB5424FF6FF7704DBBD4243
:103D100006D00720F0BC7047BB4201D09D42F8D3CB
:103D200005230B55122413885B1C13809BB2CC54C3
:103D300013885B1C13809BB20B4404881C70240AFC
:103D40005C7013889B1C13809BB2194440880870D8
:103D5000000A48701088801C10800020F0BC70475A
:103D60002DE9FC4100F12807884638681646B0B3B3
:103D7000002523E03188401C08F801001621308816
:103D8000401C308080B208F800103088401C308021
:103D900080B2404421880170090A41703088801C3B
:103DA0003080A2884AB1A168C9B180B24044F7F717
:103DB000CDFD3088A188081830806D1CE8B23979B3
:103DC00088420FD23868E9B201EB410200EB82046D
:103DD000A088801CFF28CDD30C20BDE8F6810720E9
:103DE000BDE8F6810020BDE8F6812DE9FC471746C5
:103DF0000546B7F80080002405F12C090E463C80EA
:103E000099F8011071B3B8F1090FC0F0FD80684650
:103E10006DDF002840F0F4803888082131541B21E0
:103E20003888401C3880062280B231540DF10101DF
:103E30003888401C388080B23044F7F787FD3988D5
:103E4000891D39809DF80000400805D189B274545D
:103E50003888401C388005E089B2012272543988C4
:103E6000491C3980A878F8B13988091D8845C0F007
:103E7000CB80684679DF002840F0C2803988032073
:103E8000705419213888401C388080B231543888E9
:103E9000401C388080B23044BDF800100170090A1F
:103EA00041703888801C3880E878A8B13988CB1CEC
:103EB000984540B2C0F0A88002227254012239888D
:103EC000491C398089B272543988491C398089B2B9
:103ED00070543888401C38806868A8B13988005709
:103EE000CB1C9845C0F09080022272540A22398877
:103EF000491C398089B272543988491C398089B289
:103F000070543888401C3880288958B1CDF8048016
:103F1000009733460622022105F10800FFF7C7FE8D
:103F200004006ED1288A58B1CDF80480009733463A
:103F30000722032105F11000FFF7B9FE040060D14C
:103F4000288B58B1CDF804800097334615221421F0
:103F500005F11800FFF7ABFE040052D1286A30B11A
:103F600043463A463146FFF7B9FE040049D1D5F839
:103F700024A0BAF1000F30D0BAF804003988801CB0
:103F800043189B1C98453FD3FF283DD2401C7054DA
:103F9000FF213888401C388080B231543888401C5A
:103FA000388080B23044BAF800100170090A4170BC
:103FB0003888801C3880BAF804206AB1DAF8081012
:103FC00009B907241DE080B23044F7F7BFFC3988F7
:103FD000BAF8040041183980002499F8000038B17B
:103FE00043463A4631462846FFF7BAFE040008D158
:103FF000287830B143463A4631462846FFF7B5FDAA
:1040000004462046BDE8F6870C24FAE738B40028B9
:1040100018BF002A22D00024651C8D4210DA1588B2
:10402000AC4203DB05196D789D4209D02546045D3D
:104030002C19641CA4B2EFE7138080B232BC704725
:104040008C420BDA005DA31C00281EBF401E84B208
:10405000002C03D014FA83F4A142EDDA32BC002024
:1040600070471CB504460020ADF8000013466A46B0
:104070002046FFF7CBFF10B1BDF80000204416BD6D
:104080001CB52D480168002934D52A4C2068A16848
:10409000884204D32949087808B9FBF7ADFDFBF73E
:1040A00030F8012826D020686168884208D30120B2
:1040B000FAF7B8FAF0B9606800F6B830606019E055
:1040C000A168884209D30120FBF7DDFD90B9A06803
:1040D00000F5EA403030A0600CE0194C206800F098
:1040E00054F91849086028B1FAF723FC10B9206880
:1040F00000F055F91448154A01681368994205D033
:10410000FCF706F9BDE81640FFF7C4BA1048D0F82E
:10411000001411F1010F03D0BDE81340FEF748BBB6
:10412000FBF73BFB012803D1BDE8134001F0F0BDD4
:1041300013BD0000B8350020A02F0020F85B002040
:10414000203600205C5E0020AC5A0020B05A0020CF
:10415000882B002010B52149214C0A6800E00C345E
:10416000A06840B120688242F9D3A06880472168E6
:10417000606841182160002010BD2DE9F041194D03
:104180002888D0B100242F1DA046144E28888045D1
:1041900010DA386808B9641C08E03168814205D338
:1041A000B868804700285CBF002038600C3708F1F1
:1041B0000108EBE70CB9002028800020BDE8F08161
:1041C00010B5064C074B226889180C22504318443E
:1041D000416005211980002010BD0000B835002085
:1041E00058360020AC36002005E00A684B689A4239
:1041F00009D1083141600268416853689942F4D19D
:10420000002181607047826070470160096804E0A6
:104210000A684B689A4207D10831416002684168D8
:1042200053689942F4D1002282607047816859B185
:1042300003689A685118426881605368994203D1B3
:1042400002F108014160CFE77047FEE730B4EFF3B9
:10425000108272B6144B996871B901249C6013499D
:10426000134C25680D401D602160616859604FF056
:10427000FF316160002100E00121017002B962B6E6
:1042800030BC7047084A916861B158B9EFF31080AB
:1042900072B6084913680B6053684B600021916047
:1042A00000B962B670470000EC5D0020FC06FFBD5F
:1042B00080E100E000E100E080B5012289B2F9F779
:1042C00006FC17490A68002804D4521CB2F57A7F0C
:1042D00028BF00220A6002BD00B5C1B04FF4807350
:1042E000009301AB01F016FD01460129B2BF4FF06A
:1042F000FF3001A8FFF7E0FF41B000BD0022002120
:104300000120E9E7014600220020E5E7002205211F
:104310000520E1E70348826C0021F9E70000000076
:104320003C5E0020B8350020F8B505460E46AF00CB
:1043300006FB057710373846F5F7F4FD040001D188
:104340000020F2BD3946FFF70DFC00202560A0607B
:10435000E060666004F1100000EB8500002104F1CC
:10436000100203E042F82100491C3044A942F9D36D
:104370002046F2BD81680EE081680268491C9142C6
:1043800028BF0021816000207047C1688268914287
:1043900001D10020704700EB810000697047C168BF
:1043A0000268491C914228BF0021C160002070476B
:1043B0001CB5049C0094001D00F095FB16BD7FB554
:1043C00075208DF8080001203F4D404C2978019060
:1043D00003AE0096012302AA2046FEF79FF8A8B973
:1043E0009DF80C00672818BF08200FD11F208DF8FA
:1043F000080002AE0F2100F012F838B9202000F0BA
:104400000BF818B9212000F007F818B1FBF7AEFF40
:104410004FF0FF3004B070BD8DF808004621717078
:10442000012000900223297802AA2046C0E778B52F
:1044300085B004460B208DF804000120224E234D48
:1044400031780090012301AA2846FFF7B1FF30B967
:1044500031780C2302AA281D00F05EFB38B1718868
:10446000491C7180FBF782FF4FF0FF3028E002A863
:104470009DF80810427842EA0122228081789DF856
:104480000B2042EA01225242628001799DF80D2000
:1044900042EA01225242A28081799DF80F2042EA2D
:1044A0000122E280017A9DF8112042EA0122524263
:1044B0002281817AC07A40EA012040426081002056
:1044C00006B070BD00000000DC370020343600204C
:1044D00028B100BF2EA1800141F0010108477047BB
:1044E000F8B50446FBF7E8FC0546FBF7E9FC244F6A
:1044F00006463868B0F5967F41D3B97D01293ED094
:104500000120B8750220FCF720FD387EB0B94FF4C9
:10451000FA710320FFF754FEFBF7AFFCFBF7B2FC88
:1045200040F2A460FFF7D4FFFBF7AEFC4FF44870F5
:10453000FFF7CEFFFBF7ADFC052000E00720FBF7FF
:10454000DBFE2046F9F70CFC012D204607D100F5D3
:1045500098508830012E07D100F5FA6004E0012E52
:1045600004BF00F5B8507030FAF768F83C64204694
:1045700001F01FFD2046BDE8F240FFF7C3BEF1BDCC
:10458000B83500200000000000000000000000001E
:104590000338FDD87047000030B5A3B001F0CAFD64
:1045A000040034D00020009001226946F9F75DFD37
:1045B0000125002810D4009803280DD20546782242
:1045C00005A9F9F793FD002806D40120009005A95C
:1045D000A2682846904705E0002000900021A268CC
:1045E0002846904700900098002810D4656901ABD8
:1045F00002AA03A904A8A847019B029A0399049858
:10460000FDF752FCE068FDF78FFC002001E04FF061
:10461000FF3023B030BDFEE70F480168084738B5CA
:104620000D460E49884214D100248DF8004068469A
:10463000FFF70CFE08490879002811BF01240D601E
:1046400001220A719DF80000FFF71CFE0CB1112039
:1046500032BD002032BD0000345E0020002000404A
:1046600001460320CA0748BF4FF402408A0748BFEB
:1046700048F20120490748BF48F202207047000075
:104680002DE9F84305460E462979DFF87405904672
:10469000C1EB011200EB820707F12D049946607807
:1046A00010B10820BDE8F2830FF27852286852F862
:1046B0002110FFF7B4FF10B11120BDE8F283C7F855
:1046C0000080C7F80490B86020702071E07040F25C
:1046D0000C61707BE0723268DFF8280540F8221028
:1046E000736840F8231029687068326801F5A16387
:1046F0001A605860B068D8613868E8B1307B090347
:1047000009164001002903D4DFF8FC24505406E0C8
:10471000DFF8F82401F00F01114401F8040C2968B6
:104720000903091608D4012201F01F00DFF8E03464
:104730008240490943F82120012060700020BDE833
:10474000F2830279DFF8B8140068C2EB021301EBC0
:1047500083010523C0F80035022281F82E2070471E
:1047600001F12C03D1F828C09A68624504D2496A45
:10477000895CC0F81C150FE01A7812B10121C161E3
:1047800006E091F820104A0604D50122C2615A7051
:10479000002070470121416101207047F8B400F505
:1047A00082760022336823B132603268009201229F
:1047B000009B01F12C05EB787BB100243462336A55
:1047C00000930023009CB361B36900930023009C15
:1047D000736073680093009C25E0336AB3BBB469CF
:1047E000002C3CD17368F3B1746073680093009C33
:1047F000336A5BBBAB688C6AA34214D200F5A06439
:10480000A6694C6AE654AB685B1CAB608C6A661E9A
:10481000B34247D191F82060770643D40223C0F811
:10482000003201230362002A4AD000226A70EA782B
:10483000002A42D1AB68896A8B423CD000F5A06067
:104840000021016005210160012035E00023336271
:10485000336A00930123009C4361EB70E3E7B3618B
:10486000B3690093009CAC68641CAC60336A002B95
:10487000ECD18E6AB44205D24B6A1B5D00F5A06490
:10488000E361D0E72B7813B10121C16115E091F804
:1048900020305C0603D50121C16169700DE0012360
:1048A0004361C0E7A342BCD10B6A5C06BBD5B8D557
:1048B0000220687001E00020E870F2BC0020704720
:1048C000F2BC01207047FEB50446DFF84C030090AF
:1048D000002504F582700E46056006F12D0701687B
:1048E0000191019A0562016A0191019A85618169CC
:1048F0000191019A45604068019001200199C4F836
:1049000000527563BD702062387801281CBF0121F8
:10491000A16031462046FFF723FF3068E8B140F23E
:104920008621B160B068C4F8040315E03146204622
:10493000FFF734FF00281EBF0098401E00900CD1E6
:104940000EE003250098012806DA04F2C440002195
:10495000C16303250521C1636DE000990129E5DAF2
:10496000B8780028EED004F2C44108680860002836
:10497000E7D0FFF775FE0546E4E7FEB50446A64816
:104980000090002504F582700E46056006F12D07A3
:1049900001680191019A0562016A0191019A85619C
:1049A00081690191019A45604068019001997563A0
:1049B000BD70B06A012805D196F82010480658BF8E
:1049C000022000D50120C4F80002012020623978BD
:1049D000022918BF20603068E8B140F28621B1603A
:1049E000B068C4F8040315E031462046FFF7D6FE50
:1049F00000281EBF0098401E00900CD10EE0032539
:104A00000098012806DA04F2C4400021C16303259E
:104A10000521C1630FE000990129E5DAB878002883
:104A2000EED004F2C441086808600028E7D0FFF720
:104A300017FE0546E4E7284603B0F0BD2DE9FC412A
:104A40000D4605F12C04617801290DD11178012959
:104A50000FD000F541766F4F7760217961B1A8687A
:104A600030601120BDE8F6810229F2D111780129C8
:104A7000EFD00820BDE8F6819E0806F0010686F01A
:104A8000010626712B6205F10C0192E8C05181E804
:104A9000C0515168A962D16869625178C0F888151F
:104AA000117801290AD0002906BF5B0903F0010330
:104AB000012323702946FFF706FF02E02946FFF78E
:104AC0005CFF296809B900222271BDE8F68130B483
:104AD0001346047900680A464949C4EB041501EB02
:104AE000850130BCAAE7F0B585B06D460A9C00266A
:104AF0000027B446A5E8C010C0C58DF80110039288
:104B00000193002C14BF202200226946FFF7DFFF2B
:104B100005B0F0BD000000002DE9F84143A595E87F
:104B2000C05185B06C4684E8C0518DF801100392E5
:104B3000019300226946FFF7CAFF06B0BDE8F08185
:104B4000F8B586B005460C46FFF728FE00284DD183
:104B500004F12C01C878F0B9207B022811BF03288A
:104B6000626AA3699A4216D1E269626200236269AD
:104B7000A262226A4B70520902F001020A700328F5
:104B80002146284603D1FFF79EFE07B0F0BDFFF790
:104B9000F4FE07B0F0BD04F10C0292E8C85001A881
:104BA00080E8C850C87898B1D5F8C404C5F8C404E2
:104BB000820748BF01200BD4420748BF022007D418
:104BC000C20748BF032003D404228DF8002001E06F
:104BD0008DF8000000220A7194F82000420701D5E8
:104BE000C87818B1616822686846904707B0F0BD80
:104BF00003490A48A4E70A494FF04020A0E7000013
:104C0000F45900200007005000E400E018ED00E037
:104C100000E100E086420400A08601000030004070
:104C2000305A0020F14B0200F74B02000100000057
:104C30000000000000000000000000000000000074
:104C400010B584B00A4601788DF8001003798DF80C
:104C5000043041793C4B8DF8051003EB82048168E8
:104C60008DF80610C1688DF807100169029140693E
:104C70000390A16853F822206846904704B010BD05
:104C80002DE9F84F80460E4698F800B02E4892461F
:104C900000EB8B0140F82BA08B60707B00284CD080
:104CA0002A4832682A4C40F20C6140F82210012751
:104CB000736840F823100025316807FA01F121607C
:104CC000716807FA01F1216040F20D61326840F825
:104CD0002210736840F8231021A040F001094FF41E
:104CE0008070C847A0687168C840C0071AD430688F
:104CF00007FA00F060606D1C4FF48070C8473068A0
:104D000007FA00F020604FF48070C847082DE9DDF5
:104D100009E05B46314608F1040001B0BDE8F04F00
:104D2000FFF7AEBC4DB1706807FA00F060604FF459
:104D30008070C847706887402760BAF1000F14BFC1
:104D4000044A0022E5E70000D05D00200007005083
:104D500008050050414C0200000000000000000067
:104D60000338FDD87047000078B404796C4B04EB2D
:104D7000440503EB8504237A13B172BC0820704705
:104D8000226000264A68626000220AE04FF4A073A5
:104D9000D5B203EB850503685E51521C5B59009345
:104DA000009D4579D3B2AB42F0D30268CB781203B1
:104DB00012165B01002A02D45A4DAB5405E05A4D3D
:104DC00002F00F022A4402F8043C03681B031B167E
:104DD00007D4012503F01F02544E95405B0946F8A5
:104DE000235000684A78D0F804359B0802F003028B
:104DF00042EA8302C0F804258A78D0F808359B0877
:104E000002F0030242EA8302C0F808250978D0F8CC
:104E10001025120901F00F0141EA0211C0F8101526
:104E200001202072002072BC7047026801211160CD
:104E30000223FFE700793A4900EB400201EB8201CF
:104E40000B72704700680121016070470068012102
:104E50004160704700680121C160704778B4006804
:104E60004FF480348C4000F5417553B14FF4A0737A
:104E700003EB81030026C650C3580093009E2C60AC
:104E800000E06C6000EB8100C0F8402571BC704709
:104E9000FCB41C460568069BD5F8006240F2011779
:104EA0008F40BE43C5F80062D5F800623443C5F8B0
:104EB000004202B0F0BCD1E72DE9FC410546904626
:104EC00000275FEA08000E461BD04FF480344FF4F1
:104ED000A07000EB870211B2685800281EBFD5F8F9
:104EE000043304FA07F0034208D0002068506858E1
:104EF000009010B200997168326890477F1C474556
:104F0000E5DBBDE8F381042205490948D4E7042222
:104F100008490948D0E7042208490948CCE70000BD
:104F20007C5C002000E400E018ED00E000E100E01F
:104F300000800040885C002000900040945C0020CD
:104F400000A00040002818BF002901D10E207047A2
:104F500001601146026813681847F8B50600154647
:104F600018BF002D0F461C4601D10E20F2BD30683F
:104F700008B90820F2BD0CB90920F2BD17F0030FE3
:104F800004D12246304600F089F808B91020F2BD5D
:104F9000234634682A46A56839463046A847F2BDFC
:104FA000F8B50400154618BF002D0F461E4601D166
:104FB0000E20F2BD206808B90820F2BD36B1606845
:104FC0004068B6FBF0F100FB116008B10920F2BDAA
:104FD00017F0030F08BF15F0030005D1324639461C
:104FE000204600F05BF808B91020F2BD069800904A
:104FF0002A4620462468E56833463946A847F2BD6C
:10500000F8B505000E4614461F4601D10E20F2BD2C
:10501000286808B90820F2BD0CB90920F2BD6868FB
:105020000268511E0E4205D162433146284600F007
:1050300035F808B91020F2BD22462C6828462569AB
:105040003B463146A847F2BD38B500281CBF016871
:10505000002915D10D490E480E4B091AA1FB033248
:10506000140909D00C4D296819B1C9692846884727
:1050700020B91435641EF6D1002032BD012032BDA6
:10508000C969BDE83440084700000000F43700203B
:10509000E0370020CDCCCCCCE0370020C36899426B
:1050A00007D300695118491E88428041C043C00F90
:1050B000704700207047FEE710B543689C184460B5
:1050C00041B103E013F8010B01F8010B1046421E39
:1050D0000028F7D1012010BD38B584B0044615462C
:1050E00069B920681D4A904209D000E0103D102D9A
:1050F00015D9102200F0C3F80028F7D10DE0A06800
:10510000A84238BF002008D323682A462046984783
:1051100018B1A068451BA560012005B030BD2A4626
:1051200000F0ADF8F9E710B50446A06840B1236877
:1051300001222046984718B1A068401EA0600120B7
:1051400010BDF8B5054B0093019102920023039323
:1051500069461022F6F70AFC05B000BDB9500200FE
:10516000F8B50C4605466946FFF7DDFFE0B19DF84E
:105170000000010603D4064626600120F2BD072781
:1051800000F07F0669462846FFF7CDFF60B19DF825
:10519000000000F07F00B84006439DF80000FF1DAE
:1051A0000106E9D5202FEDD30020F2BD2DE9FC4109
:1051B0000E46002700240025804669464046FFF73A
:1051C000B2FF80B19DF8000000F07F0000213A4658
:1051D00000F0FCFF04439DF800000D43FF1D010695
:1051E00003D5402FE9D3002002E0C6E900450120A5
:1051F000BDE8F681F8B507461C460D460020164668
:1052000020702870306069463846FFF7A9FF28B93A
:10521000B86808B9012121700020F2BD009810B9CA
:1052200001212170F2BDC00830600120009901F019
:1052300007012970F2BD1CB5044631B101290ED019
:1052400002290ED0052913D017E0012200F017F82B
:10525000A0B19DF800000106F7D4012016BD082278
:1052600007E000F041FB48B1009A0021204601E030
:1052700004220021FFF730FF16BD002016BD69464D
:10528000204629E738B50D46044600F02DFB80B1D5
:10529000284621461022F6F769FBA8680099884243
:1052A00001D2002032BDA9600098A168091AA1604E
:1052B000012032BD2DE9FF410446164608467168BB
:1052C0000FF2AC658A7802F00F0355F8238012F0D4
:1052D000300709D0102F04D0202F07D0302F36D020
:1052E0004AE0726901201070326942E0022822D13E
:1052F000042B20DC756969462046FFF7C3FF0127B0
:1053000018B93AE02888401C2880029868B1716872
:1053100028884A89904208D20B893269584302444E
:105320006846C0470028EDD10027019860600298C8
:1053300010BB384621E0736932691F880E8948899D
:105340007E438742324417D27F1C1F8011E073696D
:105350000888188002F00F02072A08D109893069ED
:10536000FEF700FC70683169C06800F0FEF8326931
:1053700071682046C04700E0002004B0BDE8F0811D
:105380002DE9F841144687B025690646286818B902
:105390003046FFF750FF3DE0022911D16946304603
:1053A000FFF770FFD8B161682B682A1D68469847DF
:1053B000A8B102980028F6D101987060012029E078
:1053C000E84671B1012903D0052908D1042700E07E
:1053D00008273A4669463046FFF77EFE80B900202E
:1053E00018E000277F1C0B2FF9D2012241463046DE
:1053F000FFF772FE0028F2D018F8010B0106F1D475
:105400003A46694603A8FFF79CFE61682B682A1D8F
:1054100003A8984708B0BDE8F08110B553689C78A0
:1054200014F0C00402D0402C03D005E0BDE81040C9
:1054300040E7BDE81040A3E7002010BD70B50D4661
:105440000446286886686A683146204600F0CFFE28
:105450006868206105F10C006061B07800F0C00060
:10546000802804BF291D216170BD2DE9F84386B055
:1054700006461869B76804688946904600E0A46843
:10548000ECB1B06887421AD1206805682DB1434657
:105490004A4621463046A8470EE0806801884945C3
:1054A000EDD121466846FFF7C9FF012020736A4607
:1054B00041463046FFF7B1FF0028E0D100E001206F
:1054C00007B0BDE8F08310B586B04268937803F06A
:1054D0000F0108290ED100690468002C43D0002177
:1054E000217368462146FFF7A9FF6846FFF7EBFFE7
:1054F000A468F2E713F0C00127D103F03004102CA8
:105500000DD1436919709178D368006901F00F01DA
:10551000072910D10146184600F027F823E003F0D0
:10552000300120291CBF03F03003302BEBD1406940
:105530000021018017E0118923B10A461946F6F7C8
:1055400005FA10E0FEF70EFB0DE080290BD1016992
:1055500000220A6003F03001202919BF03F0300354
:10556000302B4069028006B010BD80B50A4686B077
:105570000146684600F03BFE38B16846FFF7A3FFDE
:10558000684600F046FE0028F7D107B000BD2DE9BF
:10559000F8438AB002AB0024C3E90044054604A8DE
:1055A00000F025FE00274FF001094FF0FF360DF106
:1055B0000808A868002838D00DF1010301AA69463F
:1055C0002846FFF717FE60B3019904A800F061FEBA
:1055D000002840D10198B8421DD3059C05988178D8
:1055E00001F00F01082934D004A800F012FE05983C
:1055F000A042F3D137460198B8420CD3AC689DF86D
:105600000020014604AB2846FFF72FFF002856D0A4
:10561000A8688442CDD19DF800102846FFF70BFE04
:1056200039E09DF80100002849D005988578069C4E
:1056300004A800F0EEFD0028F7D115F0300F03D1DB
:105640000599088800B1641C002C3AD0002061093B
:105650002AE00788CFE70598817811F0300F0CD148
:105660000698402809D2410958F8212000F01F006F
:1056700009FA00F0104348F82100EC682CB19DF8BD
:105680000020019904AB2846A0479DF8001004AA09
:105690002846FFF7C2FE00288BD110E058F82020E2
:1056A00012F1010F0BD1401C8842F7D304F01F0404
:1056B00058F82100C4F12004E640B04201D0002097
:1056C00000E001200BB0BDE8F08370B504460D4644
:1056D000164631462846FFF748FF324629462046FF
:1056E000BDE8704053E73EB50C466946FFF75EFDE6
:1056F00068B1DDE90023DDE900015B084FEA320211
:10570000C50744BFD243DB43C4E9002301203EBDAB
:105710001CB50C4604226946FFF7DEFC78B19DF803
:1057200000009DF8011040EA01209DF8021040EAB7
:1057300001409DF8031040EA01602060012016BD81
:105740001CB50C4608226946FFF7C6FCF0B19DF86F
:1057500000209DF801009DF8043042EA00229DF8E7
:10576000020042EA00429DF8030042EA00629DF80E
:10577000050043EA00239DF8060043EA00439DF834
:10578000070043EA0063C4E90023012016BD3EB5CB
:1057900000F051F818B32A89DDE90001082A08D180
:1057A000C4E90001D4E900238B4215D1824215D00F
:1057B00012E0C117042A03D120600246D317F3E791
:1057C000022A03D12080B4F90020F7E7012A03D18F
:1057D000207094F90020F1E700203EBD01203EBD7D
:1057E0003EB500F028F828B3288908280AD1DDE959
:1057F0000001C4E90001DDE90023994217D190427C
:1058000017D014E0042804D1DDE900012060002154
:10581000F1E7022804D1DDE9000120802088F6E7C5
:10582000012804D1DDE9000120702078EFE7002095
:105830003EBD01203EBD0D4614466946B6E43EB568
:105840000D4614466946FFF74EFF38B328890828ED
:105850000AD1DDE90001C4E90001DDE90023994234
:1058600019D1904219D016E0042804D1DDE90001D5
:105870002060C117F1E7022805D1DDE90001208091
:10588000B4F90000F5E7012805D1DDE90001207039
:1058900094F90000EDE700203EBD01203EBD114619
:1058A00036E711464CE77CB50E460446154600F037
:1058B0001BF8C0B10098B0F5803F0BD20099801C56
:1058C000884207D3B17801F0C001802902D0318924
:1058D000814201D2002076BD00982880A91C009A40
:1058E0002046FFF7F9FB76BD694639E47CB50E46E4
:1058F00005461446FFF7F8FFB0B100980099401C28
:10590000884207D3B17801F0C001802902D03189E3
:10591000814201D2002076BD009A21462846FFF739
:10592000DBFB009A0021A15476BDF8B50D4684B08A
:10593000EF6800F017F800281ABFE8680028002078
:105940000ED0A87800F0300020283246394668464C
:1059500002D1FFF7BAFE01E0FFF719FE019961607D
:1059600005B0F0BD0446164669468BE40000000011
:105970008F570200E15702003F5802009F58020073
:10598000A3580200A7580200ED5802002B5902004C
:105990000000000033B58BB00446002000900C9945
:1059A00081B1002529460CA800F09FFC38B1009871
:1059B000694601EB400295800098401C00906D1CE8
:1059C000142DEFD32046694687E082B012B102B0B1
:1059D00000F076BC02B000F07DBC2DE9F04F074628
:1059E00097B03888B7F80480102806D0112845D021
:1059F000192865D01A2846D06CE0DFF80461B06839
:105A0000C04300906846716800F086FC00990CA8BD
:105A1000FFF7C0FF01A80CA92C22F5F7A7FF0198FA
:105A200098B10DF108090546B9F800A006F1040B7C
:105A30001E245146584600F04DFC641E0BF1040B29
:105A4000F7D16D1E09F10209EED1B8F1140F03DB95
:105A50000420FAF7C3FC3DE0414606F1080000F0DF
:105A60002FFC4146301D00F02BFCF87B022831D181
:105A7000414606F10C0000F023FC2BE04146214892
:105A800000F028FC26E03D7A1D4C2D09042DACBF0A
:105A900001220022414604F11800FFF796FF022D73
:105AA000CCBF01220022414604F11400FFF78DFF14
:105AB000022DACBF01220022414604F1100007E094
:105AC000387A38B97A7A1048D20802F00102414691
:105AD000FFF77BFF17B0BDE8F08F2C22F5F746FFEC
:105AE0000DB030BD10B51428044606DA214607482B
:105AF00000F0FBFB08B1204610BD142010BD0000D3
:105B00007859002080590020905900207C590020AD
:105B10000068D0F80405704790F90410080007D415
:105B2000012201F01F00064B8240490943F8212061
:105B3000704702490868896808470000105E002025
:105B400000E200E0000000000000000050B411B9C5
:105B500050BC0E207047144694FBF3F603FB16442A
:105B600014B150BC0920704701608281002141605E
:105B70008160C381002050BC7047000081B050E8B4
:105B8000022FC188B2EB324F4FF0000317BF92B221
:105B900041EA014142EA014104E04268B2EB324F7E
:105BA00008BF012340E80212002AE8D18DF8003036
:105BB0009DF80000002814BF0020112001B070479C
:105BC0003CB450E8015FAAB2C3891A4483899A425F
:105BD00028BFD21A03899A4202BFBFF32F8F002435
:105BE00007E0C2EA050240E80123002BE9D14FF0AB
:105BF000010401958DF80040019A0A609DF800208B
:105C0000002A1DBF006809884018002036BC704774
:105C10000A8849888A4209D150E8011FC1EA014136
:105C200040E80112002AF7D1012070470020704798
:105C30003CB450E8025F1FFAA5F2C3889A4202BF43
:105C4000BFF32F8F00240DE0C3891A4483899A4241
:105C500028BFD21AC5EA024240E80223002BE8D14D
:105C60004FF0010401958DF80040019A0A609DF8FB
:105C70000020002A1DBF006849884018002036BC5B
:105C8000704700000A8849888A4209D150E8021FFB
:105C9000C1EA214140E80212002AF7D101207047F1
:105CA0000020704762F30F2262F31F42401810F089
:105CB000030308D0C91A1FD3DB0748BF00F8012D22
:105CC00028BF20F8022D130030B4144615461039B1
:105CD00028BF20E93C00FAD8490728BF20E90C007A
:105CE00048BF40F8042D890028BF20F8022D48BF86
:105CF00000F8012D30BC7047C91818BF00F8012DFD
:105D0000CB0728BF00F8012D7047FEE700F020BB4D
:105D100000F02BBB2DE9F84F012896B098464E4D68
:105D20004E4F4F4E38D111A8F9F7C4FD0CA8F7F724
:105D30003DFF01220BA90020F8F797F9307E441EA1
:105D4000A4413878E40F20B1FBF7D7FC00F1C80775
:105D500002E0FBF7D2FC0746F9F7A4FC2968414DA5
:105D60000A910CAAF16D099108940692029011AB68
:105D70000B99306E079105930190039706F11B0371
:105D80002968049140463849D1F800203BA100928F
:105D90000222FAF703FB5BE0002818BF02280991F2
:105DA00044D108000CBF4FF0000A4FF0020AFAF786
:105DB00083F88346FAF784F88DF82000387818B114
:105DC000FBF79BFCC83001E0FBF797FC274A2968EA
:105DD0001388274CDFF89C90079106936188B9F8E7
:105DE0000030254F3A885B1A059302232188521A06
:105DF0009DF82010049201EA0B0103910290524693
:105E0000DDF8240029A1019006F11B000090404616
:105E1000FAF7C4FA39882288914218BF2180B9F86C
:105E200000106288914213D0618011E005280DD1E5
:105E3000D5F8000026A10290019206F11B030998F3
:105E4000009002224046FAF7A9FA01E04FF0FF3035
:105E500017B0BDE8F08F00003C5E0020845E00209B
:105E6000B8350020545E0020B02F0020485D00208F
:105E7000485E00205E5D0020DE370020513D313B52
:105E8000323B25643B25733B25733A25732C2573E0
:105E90002C25642C253038582C25732C25732C2563
:105EA000642C25642C25643B25640000513D256449
:105EB0003B323B25643B25733B25642C25642C2514
:105EC000642C25642C25642C25643B25640000008B
:105ED000513D353B323B25643B25733B25642C25E6
:105EE000643B2564000000002DE9F04100F0C6FA93
:105EF000FBF700FC584C617D40F2C67290420DD217
:105F000009B901206075206910B90620FBF71DF85A
:105F1000206906281FD2401C20611CE0A0F2C77037
:105F200039280ED2B9B9206900B12161E068401C5E
:105F30000128E0600FD9012060750520FBF705F806
:105F400009E0012907D1002060750120FAF7FDFF63
:105F500000202061E060414C2068401C96282060B1
:105F600024D3002020600026F9F7A6FF0746F9F7A2
:105F7000A7FF012F05460FF21C1809D13EA0F7F725
:105F80003AFB012D41F2883609D141F6583603E03B
:105F9000012D04D141F270764046F7F72CFB606882
:105FA000864203D03046F8F749FB66600020BDE822
:105FB000F08110B52A49284B486000200860294824
:105FC0001C68C2680169141B8C423CBF8918C160FF
:105FD00010BD10B5224C6068002809DDC0B2FEF784
:105FE00091F92068401C20600428C4BF0020606034
:105FF000002010BD80B51C49088808B1FEF7BDF827
:106000001A490878012802D01949086880470020F9
:1060100002BD80B51549087810B9164A116888473D
:10602000002002BD80B50020FEF76CF9002002BD03
:1060300010B50E48084C0078E17D81420AD0E07529
:106040000020FEF75FF9E17D012903D1F9F710FF88
:10605000F9F707FF002010BDB8350020245E0020AE
:106060002C5E002058360020AC360020845E0020D4
:10607000A0350020A43500204163747561746F72EF
:1060800031203A20646973636F6E6E656374656472
:106090002E0D0A004163747561746F7232203A20CC
:1060A000646973636F6E6E65637465642E0D0A00B8
:1060B000BFF35F8FBFF34F8F37480021016041600E
:1060C00081603649C16005210160BFF34F8FBFF386
:1060D0006F8F00207047884202D35118884201D345
:1060E000002070470120704710B50A46011D0C685A
:1060F00001462046FFF7EFFF10B94FF0FF3010BD0B
:10610000A047002010BD2DE9F0410D4604462F6840
:106110009046002600E0761CA64208DA57F82600D2
:1061200042462946FFF7D7FF0028F4D100E0384661
:10613000BDE8F08130B58BB0FFF7BAFF184D286885
:1061400080474FF410314FF44030FFF7CDFF002867
:1061500008D44FF410324FF440310620FFF7D3FF3C
:10616000040001D1002015E0606880470D490866F1
:106170004FEA00020FF244010CA0F7F73CFA2C2280
:1061800029466846F5F7F2FB07480A9068462168F9
:10619000884720460BB030BD94ED00E02500000399
:1061A000F0360020B8350020F7D501004657203AD8
:1061B0002025732C2025730D0A0A000044312D4E32
:1061C00052462D302E332E3000000000D2B2203A3D
:1061D00022BF00FA02F1002070475242D041D2F1B2
:1061E000200291404140D0409040414070470160C2
:1061F0004160C2600021816041688B881A4402615D
:10620000B1F906301A444261088800B10120C0B2D9
:106210007047F8B543681A46118839B110334360A6
:10622000198829B9C2680168FFF7E1FF0020F2BDB3
:10623000917814890D4605F03006302E02BF9F7804
:1062400007F03007302F06D1958801696D42294447
:10625000002401610BE001F0F001202902D15189F5
:106260004C4304E005F0C005802D08BF042491785C
:1062700011F0300F02D18168491C816001699A8850
:10628000214411440161B3F9062011444161012008
:10629000F2BD70B504460D46666860680188A94283
:1062A00004D1807800F00F00082807D12046FFF7BE
:1062B000B0FF6068B042F0D1002070BD012070BD19
:1062C0000B46012103F01F025B09914000EB8300A4
:1062D00000F014B80B46012103F01F0291405B0946
:1062E000C94300EB830000F017B84A0950F82200B8
:1062F00001F01F01C84000F00100704710B40246D1
:1063000052E8004F44EA010042E8000393F0000F16
:10631000F6D110BC7047000010B4024652E8004F9E
:1063200004EA010042E8000393F0000FF6D110BC2C
:106330007047000010B40146012451E8000F40EA04
:10634000040341E8003292F0000FF6D110BC704710
:1063500080B51548002141700161BFF35F8F001DBA
:1063600013A1FDF752FF002002BD80B500218DF87A
:1063700000106846FDF76AFFF1EE100A20F09F005A
:10638000E1EE100ABFF35F8F0848402101609DF8DD
:106390000000FDF777FFFAF72DFF08B141DF01BDDF
:1063A00020BF40BF20BF01BD9C5D002084E200E013
:1063B000B8A10200D0A102000400000070B504469C
:1063C000207858BB6068022100F0ADF90022264B0E
:1063D0001D69586958B90021656835F9125023F8CC
:1063E00011504019491C0829F6DB01250CE06168B1
:1063F00031F9126033F9151023F81560401A80192D
:106400006D1C082D28BF0025521C012A58611D61F2
:10641000DEDDBDE87040C008FBF768B970BD000064
:106420007FB500BF1AA100BF1CA52E68009601A869
:1064300091E81C0080E81C0002228DF800206846CC
:106440000A4900F0D7F868B901A900F017F948B96E
:10645000074C0221204600F066F918B90221201DE0
:1064600000F061F904B070BD005D0020BD63020062
:106470001C5E002080B5FFF7D3FF02E080B500F07E
:106480009AF918B1F9F772FF4FF0FF3002BD000022
:1064900000000000020000010000000001000600F2
:1064A00078B5DFF83463DFF8345383B0706805F1F2
:1064B0002D0420B30021716070680090009960780D
:1064C00008B1A178D9B16968019100228DF8002046
:1064D0002989ADF80810E96809B92A740AE02A8BFD
:1064E0006A8369602A810021E96018B9DFF8F00247
:1064F0000121016068462A6890470020A0706178F9
:1065000000291CBF306800282DD00021316031687F
:106510000091009821786A8B91420AD2501A6883C0
:1065200080B22B896C68DFF8BC22181A04EB40009B
:1065300009E08A420ED1E86840B10122A27000222F
:106540006A83DFF8A0221060516003E00120A07090
:106550000020688300207060DFF88422706800905B
:10656000012000995060306960B1002131613069CB
:10657000009000200099287402208DF800006846E1
:1065800029688847706918B96C694FF000462DE09A
:10659000002070617069009000200099287404B098
:1065A00070BDB4FA84F026FA00F18C43810001F545
:1065B0008C7109B2DFF828225058B8B1002353502B
:1065C000A1F58C73525800920906890E01F0010161
:1065D00081F0010100988DF805100122DB088DF88B
:1065E00000208DF80430684629688847002CD8D1EF
:1065F00004B070BD38B4DFF8E44104F12C031A781C
:1066000012B132BC0820704721600278DFF8D8113F
:106610000A6042784A606FF00042C17899700121A7
:1066200019700021217459706161D9700024DFF85C
:10663000BC114A60DFF8A021546054680094002423
:10664000009D1460146800940024009D54615269F8
:106650000092009C8078DFF8982140011070DFF8EC
:1066600094018022026002200860987808B101221B
:106670000A600121DFF88001016051E038B4DFF8E1
:106680005C3103F11004227812B132BC1120704742
:106690000A79002A18BF012A03D1DFF85C510022D1
:1066A0002A6003EB40031A7F12B9657F6D1C657782
:1066B0000001CA791A770A7A5A774C780B78DFF892
:1066C0003C21240103F0030304F0300423438C78BD
:1066D000240204F4E0642343CC78240304F48054BB
:1066E00023430C79240404F4E02423434C79240547
:1066F00004F4801423438C79240604F0807402F19E
:10670000080523432B50151DCB790C7A2C501350C0
:106710000879002818BF012802D1374901200860F4
:10672000002032BC704738B40246304C2B4B12204C
:106730006060187C022808BF122105D01D7C012D45
:106740001BD1D86820B102212160112032BC7047D2
:1067500003F12D00DA60198343785BB91E4B18688A
:106760000028FBD000251D601B68009300981D4881
:1067700002604160022121601CE00220206003F1E0
:106780002D05012018745A6019810020D860154C1D
:10679000687820B128785983226060600AE022601E
:1067A000616000210C480E4A0160006800900120E1
:1067B00000991060B4E712490A780020012A01D03C
:1067C00008207047897F064A11B101231360704782
:1067D000012353607047000000710040C85B002037
:1067E000007000402C760040F075004004730040BB
:1067F00007E400E000E100E0007500401075004093
:10680000D85B002000000000000000000000000035
:1068100028B10FF29C41800141F001010847704707
:1068200010B5040005D04FF47A70FFF7F1FF641E35
:10683000F9D110BD80B5F8F7A4FFDFF85403006864
:10684000C10548BF042002D4410505D50120BDE89B
:106850000240FAF7B2BA01BD010448BF0220F6D4E3
:10686000810448BF0320F2D40028F4D50520EEE7C8
:1068700038B584B0002505240DF10200FDF7D7FDE1
:10688000BDF90400B0F5805FA8BF6D1C00F08BF966
:10689000641EF1D1042D04DBBD48016841F00041C4
:1068A0000160002005B030BD2DE9FE4300F004FA80
:1068B000002844BF0FF20430F6F79DFEF9F7A0FA66
:1068C0000028B34C03D5206840F001002060F6F7A3
:1068D00063FE002803D5206840F004002060FFF725
:1068E000C9FD002803D5206840F00800206014206E
:1068F000FFF78EFFF7F73CFD002803D5206840F432
:1069000080402060F8F72AFF002803D5206840F077
:1069100020002060F7F73AFD05460020F8F722FF37
:1069200000F041F9FFF7AAFD6420C04601469948EE
:106930000FF20439D0F80020A7A00FF2E828964FF4
:10694000F6F759FEB3A0F6F756FE207887A6C107E2
:106950004CBF4A46324600BFB5A100F021F920786D
:1069600041074CBF4A463246B5A100F019F92078DC
:1069700081064CBF4A463246B3A100F011F92068A7
:1069800041044CBF4A463246B1A100F009F9FFF775
:10699000BDF9FBF7ADFD002803D5206840F01000DD
:1069A00012E000F000F9FDF70AFD002803D5206889
:1069B00040F480602060F8F7B0FC002806DC00207E
:1069C000B876206840F48070206001E00121B9763B
:1069D0002078C1064CBF4A46324665A100F0E0F877
:1069E000206841054CBF4A46324662A100F0D8F803
:1069F0002068C1054CBF4A4632465FA100F0D0F87E
:106A000000F098F9002804D5206840F0400020608C
:106A100014E0F8F7D9FA00280CD46846F8F7FAFA27
:106A2000002807D49DF80000002804BF9DF801004D
:106A3000002803D1216841F400512160F9F73CFAA4
:106A400010B9F9F73DFA18B1206840F40040206011
:106A5000FBF74DFE002803D5206840F4007020604D
:106A600007F11B00F7F7D4FAF7F703F8002803D56E
:106A7000206840F480302060217848064CBF4A46A8
:106A800032463EA100F08CF8206881044CBF4A4693
:106A9000324600BF70A100F083F8207801074CBF98
:106AA0004A46324636A100F07BF82068C10348BF51
:106AB0004E46324633A100F073F800F074F8FFF749
:106AC000DDFC6846F7F772F84FEA0D0207F11B018B
:106AD00063A0F6F790FDF8F7E5FD014665A0F6F72F
:106AE0008AFD206808B1FFF7A5FEFBF78BFA26A008
:106AF000F6F781FD294E3078002814BF00200120D0
:106B0000F7F747FDF7F78FFC20A0F6F774FDF9F7CC
:106B10005BF8F9F7E9FBFBF726FFFFF7A9FE00E0BA
:106B200030BFF7F733FC401BC828F9D3F8F729FE2C
:106B3000F9F79EF9F9F795F93078012808BF00F0C8
:106B40003DF90320FAF701FA216849B1FFF772FE17
:106B5000206828B14BA0F6F74EFD4FF0FF3003E060
:106B60004DA0F6F748FD0020BDE8FE836F6B0000E6
:106B700074776900696D75007274630073706900E1
:106B800061646300626C65000D0A00000D0A0A0072
:106B9000545E0020B02F0020B8350020845E002015
:106BA0004046F6F728BD14203AE680B50120F8F7F4
:106BB000D9FD0020F9F716F8002002BD6770696F53
:106BC00074652C206E6F7420696E697469616C69DC
:106BD0007A65642E0D0A00000D0A537461727421E7
:106BE00020434C4B3D36344D487A2C20494D553D81
:106BF00034472C3530304450532C2054494D4552A5
:106C00003D2564487A2C205645523D25730D0A0ACD
:106C1000000000003C5253542D44312E303E0D0AEA
:106C20000A000000253873203A2025730D0A000061
:106C30006770696F000000006661756C7400000089
:106C4000756172740000000074696D657200000067
:106C50007469636B0000000077323571000000003A
:106C60000D0A4944203A20257320282573290D0A4E
:106C70000A00000054494D45203A2025730D0A0AA8
:106C80000000000053797374656D204661696C756E
:106C90007265210D0A0A000053797374656D2052E4
:106CA00065616479210D0A0A0000000000000000FF
:106CB0000338FDD87047000080B51A4900200860ED
:106CC00000F05CF968B900BF19A0016800910322C7
:106CD0008DF8012069460FF235020B2000F09CF977
:106CE00020B1F9F743FB4FF0FF3002BD01210B202B
:106CF00000F0ECF90C480D490068C00A00F00100F2
:106D000080F001000870002002BD00000B2808D1AF
:106D1000054806490068C00A00F0010080F0010043
:106D2000087070472C07005010050050845E00204A
:106D3000030002001FB5684612A11022F4F716FEE8
:106D400011208DF802000E210D208DF801108DF814
:106D500000004FF08051002002918DF80C001224A9
:106D60008DF80340002300226946054800F0E0FA50
:106D700018B1F9F7FBFA4FF0FF3004B010BD000076
:106D8000A8350020FFFFFFFF06FF000000000040C5
:106D900000000000000000000000000000000000F3
:106DA00010B5040008D000BF4DA14FF47A4041F067
:106DB00001018847641EF6D110BD00002DE9F0479F
:106DC0003FA40FF2DC0A2A4E2A4FDFF8AC800FF204
:106DD000B0094846F6F70FFC0CE038683168884285
:106DE00003D0F9F795FAFCF755FC00F032F80120D2
:106DF000FFF7D6FF98F804010028EED05046F6F7CA
:106E0000FAFB40F6B830FFF7CBFFF7F7BFFA0546BD
:106E100098F804010128DCD1F7F7B8FA85420AD2C4
:106E20000020FDF76FFA2046F6F7E5FBF7F7AEFA1C
:106E300000F56A45603538683168884203D0F9F753
:106E400067FAFCF727FC00F004F80120FFF7A8FF21
:106E5000DEE710B5F7F79AFA084C2168814206D2AE
:106E6000FFF70CFBF7F792FA00F6B830206010BD80
:106E7000B05A0020AC5A0020F4370020405E0020B9
:106E8000436865636B696E6720424C4520636F6E93
:106E90006E65637469766974792E2E2E0D0A000072
:106EA000476F696E6720746F2073656E6420424C73
:106EB00045206D657373616765732E2E2E0D0A0074
:106EC000537461747573206D6573736167652C20ED
:106ED00073656E742E0D0A000000000000000000B3
:106EE0000338FDD87047000038B40FF20C44256811
:106EF00000950B1898420DD26C4604EB800050F8B8
:106F0000043BD3F820451460491E52F8044BC3F8E3
:106F10002045F4D131BC7047DFF8B42302EBD00137
:106F2000012391F8542000F0070003FA00F0104309
:106F3000FFE781F854007047F0B4140007BF08243D
:106F40000C2500240825DFF888634FF0FF3306EB9B
:106F5000840700E0641CAC420DD257F804CB9C457A
:106F6000F8D1331883F8304046F8241012B931199B
:106F700081F84800234658B2F0BC7047B8B4DFF837
:106F8000502302F15001087A10B1B2BC08207047BA
:106F9000002302F130044FF0FF35DFB24FF0000C58
:106FA000780908BFAC4607F01F072CFA07F0C007A6
:106FB00048BF25705B1C641CD8B22028EDDB15602F
:106FC00055609560D560156155619561D561156213
:106FD00055629562D56202F15400002202600D7084
:106FE0004D708D70CD70C020DFF8E822DFF8E832F8
:106FF000107040221A60DFF8E4020023036000688A
:10700000DFF8DC3200904FF00040009A1860012356
:107010000B720020B2BC70472DE9FC410546DFF839
:10702000B0627019002490F930000F460028114614
:107030000ED5BA78520802F001022846FFF77CFF0D
:10704000804618F1010F05D104242046BDE8F681E1
:107050000824FAE7B878410715D4C0070AD54FF0DD
:10706000A04000EB8500D0F8001721F00201C0F825
:10707000001705E07878DFF87012800041F82500ED
:107080002846FFF749FFB8783978820713D5954A23
:10709000964852F82830034042F828302D0209045F
:1070A00052F8280005F4F85501F440310D4305432A
:1070B00042F82850C9E706EB080090F8480040EA7B
:1070C000811006EB080181F84800BEE738B4804B18
:1070D0001C1894F93020082A23DA20D2814850F86D
:1070E000225045F0010540F82250900000F58070D4
:1070F00000B200F1804000F5C04000250560002985
:1071000000680090009D1EBF94F9301053F82100D4
:10711000002804D0012101FA02F271490A6031BC51
:107120007047991891F948100906890F032905D16C
:107130006F490968C140CA0702D503E0012901D19E
:10714000022100E003214FF0A04202EB8000D0F8C2
:10715000002722F44032C0F80027D0F8002742EA86
:107160000142C0F8002731BC704700002DE9F84FFC
:107170004FEA000760A55F4EDFF86CA1DFF8509181
:107180004FF0010809F1500B04249BF9001011F194
:10719000010F3BD0C8B220F0C000C30800F00702C6
:1071A000FB5C08FA02F21A4230D04FF0A04C0CEB14
:1071B000800C5AF82030DCF800E72EF4403E090637
:1071C0001B0CCCF800E7890F03F00303022BDCF85B
:1071D00000E70CBF032202224EEA0242CCF800274D
:1071E00008FA00F2326009EB000292F9302059F8F7
:1071F00022205AB1032908D0022B02D1012905D13E
:1072000003E0032B08BF022900D19047641E0BF155
:10721000010BBAD12A680092D2F820253A60009971
:10722000C1F8202538680028ACD1BDE8F18F2DE9E0
:10723000FC41002500954FF4807101220820284B65
:107240000CB204F1804404F5C0442668012E08D134
:107250001E68164205D00026266015432468019456
:10726000019E5200091D401EEAD11C4801680129F7
:107270000BD1002202606A4600680190002001994B
:107280000121FFF731FE45F00045290618D00126FF
:10729000144FDFF83C8008242E420BD03868396840
:1072A000D8F80020130005D0090C01F00301C0F349
:1072B0000420904776003F1D641E08F10408EBD1BE
:1072C000002D44BF6846FFF751FFBDE8F381000081
:1072D000DC5A002006E400E000E100E07C610040B0
:1072E000046300401065004000070050FFE0FCFF11
:1072F00010050050200500500000005018B585B062
:107300000A4601788DF80010436801938168104B9C
:107310008DF8081003EB8204C168039100698DF8B1
:107320001000E16853F822206846904706B010BD6F
:1073300030B40478064D45F8242005EB8405EB6055
:1073400002B1044A234630BC001DFAF72DBF0000ED
:10735000185D0020FD720200000000000000000027
:1073600028B10FF2DC21800141F00101084770478C
:1073700010B5040005D04FF47A70FFF7F1FF641EDA
:10738000F9D110BD2DE9FF470746002F894603DDDF
:1073900040F2FF18C14505DB0720F8F7E7FF4FF083
:1073A000FF3028E015480FF2E41A078000214180E1
:1073B0008180C18000E07F1C474508BF0127394616
:1073C0005046F6F718F910261025122402E00A207C
:1073D000FFF7CEFF6846F7F7ACFA0028F7D446204F
:1073E000FFF7BEFF641EF5D16D1EEED1761EEBD108
:1073F0004F45E0D1002004B0BDE8F087485D002093
:107400002DE9F14F00288AB004DD40F2FF108142DF
:10741000059105DB0720F8F7A9FF4FF0FF3071E079
:1074200000210A9F049100258A460391029100E001
:107430007F1C0498401C40F2FF1104908F4208BF4B
:1074400001270FF248103946F6F7D5F8A846002470
:107450004FEA083000EB0740002600EB04294FF00C
:107460000E0B0BFB069B0E2206A95846F7F7E1FD13
:107470004620FFF775FF44EA0800304306D1BDF906
:1074800018100FF214105A46F6F7B5F8BDF91800A7
:10749000B84204BFBDF91A00404508D1BDF91C002F
:1074A000A04202BFBDF91E00B0426D1C01D00AF11E
:1074B000010A761C122ED2DB641C102CC8DB08F1EA
:1074C0000108B8F1100FC2DB0FF2E80053462A465C
:1074D0003946F6F790F803982D1802980395504412
:1074E0000290002505988742AA46A1D103990298E7
:1074F000059B0A9A0091019004990FF2E000F6F7BB
:107500007AF800200BB0BDE8F08F38B5012814469A
:1075100002D14FF0FF3032BD65680FF2EC0100F090
:1075200030F840B9E068F6F7F3FE00F026F8294697
:10753000BDE8344026E70FF2DC0100F022F840B944
:10754000E068F6F7E5FE00F018F82946BDE834409B
:1075500056E70FF2CC0100F014F818B9BDE831403D
:10756000F6F748BB0FF2C40100F00BF818B900F0B1
:1075700005F8F9F722FC002032BD0546A068F6F7B1
:10758000C7BE2846F6F770BF00000000626C6F634C
:107590006B2025640D0A0000666C6173685F626C85
:1075A0006F636B203A2025642C20253038580D0A53
:1075B00000000000626C6F636B2025303264203A5B
:1075C0002076616C69642025642C20696E76616C7C
:1075D00069642025640D0A0A000000002564206209
:1075E0006C6F636B732825642C202564292C20760E
:1075F000616C69642025642C20696E76616C696415
:107600002025640D0A00000073646174615F777265
:107610006974650073646174615F636865636B00BE
:10762000626C655F74657374000000006661756C60
:10763000745F6C6564000000000000000000000042
:107640000338FDD870470000024613689868002888
:1076500000D1704770B586B06B4600240025002627
:1076600070C370C3019190680590107910B1012822
:107670000AD011E001208DF8000011690291D06854
:1076800003905069049007E002218DF80010D06843
:107690000003029051690491684611688A68904716
:1076A00006B070BD1CB59D4C217A49B904F1B401F6
:1076B00004F1A400FEF7BCFA606108B9606013BD74
:1076C000022063692072187910B1012813D024E0D8
:1076D00098695A69121AB2F5805F09D29208012A94
:1076E00098BF0122D9681B694118C01829DF06E03C
:1076F0004FF48062F6E7D8681969081828DF10B1DE
:10770000112807D009E0207CB0B9BDE81C40002159
:1077100002209FE00120207213BD60690321FFF762
:1077200093FF00202072606004F1B40104F1A40012
:10773000BDE81C40FEF7A6BA13BD10B5774C201D5E
:10774000FEF7F8FD002804BF607C002802D1BDE8E8
:107750001040A7E710BD000010B500BF71A16F4C2D
:1077600041602046FEF7E6FD50B9F9F743FD20746D
:107770001C238C2204F1180104F1A400FEF7E6F9A1
:10778000002010BD10B5654C14212046F7F7BCFF52
:1077900004F1A400FEF7F2F9002010BD2DE9FC472A
:1077A00006460D46DFF8788192469946694640467E
:1077B000FEF706FA040008BF042013D00A9F1C211C
:1077C000FCF7D0F9002020712660A7602561C4F87D
:1077D0000CA0C4F8149069464046FEF719FAFFF76A
:1077E000ACFF0020BDE8F68780B510461A46F4F7D6
:1077F000ADF8002002BD2DE9F84381460F46DFF8C1
:10780000208115461E4669464046FEF7D9F9040018
:1078100008BF042011D01C21FCF7A4F9012020711D
:10782000C4F80090A6603F0BE7606561694640467A
:10783000FEF7EEF9FFF781FF0020BDE8F28308466E
:107840007047002070473548017A481E8041C04388
:10785000C00F70471CB5022818BF032843D12F4C16
:10786000217A00293FD0022934D1022802D00328EE
:107870001ED02FE060690021E160017959B1012932
:1078800028D10169491C01614069814222D100204F
:107890002072002115E081694269531AB3F5805FB7
:1078A00088BF4FF4805359189142816112D1EEE79D
:1078B000E068401C0928E0600CD30020E0602072E2
:1078C0000D216069FFF7C0FE04F1B40104F1A400CA
:1078D000FEF7D8F9607C10B9BDE81340E2E6BDE8D8
:1078E0001340F9F77CBC13BD0C4801214174007AA8
:1078F000401E8041C00F7047012882B004D1074963
:1079000000204874012004E0032805D10349002029
:107910004874087402B0C5E602B07047C058002031
:107920006459002000100000040000000100000065
:10793000BFF34F8F7E497F480A6802F4E06202433A
:107940000A60BFF34F8F00BFFDE7F8B57E487F4A5E
:10795000016811F1010F08BF1178062905D17C4992
:107960000B68C3F304217B4B19601378062B02BF0D
:107970009168C1F30311032902D1774B774919604C
:1079800003687749774C13F1010F08BF1378062B72
:1079900003D12368C3F342334B601578724B062D35
:1079A00002BF9568C5F30315032D03D15D6F25F064
:1079B00080755D67056815F1010F08BF1578062D04
:1079C00004D16A4D00262E606E600E601578062D7B
:1079D00001BF9568C5F30315032D8D661578062D37
:1079E00002BF9568C5F30315032D08D1604D052628
:1079F0002E600126AE670026AE603F266E600568E9
:107A000015F1010F03BF15789668C6F30316466893
:107A1000062D26D1F61E012E23D9564E564D376817
:107A20002F6077686F60B768AF60F768EF6037699D
:107A30002F6177696F61B7692F62F7696F62376A83
:107A4000AF62776AEF62B76A2F63F76A6F63376B6B
:107A50002F64776B6F64B76BAF64F76BEF64366C52
:107A60002E65056815F1010F08BF1578062D04D1A4
:107A70006469424D04F04F042C60046814F1010F56
:107A800008BF1478062C06D13D4A1468E50744BFA8
:107A90006FF0010515600268062A08D14468E41EEB
:107AA000022C04D9374A146844F4806414601A68BC
:107AB00042F470021A60BFF34F8FBFF36F8F0368F9
:107AC000314A062B05D14068C01E032884BF906848
:107AD0000862D068194B184CC10709D501212160F3
:107AE00018680028FCD0D5686D086D00D56011E0DD
:107AF000116800295CBF5068002815D5012121605C
:107B000019680029FCD01520106018680028FCD0E6
:107B10001521516019680029FCD0002020601868E8
:107B20000028FCD0FFF704FF054806490160F1BDBD
:107B30000CED00E00400FA0504E5014000E401401A
:107B4000543600200090D00330010010E00F00F008
:107B5000240300104035014074C007400DF0ADBA59
:107B6000380500404402001088ED00E00C010040A0
:107B7000105600400404001020C50040E40E0040F0
:107B8000000400403C170040001200102DE9F04FA7
:107B900089B0044600680293CDE9041200F0D7F8DA
:107BA000049B5A1C00EB820650F822301E44A36846
:107BB0000393236903EB82034FF0180853F8047C06
:107BC000039B304608FB073700F0CBF84FF0000965
:107BD00006900621304600F0D1F80546002800F056
:107BE000AF800368994580F0AA8009F10109226AF3
:107BF00050F8293008FB03739968013100D19A606D
:107C0000DA60E6E7236A03F10108C4F820800A215C
:107C1000304600F0BCF810B133183058184405F164
:107C2000010A00EB8A0B50F82A309B4400230821FC
:107C30005846079300F0A2F8079B002841D1129BF9
:107C4000059A00935946029B204600F0A8F80022AE
:107C500006215846079200F091F8079A034600283B
:107C60003FD108215846079300F088F8079B002869
:107C700044D1039A6369DDF808E0E06909FB032356
:107C8000059A0EEB800CE64543D15546069B9D4276
:107C9000B8D100254FF018080821304600F06EF8E2
:107CA000002850D003689D424DD20135226A50F819
:107CB000253008FB03739968013100D19A60DA60BE
:107CC000EAE702689342BAD2013350F8232009FB55
:107CD000027291680131AAD1C2F80880A7E7002397
:107CE000BFE701688A42FAD2013250F82230002BF5
:107CF000AEDB09FB0373216AD960A9E702689342EE
:107D0000B7D20133216A50F8232009FB0272D160F7
:107D1000A7E75068A8420DD190680499884209D11C
:107D20001068C3E9000E9868013008BFC3F80880E6
:107D3000206AD86018330C320EF1040EA3E7002538
:107D40004FF01809A2E7002009B0BDE8F08F10B588
:107D50000821044600F01BF810B1231820581844DD
:107D600010BD0368C31A1A880A2A05D95B89C2188C
:107D700013B1C358D05870470020704710B504465F
:107D800000F005F810B123182058184410BD0368FE
:107D9000C01A03888B428CBF405A002070472DE9DF
:107DA000F3470468DDF8289006460D462046062174
:107DB00017469846FFF7EBFF00284CD023182058B1
:107DC00003EB000A04212846FFF7E1FF00B1285821
:107DD000441C0AEB84005AF8243000220A2118447B
:107DE00000F05AF877284DD0812836D0762843D134
:107DF000284600F05AF85C2849D1284600F05BF884
:107E0000054600220421284600F046F800220446D8
:107E10000621284600F040F8621C05460BD0336A64
:107E2000013333623A46CDF800904346214630464E
:107E3000FFF7ACFE08BB6B1C1ED0336A0133336204
:107E40003A46434629463046CDF8289002B0BDE870
:107E5000F047FFF79BBE8246B4E7284600F025F8BE
:107E600067280DD1284600F026F80421002200F0F2
:107E700013F8411C04460CD1002002B0BDE8F08785
:107E80000020F2E7284600F010F85D28B4E700254E
:107E9000B7E74FF0FF35C2E738B505461446FFF7A0
:107EA00076FF00B12C58204638BD08B500220A21C3
:107EB00000F00BF808BD10B50C210446FFF767FF72
:107EC00010B123182058184410BD38B50546144683
:107ED000FFF75DFF00B12C5C204638BD00000000BC
:107EE000010001000000000001000000000000008F
:107EF0000200050001000000220000000000000058
:107F00000000000000000000000000000000000071
:107F1000010001000000000001000000000000005E
:107F20000200050001000000420000000000000007
:107F30000000000000000000000000000000000041
:107F4000010011000400FCFF04000000000000001C
:107F5000020011000400FCFF04000000000000000B
:107F6000030021000400FCFF0400100000000000DA
:107F7000040011000100FFFF0100000000000000EC
:107F8000050011000200FEFF0400000000000000D8
:107F9000060011000400FCFF0400000000000000C7
:107FA000070011000400FCFF0400000000000000B6
:107FB000080017000200FEFF24000000E07E02001F
:107FC000090010000100FFFF01000000DC7E02003C
:107FD0000A0027000200FEFF44000300107F020099
:107FE0000000000000000000000000000000000091
:107FF000010011000100FFFF01000000000000006F
:10800000020017000200FEFF64010000407F020032
:108010000000000000000000000000000000000060
:10802000010007000000000068010000F07F02006E
:10803000020001000000000001000000000000003C
:1080400003000500010000004200000000000000E5
:108050000000000000000000000000000000000020
:10806000010017000400FCFF68010000F07F02001F
:10807000020017000400FCFFAC0100002080020099
:1080800000000000000000000000000000000000F0
:108090002DE9F04F06468BB04FF0000A06F1700054
:1080A00000F0D0F8504502DC4FF0000B59E0356885
:1080B0002846FFF74CFE0AF1010300EB830250F85B
:1080C00023300621D31828460093FFF760FE0446AC
:1080D00010B12C582B181C44F06EC068C046039099
:1080E0000098FFF73EFE4FEACA0304900193002771
:1080F000049B9F4202D10AF1010ACFE700980A21AE
:10810000FFF745FE20B1009B009A03441058184425
:10811000013700EB870550F827301D44042128461D
:10812000FFF735FE00B128582368834240F287806C
:10813000013004EB800854F82030019A71689844AB
:10814000D6F880304FEA47199A58A9F120094A44D5
:108150001C32404600F07CF8834630B1404600F0C7
:108160009FF858460BB0BDE8F08FD6F88030019AE2
:108170009B584B44DB69002B61D0D3F814800990E5
:10818000B8F1200F4FF00E01284646D1FFF7FFFD52
:1081900000283AD14FF0000BCDF808B00621284650
:1081A000FFF7ECFDC046C046082105902846FFF7C2
:1081B000E5FDC046C046019AD6F8803006909B582F
:1081C000079303EB09081C220021404600F07EF8CB
:1081D000079B059A43F80920069BC8F80430099BC1
:1081E000C8F81030029B1421C8E9053B2846FFF768
:1081F000C5FD00283FF47CAF0368002B3FF478AF47
:10820000C046C046C8F8080072E72B582A18D11893
:10821000043152F803B00291C0E7FFF7B8FD70B91E
:108220007068036841469B68984740B1039A09AB60
:10823000294600F055F883460028ABD091E74FF06F
:10824000010B8EE708B58068FFF781FD006808BD67
:10825000002370B513600C460546164600F020F862
:10826000CD2801461ADC202808D0236820461B6848
:1082700098473060B0FA80F0400970BD2B68EB1A67
:108280001A88062A0AD9DB88E9183BB1EB5822681C
:1082900004335268194420469047EAE70120ECE78E
:1082A0000168411A02460B880A2B09D94B8903B190
:1082B000C358888800B110569842B8BF1846704716
:1082C000042B4FF00003F4D81846F5E710B5044628
:1082D00010460A4601462046FDF7E4FC204610BD44
:1082E0002DE9F0410D46044616461F4600F008F8F9
:1082F0003B46014632462846A446BDE8F041604769
:10830000044B1A681AB9044A044911601A601868C3
:10831000704700BF745E0020785E002038A2020023
:108320002DE9F04F9946436891B0CDE90713054612
:108330000023884681690F9307A8174600F0C9F803
:10834000044600285FD1059005A907A800F002F9AE
:108350000446002857D10646A7F1040A4046FFF715
:10836000F6FC0268059B96423ED33A46194607A89A
:1083700000F058F90446002845D1284600F0E5F9F8
:108380002146024600974B4607A8FFF7FFFB04462D
:10839000002838D16868036810211B6BDDE9097A71
:1083A000984706466868036810229B6831469847DC
:1083B0008046002800F08B80286903683246DB691C
:1083C00041469847D5F810B03E46A146CA451ED151
:1083D0006868D5F810B003685B6A98470026814644
:1083E00031464FF0FF3349E001362A6850F8261035
:1083F000146B5AF8362000EB860C61442846A047DF
:1084000004460028AAD0204611B0BDE8F08F337D85
:108410001BB909F101091836D8E71021306800F0BE
:1084200098F93269531C0146DBF8003008D19C688A
:108430005846D6E90223A04704460028E9D0E2E7DF
:108440000092DC685846D6E90223A047F4E73A7D5B
:1084500092B1DBF8002006939469039106AA58466E
:10846000A04704460028CED1069A786803994A446A
:10847000026001314FF0FF3301361837B245E6D1C3
:1084800007A800F06DF9686803684146DB68984703
:10849000686803685B69984704460028B3D1686838
:1084A000E96903681B6A984704460028ABD128692C
:1084B00003681B6998472B6A834238BF2862686843
:1084C000296A036810229B6A984704469BE70124A7
:1084D00099E72DE9F843044600688846FFF737FC22
:1084E000636801681A688900956818460422A847DD
:1084F0000746206160B30026D4F800903546484610
:10850000FFF725FC03689E4212D36068C4F81C8004
:108510000368C4E90555182145449B68E5600422B9
:1085200069439847A060B0FA80F04009BDE8F8833D
:1085300047F826504846FFF70AFC013600EB860252
:1085400050F82600104400F019F903681D44D6E7DE
:108550000120EBE72DE9F0470568074688462846E5
:108560001021FFF714FC10B90020BDE8F087DFF8F8
:10857000B090002610212846FFF709FC00284DD0B6
:108580002B582A18D118D3589E42EDD2013601EB50
:10859000860A51F826309A4404215046FFF7F7FB2B
:1085A0000028E7D00AEB00025AF80030D458D0185F
:1085B000172C2246494628BF1722043000F0E8F85D
:1085C0000028D7D1172CD5D10C212846FFF7DFFB87
:1085D000044610B12C582B181C4406215046FFF7B6
:1085E000D6FB08B15AF80000431C04EB830254F890
:1085F0002340144404212046FFF7C9FB60B12258F0
:1086000023181344103353F8042CC8F80030BB6906
:108610009A42AFD00120A8E7C368FFDE0368FCE7F9
:10862000D0A102002DE9F04F85B0836800930025AA
:10863000131F04460191AA4602934FF0FF3B2068A6
:10864000FFF785FB03689D4211D363690099E069D8
:10865000182202FB0313012400224FF0FF31904245
:1086600003F1180369D1002005B0BDE8F08F013592
:1086700000EB850850F825309844029B53F835608C
:10868000236903EB850332464146204653F8047CB8
:1086900000F092F80028E7D1009B182101FB073970
:1086A0000746404600F06AF803689F42C7D2C9F8FF
:1086B00004604946304600F0BCF80028D4D1336845
:1086C000C9E902BB013763BB4046039300F056F88B
:1086D00000EB870C50F82700604400F0C4F8039BBF
:1086E00020B9D9F80030003B18BF012389F81430B5
:1086F000019BFBB153F82A30C9F810304046039370
:1087000000F03CF800EB870C50F82700604400F0C4
:10871000AAF8039B38B90AF1010A09F118090C36C5
:10872000BFE70346E2E70133F5D04FF0010389F8D4
:108730001430F0E7C9F810B0EFE743E9041103F88B
:10874000044C43F8081C013289E7C069042100F099
:1087500095B8431E0B44B3FBF1F301FB03F07047E4
:1087600010B504464068A1680368DB6898476068F4
:1087700021690368DB689847002010BD10B504210B
:108780000446FFF704FB10B123182058184410BD0D
:1087900004E010F8013B6BB1491C521E52B10B783A
:1087A00090F800C09C45F4D002D24FF0FF307047E3
:1087B00001207047002070472DE9F34708460C461A
:1087C0001646FFF7CEFA4FF0000805464FF0FF3788
:1087D000A84501D1002029E00A212046FFF7D7FA59
:1087E00010B123182058184408F1010800EB88093B
:1087F00050F828304FF0000A994414214846FFF7FA
:10880000BDFA0028E4D003689A45E1D20AF1010AD2
:1088100001A950F82A3001970C2000FB036000F0FA
:1088200008F818B9019B002BE7D0012002B0BDE881
:10883000F087436873B50D469BB119680022012487
:10884000914209DC007A01A900F01EF810B9019BE1
:1088500063432B6002B070BD53F8046F0132744360
:10886000EEE70124EEE710B50E210446FFF78FFA7C
:1088700000B1205C003818BF012010BD4B1E184409
:10888000B0FBF1F048437047122804D8092804D8F7
:10889000022824D858BB012070470A380828FAD883
:1088A00001A353F820F000BFD7880200F38802002C
:1088B000F7880200F3880200EF8802009788020020
:1088C000EF88020097880200EB88020012F4887F8C
:1088D0000FD10728DFD102230B600020704701234E
:1088E00003FA00F212F4127FF0D00123F4E704231C
:1088F000F2E70823F0E71023EEE700BF2DE9F04F81
:10890000016887B00546C06E00F0CEF8014638B960
:10891000012385F891300124204607B0BDE8F08F8F
:1089200005F1700738460161C0462846FFF7B0FBE5
:1089300004460028F0D105F1A00601463046016149
:10894000C046384600F0ECF804460028E4D1012186
:1089500030460161C046384600F013F9044600284D
:10896000DAD1022130460161C046D5F8802029685D
:10897000E86E05F1940300F034F904460028CBD1E9
:10898000D5F8941030464161C046EF6E28683B68C8
:10899000D3F81C8000F041F981003846C047C5F883
:1089A00098000028B7D0A34625E0D5F880201B68A2
:1089B000049238460393FFF7CAF94368043306214B
:1089C0001844FFF7DBF90134D5F898A0CDF800B0D2
:1089D00050F82430049A39464846039FB8474FEA76
:1089E0008408A8F10408D5F898304AF8080053F82C
:1089F0000830002B8FD02F68384600F00EF9D5F8DC
:108A00006C90A042D9F80030CFD83846DC6900F02D
:108A10000FF981004846A047C5F89C0000283FF4A4
:108A20007AAF0024A346D5F80080404600F000F954
:108A3000A0420ED8284600F006F9044600287FF42C
:108A40006BAF012385F89030032130460161C046A9
:108A500062E7D5F86C90D5F88020D9F800300592FF
:108A60001B6804934046FFF772F9436804330821FA
:108A70001844FFF783F90134A700D5F89CA0CDF87E
:108A800000B03B1F059A0393049F50F824304146E1
:108A90004846B847039B039A4AF80300D5F89C3030
:108AA0009B58002BBFD136E7F8B5037D04460E4630
:108AB00013B100252846F8BD0123037580680368BB
:108AC00004229B6808219847A368144AC0E9002340
:108AD000E060204600F0C4F80028EAD1A5682B68C1
:108AE00030469F68FFF733F9016804222846C90021
:108AF000B84705460028DCD023680246DB6A3146C9
:108B0000204698470028D4D123682A469B6A3146DC
:108B1000204698470028CDD0CBE700BFF0A1020047
:108B20002DE9F047D0F8149004460026E3691B684D
:108B30009E4204D3C4F814900020BDE8F087A068DA
:108B40006661314600F09BF84FEAC60A804600276E
:108B5000474501D10136E9E7236953F80A5005EB8F
:108B60004715D5E90410EB695A691B68202A06BF2E
:108B7000AA690146002213B160689847E86001378E
:108B8000E6E72DE9F843D0F8148004460025E369B0
:108B90001B689D4204D3C4F814800020BDE8F8830C
:108BA000A0686561294600F06AF84FEAC5090746E2
:108BB0000026B74201D10135E9E7236953F80910CE
:108BC00001EB4611CB699B682BB93146E06800F098
:108BD0006AF80136EDE7606898470028F5D0012073
:108BE000DCE72DE9F0411D46037D04460E4617469D
:108BF0008BB1036882691B6C2946984748B9236882
:108C00003A46D3F83C802B6831462046C04700B92D
:108C10002075BDE8F0810120FBE708B5FFF797F864
:108C20004368043306211844FFF7A8F8006808BD1C
:108C300008B5FFF78CF84368043308211844FFF7A0
:108C40009DF8006808BD10B500F17004204600F0E2
:108C50004BF820B92046BDE8104000F06FB810BDB9
:108C6000002310B5044683614068036804229B69B1
:108C700090219847E061B0FA80F0400910BD036888
:108C8000C31A1A88082A0CD91B89C2180BB1C358F9
:108C90001344013103EB810053F821301844FFF7EE
:108CA00060B80023F5E7036870B55B6904460D46BC
:108CB0009847C0B92046FFF748FDA2690C235A43E4
:108CC0008318984209D16068E1690368DD699032D0
:108CD000AC460423BDE8704060474168013108BFDD
:108CE00045600C30EDE770BD2DE9F843D0F81480F5
:108CF00004460025E3691B689D4204D3C4F8148030
:108D00000020BDE8F883A06865612946FFF7B7FF3A
:108D10004FEAC50907460026BE4201D10135E9E701
:108D2000236953F8093003EB4613DA6922B112695B
:108D300012B1D968606890470136EDE72DE9F04F30
:108D4000054685B000264FF00C0BEB691A68964279
:108D500007D3A869002863D10023184605B0BDE8F1
:108D6000F08F013603EB860853F826304FEAC60928
:108D70009844A9F10809002704214046FFF707F8A5
:108D8000002853D058F8003008EB0002D118D3580F
:108D90009F42DAD2013701EB870451F827301C4497
:108DA0000E212046FEF7F3FF0028E5D0235C002BC0
:108DB000E2D02B694B440BFB07FA5868AAF10C0A66
:108DC00003A95044FFF735FD03460028C5D10190A3
:108DD00006212046FEF7DBFF0146A0B12256019B8B
:108DE000092A1BD10C212046FEF7D1FFA0B1231880
:108DF00024581C440A212046FEF7C9FF98B1225886
:108E00002318134459682B69039A4B445B6853F841
:108E10000A00FFF75BFAAFE70446EBE71946F2E713
:108E200000F006F898E743688368FFDE0368FCE714
:108E300070B5054600241426AB68A34201DC00206F
:108E400070BD2B6806FB04330134DA6893F9101007
:108E50009868FFF73BFAEFE72DE9F04F85B01C4625
:108E60000F9D80468A469346002120222846FFF720
:108E70002DFA204600F0B4F805F11C0100F0B8F816
:108E80000746002850D12046FFF7EDFC0E99A87741
:108E9000204600F0B9F8002814BF012302232861FE
:108EA0006B7703AA05F11801204600F0C7F80746C2
:108EB000002839D104212046FEF769FF002837D069
:108EC000221820581044C046C04668610C21204634
:108ED000FEF75DFF40B3235826181E44304600F0CD
:108EE000E0F8044600B30368F3B1304600F0E3F85D
:108EF000D0B10368C3B16368AB60304600F0DBF803
:108F00004368EB60304600F0CCF8D0F80090BBF13D
:108F1000000F0FD0DAF8003004229B680C21504675
:108F200098470446E0B90127384605B0BDE8F08F00
:108F30002A48CAE7D8F8003004229B680C21404632
:108F4000984704460028EED0D8F800304846D3F8B9
:108F500008A001308000042201464046D0470AE0C4
:108F6000DAF800304846D3F8088001308000042247
:108F700001465046C04760600028D4D0304600F01B
:108F800090F8C046C046636820609A46C3F80090D7
:108F90004FF0000BD9450ADC10213046FEF7F7FEF2
:108FA00000B13058A06001232B706C60BCE73046E4
:108FB00000F081F8026801928046304600F071F8B6
:108FC000019A03689A4208BF08EBCB080BF1010B2A
:108FD000D8F804304AF8043FDCE700BFCCA3020015
:108FE00010B506210446FEF7D2FE00B1205610BD92
:108FF00038B504460D46FFF783F929460246204658
:10900000BDE8384000F061B838B50D460821044687
:10901000FEF7BDFE00B12058013005EB800455F885
:1090200020301C4404212046FEF7B1FE28B123580D
:109030002218D118D05800B1081D38BDF7B5144614
:109040000268821A03461788042F0D4626D9918894
:10905000461809B3405831183058012601EB8000FA
:10906000814214D1062F1AD9D08800B118560DF1BB
:109070000701FFF7BDFF40B99DF807002146FFF744
:1090800003FC10B9236873432B6003B0F0BD51F8A3
:1090900004CF0CFB06F6E3E70126E3E701260020F8
:1090A000E5E710B508210446FEF771FE10B123185C
:1090B0002058184410BD10B50A210446FEF767FE7B
:1090C00010B123182058184410BD11282DD8DFE8FE
:1090D00000F0093012161A1E200E22180C241C262D
:1090E0002814102A0123002021E00B23FBE707238B
:1090F000F9E71123F7E70223F5E71023F3E703234A
:10910000F1E70923EFE70423EDE70D23EBE7052360
:10911000E9E70623E7E70823E5E70C23E3E70E2367
:10912000E1E70F23DFE71223DDE7002301200B70C7
:1091300070470A23D7E72DE9F04F90F8283085B023
:1091400004469BB385688DB3D0E90467002380F89B
:1091500028301A46D4F808C09C454FEA820E06EB28
:10916000820007EB820124DCACEB020200F09EF8E7
:1091700001230022C4E90732A669D4F80C80D4F890
:1091800024B04FF0FF33B3603B68736008EB03110A
:10919000B1464968013108BF4BF823205BF8233002
:1091A00033604FF0010AA368534525DC05B0BDE8E4
:1091B000F08FD4F80C80D4F8249008EB031C18012D
:1091C000DCF8041058F80000B1F1FF3F1CBF46F86E
:1091D0000E0047F80E304FEA83080BBF05F1FF354C
:1091E000DCF8041046F82500013208BF47F82530A6
:1091F00049F808100133ADE757F82A300093009A78
:109200001B0108EB021158F803300193D1E9022346
:109210004D6802936B1C19D100200546014603904E
:10922000029B204600F05FF8039949B14B6809683A
:109230004FEA031C58F80CC08C446545B8BF65461E
:1092400020B10168019B491B8B42E7DC009B4BF876
:109250002350E1690C234B43F218F550009B5360F7
:109260004B1CE361D9F80030AB4206DD236A936002
:1092700021620AF1010A914695E74846D0F808C0F4
:10928000BCF1FF3F06D18160C2F808C04A46F0E752
:109290007046F3E70C2303FB0CF306EB030EF358C5
:1092A000AB42F5DDC2F808C08160EFE7F0B50346D8
:1092B0000C4601250026954202DB002EF7D1F0BDB9
:1092C000D3E9007C6745BCBFC3E900C7D4E90067A8
:1092D00005F10105B8BFC4E9007603F10403B8BF86
:1092E00001260434E7E770B5054689B9016AAC691F
:1092F0000C2000FB01440C262146284600F010F803
:1093000050B9A1684C1C09D0AC6906FB0144F3E7D5
:1093100089684E1CEBD10024204670BD0446FBE753
:1093200010B54C68C16801EB04118868984205DCEF
:10933000C8689042B4BF0020012010BD0020FCE7A7
:1093400080B51F49012081F80401FAF7D7FF0028F2
:1093500004D40020FAF7D6FF002002BD4FF0FF3002
:1093600002BD80B50320F6F7C7FF002002BD80B51F
:1093700014480168B1F5967F00D2EFE7104890F8E5
:10938000041101290CBF01200420F7F7DEFD0E496E
:1093900002200880002002BD80B5F6F781FD002084
:1093A00002BD000080B5074800210176D0F800100A
:1093B00006A0F4F720F9FAF7A9FF002002BD00008B
:1093C000F4370020B8350020AC360020256420207A
:1093D000747269676765722C20656E61626C656482
:1093E0002E0D0A002DE9F74F80460D46019200240C
:1093F0002846FEF7ACFC03689C4201D3002017E02E
:10940000013400EB840750F82430FB181846009311
:10941000FFF7B4F9D0F800A0D8F8080003680C21D1
:109420009B68042201FB0AF19847064618B90120FF
:1094300003B0BDE8F08F07464FF0000BDA4504D1CA
:10944000019B043B43F83460D2E70098FFF796F99C
:109450000BF1010B00EB8B0950F82B1028468944C7
:109460000C21FEF794FC50B12918285801443A46C3
:10947000484600F007F80C370028DFD0D7E7014650
:10948000F5E7FEE7F8B516460023C2E9003346F8D3
:10949000083F0F4614460546FFF7A2FD3146FFF789
:1094A000A7FD064658B939462846FFF7ADFD042109
:1094B00020602846FEF76BFC18B9054B6360304608
:1094C000F8BD2A1828581044C046C0466060F6E728
:1094D000CCA302007365740073686F77000000000E
:1094E00064667500646E74006578636C65616E0017
:1094F000636C65616E0000007374657200000000AB
:1095000064756D7000000000726573657400000082
:10951000737461727400000074657374000000005D
:10952000656E61626C65000064697361626C650000
:10953000777269746500000066697265000000005A
:1095400068656C7000000000F7B500F1080704467C
:109550001E46C0E900120D46642200213846FEF77F
:10956000B5FE9DF82C200899304600F022F804F151
:109570007006099AE0660346009239462A4630464C
:1095800000F042F820464FF48073A4F89030002396
:10959000C4E9253350F8A02BE16EC4F89C30334663
:1095A00000F048F820460A9900F052F8204603B02F
:1095B000F0BD70B50D46102104461646FFF75EF962
:1095C0002C44211A00F070F8054600B1043086B131
:1095D000012E17D1036804229B6841F20C019847C1
:1095E000044600F085F821462846BDE8704000F0AA
:1095F00089B8036804229B682C219847044600F030
:1096000097F8F0E70024EEE710B504461046C4E9E9
:109610000203074A0023C4E90433029BA361C4E99F
:10962000002110B1FEF793FBE061204610BD00BFA2
:10963000D89C020030B5054DC0E902320023C0E9D4
:109640000051C0E90433836130BD00BF589D020062
:1096500070B500F1A00604460D46304600210161B8
:10966000C0460A4BE3610A4BA3650A4BE3650A4B0C
:10967000A3640A4B23630A4B23640A4BE36400236D
:109680006661E56384F8913070BD00BF9FBE010044
:109690002DA302005DA302007DA302006DA30200C2
:1096A00075A3020065A3020000B58BB00A4601460F
:1096B00001A800F043F804220DEB0200242100F081
:1096C00044F80A4A026044324260039A8260049A73
:1096D000C260059A0261069A4261079A8261089AFD
:1096E000C261099A02620BB05DF804FBA09A020005
:1096F000034A026000F580530022C3E9012270474B
:109700000C9F020038B503680D465B6B04222421D0
:1097100004469847054A0561C0E900240022043444
:10972000C0E9062284600275026238BDFC9B02001B
:10973000014B0360704700BFDC9E020008B50A447D
:10974000034600F011F8184608BD10B504464069FC
:109750000B46C01A114600F017F82369834294BFE4
:109760006061002010BDFEE710B5064C0460C0E942
:109770000321C0E9052144340022C0E90141C0E9C8
:10978000072210BDA09A0200B0FBF1F048437047D9
:109790002DE9F74307460E461D4614464FF00009D3
:1097A0003046FEF7EBFF03684B4501D800201CE074
:1097B00009F1010800EB880250F828001044FFF777
:1097C00052F8A8B11DB155F82930013310D101A9C3
:1097D0002046FFF72EF840B9B868019903681022B7
:1097E0009B689847206018B9012003B0BDE8F0835A
:1097F000C1460C34D4E7FEE700F030B808B1016888
:1098000008447047F0B5044685B00D4616461F461D
:10981000BC2000F025F848B100210391029101918C
:10982000009733462A462146FFF78EFE05B0F0BD6D
:10983000FFF764B8002100F025B8002100F030B82F
:1098400000F03CB8002800D1704700B581B000F0AE
:109850004BF801B05DF804EB00F059B87047FEE733
:1098600010B5044601E000F057F82046F0F75AFB27
:1098700028B9034800680028F5D08047F5E710BDF7
:10988000685E002038B5054600680C46FFF7C5F94C
:10989000A0428ABFD5F89830002053F8240038BD84
:1098A00038B5054600680C46FFF7C2F9A0428ABFEA
:1098B000D5F89C30002053F8240038BD90F8913042
:1098C00010B5044673B990F8903033B104F17000CC
:1098D0000021BDE8104000F021B8FFF70FF8002884
:1098E000F4D010BD0120FCE738B5D0F88030044634
:1098F00000F1700513B1284600F041F804F1A00012
:10990000C046C0462846C046C046204638BD00284E
:1099100018BF00F05EB87047F0F7DCBEC3691B6883
:1099200099422DE9F047D0F81480416104460E4673
:1099300004D34FF0010A5046BDE8F0878068FFF776
:109940009EF9F600814600274F4504D1C4F81480E3
:109950004FF0000AEFE723696068995901EB47115E
:10996000CB69DB68984705468246E06803685B6917
:109970009847012DDDD0002DDDD10137E4E72DE939
:10998000F843D0F8148004460025E3691B689D4223
:1099900004D3C4F814800020BDE8F883A068656192
:1099A0002946FFF76CF94FEAC50907460026BE4273
:1099B00001D10135E9E7236953F8093003EB461378
:1099C000DA6922B1526812B1D968606890470136ED
:1099D000EDE7F0F702BCFEE716480168491C0529CF
:1099E00082B0016013D28C22B1FBF2F28C2000FB1A
:1099F0001211092902D102B0F6F731BA132902D1A6
:109A000002B0F6F72EBA4F2909D059290BE04622A9
:109A1000B1FBF2F2462000FB1211092902D102B07B
:109A2000F6F724BA132902D102B0F6F721BA02B030
:109A3000704700BF605E00202DE9F047D0E9017655
:109A4000084689461C461546FEF781F9089B9DF895
:109A50002480013300EB830250F823001044FEF70A
:109A60008DFE631C00EB830450F823300C21484624
:109A70001C44FEF78CF920B109EB000359F80000F3
:109A80001844CDE908052346424639463046BDE82C
:109A9000F047FFF7E1B9FEE700000000000000001A
:109AA00031A4020031A40200959F0200DBBE010038
:109AB0003BBC010001A20200659F02008D9D0200D7
:109AC000EFBD0100FDA302000FA00200ADA2020045
:109AD0009FA102004B97020085A30200FCFFFFFF3D
:109AE0000000000005A4020001A402008DA30200F2
:109AF00095A302002DE9F34707464068DDF828905A
:109B00001D46036888469B68202116460422984714
:109B100001223B68CDE900920446D3F838A0024602
:109B20002B4641463846D04770B94EB106EBC906C0
:109B30000C235D4373685A195B5923615368636151
:109B4000204602B0BDE8F0870024F9E72DE9F3478D
:109B50001D460368DDF828905B6B0746884616466D
:109B60009847044620B90024204602B0BDE8F0879B
:109B700000223B68CDE900924146D3F838A0024666
:109B80002B463846D0470028EDD1002EECD006EB0E
:109B9000C9060C235D4373685A195B5923615368E6
:109BA0006361E1E72DE9F8430546894690461F4683
:109BB000FEF7CBFDA9690C264E43044600EB060CCC
:109BC000002264450ED10B2A12D84FF0FF3340F823
:109BD0000690C4E901383960AB690133AB610020FC
:109BE000BDE8F8836368013308BF01320C34E8E74D
:109BF0000120F5E700000000000000004D9B02007E
:109C0000F59A020023B70100FDA2020005A302009D
:109C100015A302000DA3020067C0010023A40200E7
:109C200023A40200419C0200E593020091970200E8
:109C3000E9A20200399A0200218302004BA102002E
:109C40002DE9F04106460D460024A2F108072846FA
:109C5000FEF77DF803689C4202D30020BDE8F08146
:109C6000013400EB840250F824001044FEF779F828
:109C7000B3681A684101D2F8088018460422C04728
:109C800010B147F83400E2E70120E7E71FB500BF55
:109C90000CA40EE0052818BFF6F7A0FB1FBD516805
:109CA00000981268904701A8FAF7C0FA039A002AB0
:109CB000F5D168464BDF0028ECD1214601A8FAF720
:109CC000A4FAF3E77CA202008CA2020008000000C4
:109CD00000000000000000002DA402002DA40200DE
:109CE0001D990200CDA00200039E0200EDA002001B
:109CF000399E020045820200E9A30200218B020086
:109D0000838B0200E98C02007F9902003D8D0200E6
:109D100019E050F8042BD30744BFA9F101039A18A6
:109D2000091F0023042942F8043BF9D25FEA817C31
:109D3000134604D54FF0000CA2F800C09B1CC907C5
:109D400044BF0021197050F8041B0029E1D170476D
:109D500000000000000000002FA402002FA4020059
:109D60004DA3020059A2020035A3020083A1020004
:109D700055A302003DA3020045A3020045A2020034
:109D80009DA20200EDA30200F1A30200F8B5044673
:109D90000F468068194615461E46FEF76FFD22697C
:109DA000A3699A4201D00120F8BDB842FBD1A06856
:109DB0003146FEF763FD63691B1AAB42F3D32844B7
:109DC0002061A0610020EFE770B50446FFF7B3F90A
:109DD000A06830B1A169236A0C2505FB031300209C
:109DE00003B970BD5A68E6681201B2581E689B68D4
:109DF0003244904238BF10465A1CF2D005FB031380
:109E0000EEE770B5054680680E461446FDF79FFFE5
:109E1000731C00EB830250F8230006211044FDF769
:109E2000ADFF2969013401EBC60150F824204B68CD
:109E30000C2000FB023070BD70B5054680680E46F0
:109E40001446FDF784FF731C00EB830250F82300D7
:109E500008211044FDF792FF2969013401EBC60186
:109E600050F824204B680C2000FB023070BD0346E4
:109E700010B5012483F82840D9602824B2FBF4F2FD
:109E800001EB0211196101EB820159610C2401EB14
:109E900082010020996104FB021198605A605962A6
:109EA00010BDFEE7ACA30200B4A302000000000056
:109EB00000000000BCA30200C4A3020000000000D8
:109EC00000000000CCA20200DCA2020000000000A2
:109ED00000000000000000000000000029A40200B3
:109EE00029A40200359F020067A10200C99D02005B
:109EF000E1A30200E99F02006F9E0200F5A30200A9
:109F0000E5A3020000000000000000002BA40200F6
:109F10002BA4020013B80100DDA3020025A3020058
:109F20001DA302002FB90100D9A30200F9A302006A
:109F300027A40200F0B5D0E90154AC4210DAC6689B
:109F4000270106EB0415F151C5E902234FF0FF3359
:109F50006B6001340123846080F828300020F0BD5C
:109F60000120FCE72DE9F04104460F4680681146C8
:109F70001646FEF783FC23680546D3F81C8001468D
:109F800033463A462046C04700280CBF28460020EA
:109F9000BDE8F08138B504460D4680691146FEF7EC
:109FA0006DFC63691B1AAB4208D3E3694340E3616C
:109FB000236A05440133A561236238BD0020FCE714
:109FC00010B5074979441831064C7C44163404E036
:109FD0000A68081D114488470146A142F8D110BD06
:109FE00078000000A400000070B50C460546164637
:109FF000FFF7A1F8002C08DBAB68A34205DD6B6A14
:10A0000053F824303360002070BD0120FCE72DE9B7
:10A01000F04104460E46806811461546FEF72EFCB8
:10A020002368DF6901462B4632462046BC46BDE820
:10A03000F04160474EF68851CEF20001086840F4C6
:10A0400070000860BFF34F8FBFF36F8F4FF0007049
:10A05000E1EE100A70470000B9FCFFFF94260000F3
:10A06000F4370020000000007306FFFFC703000064
:10A07000C6030000B82A00206306FFFF9A0500000F
:10A0800022000000E0370020FEE700009CA3020051
:10A09000A4A3020018A2020030A20200BCA2020087
:10A0A000CCA20200A4A30200ACA3020059770200D4
:10A0B00085770200E97702009D770200F7770200BA
:10A0C0003F780200437802004778020010B58068AC
:10A0D0000C46FDF73CFE611C00EB810250F82100AC
:10A0E00006211044FDF74AFE006810BD10B58068D7
:10A0F0000C46FDF72CFE611C00EB810250F821009C
:10A1000008211044FDF73AFE006810BD0120C0464A
:10A11000002801D0FFF754FFAFF300800020AFF319
:10A12000008000F002F800F008F880B5FCF7BCFBF6
:10A13000FCF73BFDF9F7A4FFFCE700F001B8FEE7F0
:10A1400007463846F0F71CFBFBE7836910B50C4661
:10A15000114633B18068036804229B6889009847E0
:10A160002060002010BD70B50468A468D0E90265C5
:10A17000A04720B905EB0615049B6B6070BD01205C
:10A18000FCE737B50446D0E901020B465569016882
:10A1900000954D681269E168A84703B030BD70B5FD
:10A1A000044680690E46FEF769FB31460546606944
:10A1B000FFF7EAFA401B70BD00000000000000003D
:10A1C000000000000000000000000000000000008F
:10A1D0004F66666C696E654D656D6F7279416C6C2A
:10A1E0006F636174696F6E00000000000000000082
:10A1F000F5A202001FA4020021A4020021A4020073
:10A20000036810B51B690446984718B12369A36118
:10A21000002010BD0120FCE715140200B05D0020F5
:10A220002D0D0200EC2F0020F308020000000000BA
:10A23000000000000000000025A4020025A4020088
:10A24000D5A302008368D3E9043203EBC2030C20D8
:10A250005B6800FB0130704710B4846840681346A7
:10A2600062695DF8044BFFF79DBCFEE744312D4E5B
:10A2700052462D302E332E3000000000B4A30200D1
:10A28000BCA302000000000000000000014880475D
:10A29000014800474B790200DDA20200034619B1D4
:10A2A000806908B999617047012070470269836825
:10A2B0008069824234BFC01AD01A70478D050200EF
:10A2C000C42F002059040200E02F002025130200B3
:10A2D000000000008D9C020000000000AFF3008031
:10A2E000FFF7A8FEFFF712FF8068036804229B684F
:10A2F00020211847406803689B6818474068036836
:10A300009B68184740680368DB6818474068036823
:10A310001B691847406803685B69184700F580505F
:10A320004068704700F5805080687047C0680368D7
:10A330005B691847436953F8210070474068036818
:10A34000DB681847406803681B6918474068036862
:10A35000DB691847406803689B681847C068036852
:10A360005B6A1847C06803681B691847C0680368C0
:10A37000DB6A1847C06803689B681847C0680368B1
:10A38000DB681847C2684069101A7047A0F10400E2
:10A39000FFF7DBB9A0F10400FFF7F4BFDB590200BF
:10A3A00000000000E7D8010000000000E97802008A
:10A3B000000000005578020000000000F97802005B
:10A3C0000000000000002E004300FEE70000000037
:10A3D0000020704700207047002070470120704720
:10A3E00080687047FEF7A7BE806970478069704734
:10A3F0008068704700207047012070478068704770
:10A400000438704704387047FEE7FEE7FEE7FEE7D2
:10A41000FEE7FEE7FEE7FEE7FEE7FEE7FEE7704742
:10A420007047704770477047704770477047704774
:10A43000704700F20B0001F00557100140110004B5
:10A44000000110021F1C1F1E024105821D0CF2FF9D
:10A450000001F1FF01F1FF01F1EA0112FF01ED300E
:10A460000492FF01611C1C0B6CA20200FC0800009E
:10A470004C5E002001E404FC0104FFFF146704F0BB
:10A4800003FFB82F00200001F1FF01F1FF01F1FFF0
:10A49000011101FC04810100020053444A0430010F
:10A4A000D4940295500351C90100D80C10037BCB02
:10A4B0000100E00C1009010100009FC60100C0D09E
:10A4C00001C010010000710C52E41812D70C22C810
:10A4D00018110C500391C70100E818500357C80128
:10A4E00000F00C12F50C52F80C1305CD0542950C3A
:10A4F00012010C52080C126B0C52100C12850C52EB
:10A50000180C40040B7502002095901291185228E7
:10A510000C12F10C52300C600359CE01003824119A
:10A520000C52403C2359CFAE32000C2101210710C0
:10A53000035FFE01006304312EF401333002408AD0
:10A54000F2120145500332A402000A287001B91E1C
:10A55000023253D1A30C7330008C31507001400093
:10A560004058100290D0031B0C1007B80B0000E9F4
:10A570005E0200250C12C8041003D35F02002F08EE
:10A5800012640412F50C52390C10031360020043DC
:10A5900008100370170000250C52111883316078E1
:10A5A000210192050E8341931C12630C6D060792E4
:10A5B0006F1892990C12A50C400805351500F997F3
:10A5C0000200FD97181003059802003104123504AB
:10A5D000123B04124104C345987431015220ECF738
:10A5E0001C20008016C42CF107046DDC07F200C6A5
:10A5F00014152C110C254CFF055C37C4071003699A
:10A60000B701005D04877DB7CA43C1B80C7401AFC0
:10A61000B801E0126808520001000AED26020000AD
:07A62000900100FFFF07009D
:020000040003F7
:1000000040C000204737040000000000000000004E
:1000100000000000000000000000000000000000E0
:10002000FC8800001C00000054464C3314002000E3
:100030001C001800140010000C0000000800040050
:10004000140000001C00000084000000DC00000020
:10005000708000008080000088880000030000009D
:100060000100000004000000367FFFFF0C000000CC
:100070001C0000003C0000000F0000007365727659
:10008000696E675F64656661756C740001000000ED
:100090000400000098FFFFFF1200000004000000B1
:1000A000080000006F75747075745F310000000007
:1000B00001000000040000001A80FFFF040000009F
:1000C00006000000617267735F30000002000000EC
:1000D0003400000004000000DCFFFFFF15000000FA
:1000E0000400000013000000434F4E564552534990
:1000F0004F4E5F4D455441444154410008000C00AF
:1001000008000400080000001400000004000000C3
:10011000130000006D696E5F72756E74696D655FC6
:1001200076657273696F6E0016000000907F0000A4
:10013000887F0000707F0000507F0000C07E0000BC
:10014000307E0000A07D0000107D00000032000025
:10015000F0210000E0110000D0010000C00000000C
:10016000B8000000B0000000A8000000A0000000DF
:100170009800000090000000880000006800000067
:1001800004000000E680FFFF0400000054000000AF
:100190000C00000008000E00080004000800000029
:1001A0001000000024000000000006000800040009
:1001B00006000000040000000000000000000A002B
:1001C00010000C00080004000A00000002000000FB
:1001D000020000000400000006000000322E313052
:1001E0002E3000004681FFFF0400000010000000D8
:1001F000312E31342E3000000000000000000000DD
:100200005879FFFF5C79FFFF6079FFFF6479FFFF9A
:100210006879FFFF6C79FFFF7079FFFF7E81FFFF38
:100220000400000000010000177C6D3DF80D3E3D0C
:1002300076318D3DACD6843DE2893E3DFAD12D3EEE
:10024000814FC0BDD1BE133EC409A53D806B6BBEBE
:100250008C5787BDA9DF4C3DE7E400BEF175E6BDD4
:100260001D2BFEBDE7821C3D22947E3D07E11E3D15
:10027000138BF6BDBD7853BDAC053CBDA0A3FABD44
:100280000A8050BE6277943D6E7D94BDA81009BD72
:10029000C2216FBDEE09B2BE53FD713DC88665BD7A
:1002A0006DCE25BDF2D48EBE757D6DBDDB0E3EBD1F
:1002B00040318DBD2ED684BDAB8B3EBDD4F8343ECF
:1002C0004750C03D08BE13BE2309A5BD546B6B3E0D
:1002D000FC53873DA0DE4CBD21E5003E2975E63D7F
:1002E000412AFE3D36831CBD1E957EBDE1E11EBD4B
:1002F0004D8FF63D0977533D44053C3DBFA2FA3D85
:1003000023BC5F3ED87794BD9E7C943D1211093D7D
:1003100087216F3D3682AFBD09FD71BDAE86653D5B
:100320001CD0253DB334BDBD8A82FFFF0400000010
:10033000001000000862893D6F4BC8BEA4D15ABDB1
:100340003CC3B0BE1163773EFE349FBF8C67EA3D6D
:1003500066D4BE3DCFADBE3DC760E63EE825D63E85
:10036000F22C303FBF551ABE30A4343F5BF33CBF84
:1003700024D4C4BEE32AF23E7653BD3E00234EBED3
:1003800054E3D6BD4B42B83D3E36F5BE13861E3E05
:10039000ED573ABF5211CE3D226D893DC1AD63BECE
:1003A000FF8BAEBE64EE43B90A58773C3570BCBDD6
:1003B000EE9E16BF122A02BF5DC184BE8A3BB53EC7
:1003C000E506663E99F0F43EAF93B4BE7A26F3BEDE
:1003D000119C12BF2B818BBE674E043FDB87A0BEF2
:1003E0008ABD3E3E5C6681BEFFDDAE3EBEBBF33DD8
:1003F00074BA37BEE172DCBEC2E5983E47018FBEDB
:10040000068A103F2C8E3B3EA63B103F1E3F02BE8D
:10041000242C45BF4C6A003CA079CCBEE05A863FF4
:10042000EA1C4E3E353638BF239142BF8DA0FCBE3C
:100430003E7AF53E437B933EF469F9BDEF449DBDA2
:10044000A0FFA3BEAAC02C3F237E96BF3F85243EBB
:10045000B896A83E030093BE8395EF3E52D5A63EC4
:100460000A6615BF8186B3BEC77596BECD706C3E59
:10047000C38883BF6C1D9FBD6F20A33EA55958BE86
:10048000F80E7BBF5D993B3F831E3DBFA6D9AA3EB8
:10049000278A9A3EF2FCC4BF4262943F4F8D39BF17
:1004A00061EA03BFF9040A3FE298023DF0DD153F1F
:1004B000AF7EB13DE83F3B3F606D793E966326BF1E
:1004C000E5D00B3E8E467FBFC72A0BBF30618BBF86
:1004D000B2EEAE3E3543033F34FFB4BC5F4AB2BE1A
:1004E0009F6A0B3D56C236BF6B1C86BEC715033FC5
:1004F0007EF5B8BE2F62533E1592883F3042373E9C
:100500003B019A3FE4165C3E821875BE8857143E44
:100510001848C1BE93379C3E5834CC3F5CF9CF3E5F
:100520008C35F03E8D6664BE19FC47BFBB84153F19
:100530004AB955BFDC32123EDDF57FBE863F77BE3D
:10054000FBF2733DE09CC1BE389DD4BD7690843EE5
:10055000E194CEBDCEDD3C3E6501733EE00398BD27
:100560006369D8BCEE6DFCBDE04ABBBEBAD00FBE1D
:100570001AF707BEE8E8C2BC6E346C3EE1004A3EA2
:10058000FDBC29BEB9399EBDA2ED1D3EE81AAD3EA7
:1005900020E278BD3D99503E7E91853E1CE53FBDF1
:1005A0004B9915BF18A98B3D6AC2253E10973D3D5A
:1005B00065CE09BF7CD093BAE52A70BB6ECE87BBEF
:1005C000CFF8CCBA219872BC538083BC9F4CDABB65
